:020000040000FA
:10000000084804000100000042F0000042F0000037
:1000100042F0000042F0000042F0000042F0000018
:1000200042F0000042F0000042F0000042F0000008
:1000300042F000005C74000042F0000042F000005A
:1000400042F0000082740000A874000042F000003A
:1000500042F0000042F0000042F0000088CA0000B8
:1000600042F0000042F0000088CD000020C20000F5
:1000700042F00000CAE600007EDF000042F000000F
:1000800042F000001CE7000042F0000042F00000D7
:1000900042F00000DC74000002750000BEDF0000CA
:1000A00042F0000042F0000042F0000042F0000088
:1000B00042F0000042F0000042F0000042F0000078
:1000C00042F0000042F0000042F0000042F0000068
:1000D00042F0000042F00000A4A9000042F000003D
:1000E00042F0000042F0000042F000000ECE00009E
:1000F000B6C2000042F0000042F000009EAC0000DA
:100100000869000042F0000042F0000042F00000E8
:1001100042F0000042F0000042F0000042F0000017
:1001200042F0000042F0000042F0000042F0000007
:1001300042F0000042F0000042F0000042F00000F7
:1001400042F0000042F000008AAC000042F00000E3
:1001500042F0000042F0000042F0000042F00000D7
:1001600042F0000042F0000042F0000042F00000C7
:1001700042F0000042F0000090CE00004CC30000AE
:10018000BAEB000042F0000042F0000042F0000034
:1001900042F0000042F0000042F0000052E1000096
:1001A00042F0000042F0000042F0000042F0000087
:1001B00042F0000042F0000042F0000042F0000077
:1001C00042F0000042F0000042F0000042F0000067
:1001D00042F0000042F0000042F0000042F0000057
:1001E00042F0000042F0000042F0000042F0000047
:1001F00042F0000042F0000042F0000042F0000037
:10020000000000000000000042F0000042F000008A
:1002100042F0000042F0000042F0000042F0000016
:1002200042F0000042F0000042F0000042F0000006
:1002300042F000005C74000042F0000042F0000058
:1002400042F0000082740000A874000042F0000038
:1002500042F0000042F0000042F0000088CA0000B6
:1002600042F0000042F0000088CD000020C20000F3
:1002700042F00000CAE600007EDF000042F000000D
:1002800042F000001CE7000042F0000042F00000D5
:1002900042F00000DC74000002750000BEDF0000C8
:1002A00042F0000042F0000042F0000042F0000086
:1002B00042F0000042F0000042F0000042F0000076
:1002C00042F0000042F0000042F0000042F0000066
:1002D00042F0000042F00000A4A9000042F000003B
:1002E00042F0000042F0000042F000000ECE00009C
:1002F000B6C2000042F0000042F000009EAC0000D8
:100300000869000042F0000042F0000042F00000E6
:1003100042F0000042F0000042F0000042F0000015
:1003200042F0000042F0000042F0000042F0000005
:1003300042F0000042F0000042F0000042F00000F5
:1003400042F0000042F000008AAC000042F00000E1
:1003500042F0000042F0000042F0000042F00000D5
:1003600042F0000042F0000042F0000042F00000C5
:1003700042F0000042F0000090CE00004CC30000AC
:100380009E48010042F0000042F0000042F00000F0
:1003900042F0000042F0000042F0000052E1000094
:1003A00042F0000042F0000042F0000042F0000085
:1003B00042F0000042F0000042F0000042F0000075
:1003C00042F0000042F0000042F0000042F0000065
:1003D00042F0000042F0000042F0000042F0000055
:1003E00042F0000042F0000042F0000042F0000045
:1003F00042F0000042F0000042F0000042F0000035
:1004000000480400010000004F432300607D2400E9
:1004100000018800000000000B000700206B2B008B
:100420000100200010000700000020000000E00094
:10043000020032000000020000000000D6AC020002
:10044000000000000000FE004440A900E079210007
:100450000000E0000300320000002000A00188003E
:100460004440A80000000600F8FF2000591C2100AD
:1004700091018800800078000000EB001A0037002E
:100480008180E80032A0B4009101BA00E28040000F
:1004900032A0B4009102BA00E280400032A0B40061
:1004A0000002EB00472BDE00F507B200602CE100F4
:1004B00009003A00330007000700E00002003200A4
:1004C0000059EB00010037000201E8008301E90058
:1004D000F8FF3E00040037006128E100010032000F
:1004E0000082EB00040007001101BA000200E000E6
:1004F000E3FF3A0000000600220007000700E000CA
:10050000020032003159BA00020037008100E800D1
:100510000201E8008301E90017003200190007001A
:100520000700E000020032002159BA000200370043
:100530008100E9000201E8008301E9000D003200BA
:100540000400E00003003A00E280400032A0B40062
:10055000E9FF37000B0007000700E000020032004F
:1005600011D9BA00010037000201E8008301E90057
:10057000F5FF3A008100E800E180400032A0B400BD
:10058000000006000810E600020037000910E6002F
:10059000020037008083EB00000006008003EB00C0
:1005A0000000060091018800800078000000EB0048
:1005B00015003700E280400032A0B4009101BA007B
:1005C000E280400032A0B4009102BA00E280400014
:1005D00032A0B4000002EB00472BDE00F507B200AA
:1005E000602CE10004003A000059EB008301E900AF
:1005F000FDFF3E00040037006128E10001003200E9
:100600000082EB00040007001101BA000200E000C4
:10061000E8FF3A00000006003159BA008301E90002
:100620000C0032002159BA008301E90008003200B1
:100630000400E00003003A00E280400032A0B40071
:10064000F5FF370011D9BA008301E900FAFF3A003B
:100650008100E800E180400032A0B4000000060004
:10066000F01F040000000000EED3040000000000B2
:10067000B28C0400000000007EAE04000000000008
:10068000C88D040000000000C8C90400000000007C
:10069000DCAB0400000000000CAB04000000000014
:1006A00026AB04000000000078AB0400000000004E
:1006B000A8E5040000000000B0DD04000000000018
:1006C0003CE1040000000000B4BA04000000000097
:1006D00024AF040000000000F8B204000000000095
:1006E000F4B20400000000009AB30400000000000F
:1006F00068B3040000000000FCB204000000000029
:100700000C770400000000003E77040000000000A9
:100710006E77040000000000B077040000000000C5
:10072000F4770400000000003878040000000000A6
:100730007A78040000000000E67804000000000061
:100740002E7904000000000076790400000000000B
:10075000D279040000000000487A04000000000084
:10076000C47A040000000000187B040000000000B0
:10077000347B040000000000C67B04000000000081
:10078000127C0400000000004E7C04000000000009
:100790008A7C0400000000003E7D04000000000090
:1007A000667E040000000000A09504000000000028
:1007B0001496040000000000D4950400000000001E
:1007C000549604000000000094960400000000000D
:1007D000DA960400000000006697040000000000A4
:1007E000CA97040000000000989704000000000071
:1007F0008A99040000000000FC970400000000003B
:100800005A98040000000000E69804000000000070
:100810001C9904000000000038990400000000004A
:100820005499040000000000BC990400000000007E
:10083000F499040000000000109A04000000000079
:100840007E9A040000000000B09A0400000000003E
:10085000E29A0400000000000C9B0400000000006D
:1008600056AC0400000000006022B8000602200020
:100870000000D0008180D2000482D2008582D200A4
:100880000000A0000202520083825A0003003100DF
:100890000202420083824A000000A1000603E90030
:1008A000F3FF3A0000000600020AB900001BB9007D
:1008B0000200B800810042008100430000000600F1
:1008C000889FBE008A9FBE008C1F78000006EB0048
:1008D000E00F5000E08F5800E00F5900E08F590002
:1008E00007003D006044B8006055B80000005400A7
:1008F00081805C0002015D0083815D001C0020009E
:10090000E00F5200E08F5A00E00F5B00E08F5B00C9
:1009100007003D006044B8006055B8000402540070
:1009200085825C0006035D0087835D000C00A200E9
:100930000B010700E00F5600060032006022B800ED
:100940006033B8000000520081805A0002015B0051
:1009500083815B004F0678004F05BE004F04BE0048
:1009600000000600889FBE008A9FBE003004BE00C3
:100970002005BE000404440085844C0006054D009B
:1009800087854D000898BE000A90BE0095000700BC
:1009900002003100680040001008E8004F05BE006A
:1009A0004F04BE0000000600889FBE008A9FBE0064
:1009B0008C1F7800000678003C04BE002C05BE00A9
:1009C0000400540085805C0006015D0087815D00A5
:1009D000009EBE00029EBE001000200081000700A5
:1009E000010039000000EB001C0E10004F067800DB
:1009F0004F05BE004F04BE00000006001200FA00C2
:100A0000889FBE008A9FBE008C9FBE000205BE006C
:100A10000004BE00E4B79F00F5B79F0086BF9F00AB
:100A200097BF9F000000EB00D0B79F00C0B79F00AA
:100A3000B0B79F00A0B79F0090B79F000006780056
:100A4000FD032000DFB197004FB097000381410004
:100A5000BFB09700E08F510004003D006600070022
:100A60007E805700BFFF07000300370062000700C9
:100A70007E805700CCFF0700DFB09700E08F50006A
:100A80000700350014002000050020006033B80086
:100A900008047200898472000A0573008B85730054
:100AA0000C06E8008D0F5600E6FF3400E08F500082
:100AB00006003D006FB29700FFB297000FBB970092
:100AC0009FBB97007E805700A6FF07005FA8970096
:100AD000E00F500004003A001FB49700AFB4970035
:100AE0003FB59700CFB597000800BE000A01BE00D1
:100AF0004F06BE004F05BE004F04BE000080FA0046
:100B000000000600881F780018002000881F780069
:100B1000BAFF07008F87E9004F0478000000060045
:100B2000801FEB00B5FF07008F87E900000006007B
:100B3000889FBE008A9FBE008C1F78004E00070071
:100B400005003D005100070009003D005B00070063
:100B50000006EB00060037005D00070004003D00C2
:100B60006044B8006055B800540007001C00200025
:100B7000E4FF0700E00F5600010032005A000700B2
:100B80004F0678004F05BE004F04BE00000006006F
:100B9000889FBE008A9FBE008C1F78003600070029
:100BA00003003D003900070006003D000400370047
:100BB0004700070003003D006044B8006055B800DE
:100BC0003E000700D6FF0700E00F5600010032008C
:100BD000450007004F0678004F05BE004F04BE00D9
:100BE000000006000440E10005C8E10006D0E10075
:100BF00007D8E10000000600CF01DE00028171008D
:100C0000B2B79F004F09DE000000400000007100F5
:100C1000A0B79F000FB097004F01DE008180400019
:100C20008100710091B79F007FAA9700CF20DE005E
:100C3000000040000080700080B79F000800BE00E8
:100C40000A01BE004F18DE000402420000027200DA
:100C5000F4AF9F000804440089844C000A054D004D
:100C60008B854D004FB29700DFB297006FB39700AE
:100C7000FFB3970000000600E00F5000E08F58001F
:100C8000E00F5900E08F5900000006006044B800F2
:100C90006055B8000000540081805C0002015D00D6
:100CA00083815D001C0020000820E10009A8E1000C
:100CB0000AB0E1000BB8E100000006000402540095
:100CC00085825C0006035D0087835D0000000600EE
:100CD0000006EB00E00F5200E08F5A00E00F5B00CF
:100CE000E08F5B00000006006022B8006033B800AF
:100CF0000000520081805A0002015B0083815B008A
:100D000000000600839F68000100E00002003D0033
:100D100060001000E08018000300E00002003D00C9
:100D200060011100E0811900CFFE07004F00E000D4
:100D300002003B0060001000E08018000000060088
:100D400080017800110009008280D8008001FD0038
:100D5000110009004288D8008300780000000600D6
:100D6000889FBE008A9FBE008C9FBE000404B8000E
:100D70000506B8008904460060854E000606B800E6
:100D80000A054600E0854E000706B8008B054600C0
:100D9000040EB800890446000A854E00E0854D0027
:100DA000050EB8000A0546008B854E00060EB800F9
:100DB0008B0546000416B8000A0546008B854E00D8
:100DC0000516B8008B054600041EB8008B054600CA
:100DD0000800BE000A01BE004F06BE004F05BE005F
:100DE0004F04BE00000006008001780002003700BA
:100DF000B1597800040178000202E900E00F5100C7
:100E0000FBFF3A0000000600800178000200370076
:100E100081597800040178000202E900E00F5100D6
:100E2000FBFF3A0000000600800078000041EB0064
:100E3000B14F1100FDFF3A000080EA000080400041
:100E400000000600E68747008E1F7800D0BF9F0095
:100E500066875700012F78000E003700DFB9970032
:100E6000134178006FB8970090407800814F51008F
:100E7000040032000280FB008180FB000100500072
:100E8000080037008301E800D3BF9F00000FE8008F
:100E9000040178000202E900E00F5100EFFF3A0080
:100EA000020078004F0778006F00B10000000600D4
:100EB0006D610000746800002E6300006F70000018
:100EC00079000000636F0000706900006573000026
:100ED0002073000072630000207400006F20000087
:100EE0006465000073740000206500006C650000FC
:100EF0006D6500006E740000206200007920000023
:100F0000656C0000656D0000656E000074000000F7
:100F100064650000737400000073000072630000D9
:100F2000000000005887000062870000FFFF0000FB
:100F300088870000FFFF00008D8700000000000090
:100F4000000000006D610000746800002E66000063
:100F5000696C00006C000000666900006C6C0000A9
:100F600073200000646500007374000020770000A7
:100F70006974000068200000636F00006E73000059
:100F8000746100006E74000020760000616C000047
:100F90007565000000760000616C0000756500005A
:100FA00000000000A2870000AC870000FFFF0000E7
:100FB0008887000001000000CB87000000000000CF
:100FC000000000006D610000746800002E610000E8
:100FD0006464000073630000616C000061720000D3
:100FE0000061000064640000207300006361000081
:100FF0006C61000072200000746F0000206500002A
:101000006163000068200000656C0000656D0000F1
:10101000656E0000742000006F6600002073000001
:1010200072630000206100006E6400002073000005
:10103000746F00007265000020720000657300008C
:10104000756C000074200000746F000020640000C4
:10105000657300007400000073630000616C0000A1
:101060006172000000000000E2870000F1870000CC
:10107000FFFF000088870000FFFF00008D87000051
:10108000010000002C8800000000000000000000AB
:101090006D610000746800002E610000646400004F
:1010A000006100006464000073200000737200009F
:1010B00063310000206100006E64000020730000B6
:1010C0007263000032200000746F00002064000092
:1010D00065730000742C0000206500006C65000042
:1010E0006D6500006E740000206200007920000031
:1010F000656C0000656D0000656E00007400000006
:10110000737200006331000000730000726300001E
:10111000320000004888000051880000FFFF0000F6
:1011200088870000FFFF000080880000FFFF0000AC
:101130008588000000000000000000006D610000D4
:10114000746800002E7300007562000000730000D8
:101150007562000073740000726100006374000027
:1011600073200000737200006332000020660000EC
:10117000726F00006D200000737200006331000088
:10118000207400006F20000064650000737400008C
:101190002C200000656C0000656D0000656E00008D
:1011A0007420000062790000206500006C6500007A
:1011B0006D6500006E740000000000009E88000055
:1011C000A7880000FFFF000088870000FFFF0000E5
:1011D00080880000FFFF00008588000000000000FC
:1011E000000000006D610000746800002E6D0000BA
:1011F000756C0000006D0000756C000074690000E3
:10120000706C0000696500007320000073720000BC
:1012100063310000206100006E6400002073000054
:101220007263000032200000746F00002064000030
:1012300065730000742C0000206500006C650000E0
:101240006D6500006E7400002062000079200000CF
:10125000656C0000656D0000656E000074000000A4
:10126000F2880000FB880000FFFF00008887000074
:10127000FFFF000080880000FFFF0000858800005D
:1012800000000000000000006D61000074680000B4
:101290002E6400006976000000640000697600009A
:1012A0006964000065730000207300007263000031
:1012B000312000006279000020730000726300009A
:1012C00032200000746F000020640000657300008D
:1012D000742C0000206500006C6500006D65000046
:1012E0006E7400002062000079200000656C000030
:1012F000656D0000656E0000740000004489000008
:101300004D890000FFFF000088870000FFFF0000FC
:1013100080880000FFFF00008588000000000000BA
:10132000000000006D610000746800002E6D000078
:10133000696E0000007700007269000074650000AB
:101340007320000074680000652000006D690000D3
:101350006E6900006D7500006D2000006F66000072
:10136000207300007263000031200000616E0000F5
:1013700064200000737200006332000020740000DB
:101380006F20000064650000737400002C200000D2
:10139000656C0000656D0000656E00007420000043
:1013A00062790000206500006C6500006D6500003A
:1013B0006E74000000000000928900009B8900000C
:1013C000FFFF000088870000FFFF0000808800000A
:1013D000FFFF000085880000000000000000000002
:1013E0006D610000746800002E6D000061780000DF
:1013F000007700007269000074650000732000002F
:1014000074680000652000006D61000078690000CC
:101410006D7500006D2000006F66000020730000F5
:101420007263000031200000616E00006420000043
:101430007372000063320000207400006F2000000F
:1014400064650000737400002C200000656C0000CF
:10145000656D0000656E0000742000006279000078
:10146000206500006C6500006D6500006E74000072
:1014700000000000F0890000F9890000FFFF000073
:1014800088870000FFFF000080880000FFFF000049
:101490008588000000000000000000006D61000071
:1014A000746800002E6300006C6100006D70000025
:1014B000006300006C6100006D700000207300008C
:1014C00072630000207400006F2000006C6F000049
:1014D000772F000068690000676800002062000044
:1014E0006F7500006E64000073200000696E0000DC
:1014F000746F00002064000065730000742C00000D
:10150000206500006C6500006D6500006E740000D1
:101510002062000079200000656C0000656D00000D
:10152000656E0000740000006C6F00007700000022
:101530006869000067680000000000004E8A000033
:10154000598A0000FFFF000088870000FFFF0000AD
:101550008D870000FFFF0000948A0000FFFF00005D
:10156000988A000000000000000000006D6100008B
:10157000746800002E6400006F74000000770000A3
:101580007269000074650000732000007468000038
:1015900065200000646F000074200000707200007D
:1015A0006F64000075630000742000006F66000027
:1015B000207300007263000031200000616E0000A3
:1015C0006420000073720000633200002074000089
:1015D0006F20000064650000737400002C20000080
:1015E0006166000074650000722000006120000048
:1015F00073680000696600007400000073680000F2
:101600006966000074000000B68A0000BF8A00000E
:101610000100000088870000FFFF000080880000B4
:10162000FFFF00008588000001000000FE8A000026
:1016300000000000000000006D6100007468000000
:101640002E730000746100007400000070650000DB
:10165000726600006F7200006D730000207300005E
:101660007461000074690000737400006963000015
:10167000732000006F6E0000207300007263000092
:10168000006D0000696E0000006D000061780000D0
:10169000006D0000656100006E0000001C8B000002
:1016A000268B0000FFFF00008D8700000100000076
:1016B000418B000001000000458B0000010000008C
:1016C000498B000000000000000000006D61000078
:1016D000746800002E61000072670000626F0000F5
:1016E000756E000064730000006700006574000000
:1016F0002074000068650000206900006E6400002E
:10170000696300006573000020280000617200001A
:10171000676D0000696E00002C20000061720000FF
:10172000676D000061780000292000006F660000EE
:101730002074000068650000206C0000696D0000E6
:101740006974000020760000616C0000756500007F
:10175000732000006F6600002073000072630000B9
:1017600000610000726700006D6900006E000000FB
:1017700061720000676D00006178000000000000E9
:10178000668B0000758B0000FFFF00008D87000056
:1017900001000000B18B000001000000B88B0000C8
:1017A00000000000000000006D610000746800008F
:1017B0002E7300006F72000074000000736F000051
:1017C00072740000206100007272000061790000F4
:1017D000206900006E200000706C00006163000052
:1017E0006500000061720000726100007900000075
:1017F000D48B0000DE8B0000FFFF0000F28B0000A6
:1018000000000000000000006D610000746800002E
:101810002E6D0000756C0000646900007600000009
:1018200070650000726600006F7200006D7300004A
:101830002064000065730000742000003D2000005B
:10184000286100002A620000292F000063200000A8
:10185000696E000020330000322000006269000041
:1018600074730000206500006C6500006D65000069
:101870006E7400002062000079200000656C00009A
:10188000656D0000656E00007400000061000000DE
:101890006200000063000000048C0000108C000057
:1018A000FFFF000088870000FFFF0000468C00005B
:1018B000FFFF0000488C0000FFFF00004A8C000082
:1018C00000000000000000006D610000746800006E
:1018D0002E610000746100006E3200000070000094
:1018E00065720000666F0000726D000073200000DA
:1018F0006465000073740000203D0000206100005A
:10190000746100006E320000287900002C7800001D
:1019100029200000656C0000656D0000656E000008
:101920007420000062790000206500006C650000F2
:101930006D6500006E740000007900000078000002
:1019400000000000648C00006F8C0000FFFF0000AE
:1019500088870000FFFF00009D8C0000FFFF000053
:101960009F8C000000000000000000006D6100007E
:10197000746800002E730000696E000000700000A3
:1019800065720000666F0000726D00007320000039
:101990006465000073740000203D000020730000A7
:1019A000696E00002878000029200000656C0000A6
:1019B000656D0000656E0000742000006279000013
:1019C000206500006C6500006D6500006E7400000D
:1019D00000000000B68C0000BF8C0000FFFF00007C
:1019E00088870000FFFF00009F8C000000000000BF
:1019F000000000006D610000746800002E630000AC
:101A00006F7300000070000065720000666F0000D8
:101A1000726D0000732000006465000073740000A4
:101A2000203D0000206300006F7300002878000054
:101A300029200000656C0000656D0000656E0000E7
:101A40007420000062790000206500006C650000D1
:101A50006D6500006E74000000000000FA8C00004C
:101A6000038D0000FFFF000088870000FFFF0000DB
:101A70009F8C000000000000000000006D6100006D
:101A8000746800002E7200006F74000032000000C5
:101A9000726F000074610000746500007320000024
:101AA000762000006F660000206100006E67000075
:101AB0006C65000020610000207400006F200000B1
:101AC00064650000737400000076000000000000F0
:101AD0003E8D0000488D0000020000008887000055
:101AE00002000000658D000001000000468C00002F
:101AF00000000000000000006D610000746800003C
:101B00002E73000071720000740000007065000008
:101B1000726600006F7200006D73000020640000A8
:101B200065730000742000003D2000007371000008
:101B3000727400002878000029200000656C000005
:101B4000656D0000656E0000742000006279000081
:101B5000206500006C6500006D6500006E7400007B
:101B6000000000007C8D0000868D0000FFFF00005B
:101B700088870000FFFF00009F8C0000000000002D
:101B8000000000006D610000746800002E6E00000F
:101B90007A73000065710000007700007269000030
:101BA00074650000207400006F2000006465000070
:101BB000737400002074000068650000206D000050
:101BC00069640000646C000065200000696E00001C
:101BD00064650000782000006F660000207400003B
:101BE00068650000206C00006172000067650000FD
:101BF00073740000207300006571000075650000BB
:101C00006E630000652000006F660000206E00001B
:101C10006F6E00002D7A0000657200006F200000DA
:101C2000656C0000656D0000656E00007473000057
:101C300020660000726F00006D20000073720000CB
:101C4000632C0000202D0000312000006966000098
:101C5000206E00006F740000206600006F750000A9
:101C60006E640000206F00007220000069660000B2
:101C7000207300006D6100006C6C00006572000054
:101C800020740000686100006E2000006D69000093
:101C90006E4C0000656E0000677400006800000074
:101CA0006D6900006E4C0000656E000067740000F6
:101CB00068000000C28D0000CD8D00000100000012
:101CC00088870000FFFF00008D87000001000000F2
:101CD000508E000000000000000000006D61000058
:101CE000746800002E720000616E00006400000045
:101CF000666900006C6C00002061000072720000D8
:101D000061790000207700006974000068200000FD
:101D1000726100006E6400006F6D000020760000AC
:101D2000616C000075650000730000006E8E00009D
:101D3000788E0000FFFF0000888700000000000090
:101D400000000000000000009301000024030000D8
:101D5000B704000048060000DA0700006B09000025
:101D6000FC0A00008C0C00001C0E0000AB0F0000F1
:101D70003B110000C812000056140000E3150000DB
:101D80006E170000F9180000831A00000C1C0000F8
:101D9000941D00001A1F0000A02000002422000053
:101DA000A723000029250000A826000027280000FE
:101DB000A4290000202B0000992C0000122E000006
:101DC000872F0000FC3000006F320000DF3300007E
:101DD0004E350000BA360000253800008D3900006D
:101DE000F33A0000573C0000B93D0000173F0000E7
:101DF00074400000CE410000264300007B440000F8
:101E0000CD4500001D4700006A480000B4490000AD
:101E1000FC4A0000404C0000824D0000C04E000013
:101E2000FC4F000034510000695200009B53000039
:101E3000CA540000F65500001E5700004358000029
:101E400064590000835A00009D5B0000B45C0000F0
:101E5000C85D0000D75E0000E45F0000EC60000099
:101E6000F1610000F2620000EF630000E96400002D
:101E7000DE650000D0660000BD670000A7680000B6
:101E80008C6900006E6A00004B6B0000246C00003F
:101E9000F96C0000CA6D0000976E00005F6F0000D3
:101EA00023700000E37000009E7100005572000076
:101EB00008730000B6730000607400000575000030
:101EC000A575000042760000D97600006C7700000E
:101ED000FB77000084780000097900008A7900000F
:101EE000067A00007D7A0000EF7A00005D7B00003A
:101EF000C67B00002A7C0000897C0000E47C000096
:101F0000397D00008A7D0000D77D00001D7E000025
:101F1000607E00009D7E0000D67E0000097F0000EC
:101F2000397F0000627F0000877F0000A77F0000EC
:101F3000C27F0000D87F0000EA7F0000F67F00002B
:101F4000FE7F0000FF7F00008C020000DF02000027
:101F50003003000080030000D103000022040000D1
:101F600073040000C204000014050000B305000063
:101F700054060000F10600008F0700002D08000045
:101F8000CA08000063090000FC090000340B0000CF
:101F90005C0C0000820D0000A40E0000BD0F0000CC
:101FA000D3100000E2110000E7120000EF1400005F
:101FB000CC16000092180000401A0000D61B00004A
:101FC000531D0000B51E00000B2000007922000008
:101FD0008D2400006F2600001428000090290000C6
:101FE000E02A0000112C0000252D0000052F000024
:101FF00089300000D3310000EC320000DD330000F6
:10200000AE340000673500000D36000020370000B8
:10201000FB370000B23800004A390000CC3900001C
:102020003B3A00009B3A0000F33A0000833B00007B
:10203000F43B0000513C00009F3C0000E13C0000EC
:102040001A3D00004B3D0000783D0000C03D0000FF
:10205000F93D0000283E00004F3E0000703E0000A9
:102060008D3E0000A53E0000BC3E0000E03E0000AA
:10207000FD3E0000143F0000283F0000383F0000F4
:10208000473F0000533F00005E3F0000703F0000EC
:102090007F3F00008A3F0000943F00009C3F00000B
:1020A000A43F0000AA3F0000AF3F0000B83F00007F
:1020B000C03F0000C53F0000CB3F0000CE3F000006
:1020C000D23F0000D53F0000D83F0000DC3F0000B9
:1020D000E03F0000E33F0000E53F0000E83F000074
:1020E000E93F0000EB3F0000EC3F0000EE3F000046
:1020F000F13F0000F13F0000F33F0000F43F00001B
:10210000F53F0000F53F0000F73F0000F73F0000FB
:10211000F93F0000F83F0000FA3F0000FA3F0000DE
:10212000FA3F0000FB3F0000FB3F0000FC3F0000C7
:10213000FC3F0000FC3F0000FE3F0000FD3F0000B0
:10214000FD3F0000FD3F0000FE3F0000FE3F00009D
:10215000FE3F0000FE3F0000FE3F0000FE3F00008B
:1021600000400000FF3F0000FF3F0000FF3F000075
:10217000FF3F0000FF3F0000FF3F0000FF3F000067
:10218000FF3F0000FF3F0000FF3F0000FF3F000057
:10219000004000000040000000400000004000003F
:1021A000004000000040000000400000004000002F
:1021B000004000000040000000400000004000001F
:1021C00000400000004000000040000041640000AA
:1021D0006472000065730000732000006F750000DA
:1021E000742000006F66000020730000657400001A
:1021F000746900006E67000073000000536C0000FB
:1022000065650000702000006D6F000064650000CF
:10221000206E00006F7400002073000075700000D5
:10222000706F0000727400006564000000450000DB
:10223000727200006F7200003A2000006D690000A9
:102240006E2000003D3D0000203000007846000078
:102250004646000046460000464600004620000074
:102260002100000045720000726F0000723A000009
:10227000205500006E610000626C000065200000C7
:10228000746F0000206600006C610000736800003D
:102290002062000079740000656300006F64000034
:1022A00065200000283100002920000021000000E6
:1022B00045720000726F0000723A00002055000065
:1022C0006E610000626C000065200000746F000009
:1022D000206600006C61000073680000206200004E
:1022E00079740000656300006F64000065200000E1
:1022F0002832000029200000210000004572000063
:10230000726F0000723A0000205500006E610000FC
:10231000626C000065200000746F00002066000001
:102320006C61000073680000206200007974000096
:10233000656300006F640000652000002833000022
:102340002920000021000000466C0000617300009D
:10235000686900006E670000204F00004B0000001D
:1023600074680000796D0000696F00002D4900005D
:10237000490000005F69000064000000657600000D
:10238000656E0000742E0000736F0000757200000F
:102390006365000000650000766500006E74000053
:1023A0002E61000072670000730000005F6600008D
:1023B0007776000065720000736900006F6E0000A0
:1023C000005F0000707200006F6400007563000021
:1023D000744900006400000062750000747400001D
:1023E0006F6E0000732E00005F72000061770000C6
:1023F0000062000075740000746F00006E2E000013
:1024000062610000636B000077610000726400008D
:102410000062000075740000746F00006E2E0000F2
:102420006C650000667400000062000075740000B6
:10243000746F00006E2E0000636500006E74000073
:10244000657200000062000075740000746F000087
:102450006E2E0000666F000072770000617200004F
:102460006400000062750000747400006F6E00006C
:102470002E720000696700006874000000620000AE
:1024800075740000746F00006E7300002E5F000012
:102490006D650000616E0000006200007574000050
:1024A000746F00006E7300002E5F00006E6F0000FE
:1024B0006973000065000000707200006F78000012
:1024C0002E6800006F720000697A00006F6E0000D5
:1024D000746100006C000000707200006F780000F2
:1024E0002E6300006F6D00006D2E000072780000FA
:1024F0002E5F000070610000796C00006F610000C9
:102500006473000000700000726F0000782E0000FD
:10251000636F00006D6D00002E720000782E0000C9
:102520005F6900006E740000656E00007369000052
:10253000746900006573000000700000726F000095
:10254000782E0000636F00006D6D00002E72000099
:1025500078000000707200006F7800002E630000A9
:102560006F6D00006D2E0000747800000070000098
:10257000726F0000782E0000677200006F75000017
:102580006E6400002E6100006D6200006961000051
:102590006E74000000700000726F0000782E000062
:1025A000677200006F7500006E6400002E720000FC
:1025B000656600006C6500006374000065640000DF
:1025C00000700000726F0000782E0000677200003B
:1025D0006F7500006E6400002E640000656C0000E2
:1025E00074610000006D00006F7400006F720000E5
:1025F0002E6C000065660000742E000074610000FF
:102600007267000065740000006D00006F740000C8
:102610006F7200002E72000069670000687400008D
:102620002E740000617200006765000074000000F5
:102630005F76000062610000740000005F690000C6
:102640006D6F0000740000006D6F0000746F00007B
:10265000722E00006C650000667400002E7300008E
:102660007065000065640000006D00006F7400007C
:102670006F7200002E72000069670000687400002D
:102680002E7300007065000065640000006D00009E
:102690006F7400006F7200002E6C00006566000011
:1026A000742E0000707700006D0000006D6F000058
:1026B000746F0000722E00007269000067680000ED
:1026C000742E0000707700006D0000006163000050
:1026D00063000000746500006D700000657200000A
:1026E00061740000757200006500000072630000F4
:1026F000352E000061640000647200006573000004
:102700007300000072630000352E0000636F00004C
:102710006D6D0000616E0000640000006D690000D6
:10272000632E0000696E0000746500006E73000087
:1027300069740000790000006D690000632E0000DC
:102740007468000072650000736800006F6C000020
:10275000640000006D690000632E00005F6D0000E2
:10276000656100006E000000746900006D65000086
:10277000722E000070650000726900006F64000036
:1027800000610000636300002E5F000074610000C0
:1027900070000000B091000001000000BA9100003C
:1027A00001000000BE91000020000000CB9100005D
:1027B00002000000D691000001000000E19100003D
:1027C00005000000EC91000001000000F9910000FC
:1027D00001000000099200000100000015920000B5
:1027E000010000002392000001000000329200006E
:1027F000050000003F920000050000004D9200001F
:10280000070000005C920000070000006C920000CE
:102810000700000083920000010000009D9200006C
:1028200001000000AA92000002000000B792000020
:1028300002000000CB92000002000000E1920000C4
:1028400001000000F3920000010000000593000069
:102850000200000018930000020000001E93000018
:1028600001000000249300000100000035930000E7
:102870000100000047930000010000005693000093
:102880000300000066930000010000006A9300004E
:102890000100000076930000010000008293000018
:1028A000010000008E930000010000009C930000D6
:1028B00001000000AA93000002000000B493000091
:1028C00001000000C19300000000000000000000B3
:1028D000DE000000AD000000CA000000FE000000A5
:1028E000BE000000EF000000040000000200000035
:1028F000F4B200009AB3000068B30000FCB200001C
:102900000C7700003E7700006E770000B077000083
:10291000F4770000387800007A780000E67800004C
:102920002E79000076790000D2790000487A000004
:10293000C47A0000187B0000347B0000C67B0000D6
:10294000127C00004E7C00008A7C00003E7D00006E
:10295000667E0000A095000014960000D49500004B
:102960005496000094960000DA96000066970000E6
:10297000CA970000989700008A990000FC97000011
:102980005A980000E69800001C9900003899000051
:1029900054990000BC990000F4990000109A0000BE
:1029A0007E9A0000B09A0000E29A00000C9B0000A2
:1029B00056AC000042610000636B000077610000CC
:1029C000726400002062000075740000746F0000E3
:1029D0006E200000737400006174000075730000C5
:1029E00020630000686100006E67000065640000FD
:1029F000004C000065660000742000006275000055
:102A0000747400006F6E0000207300007461000099
:102A1000747500007320000063680000616E0000A0
:102A20006765000064000000436500006E740000EC
:102A3000657200002062000075740000746F000071
:102A40006E20000073740000617400007573000054
:102A500020630000686100006E670000656400008C
:102A6000004600006F720000776100007264000091
:102A70002062000075740000746F00006E2000007A
:102A8000737400006174000075730000206300001F
:102A9000686100006E67000065640000005200007D
:102AA000696700006874000020620000757400000F
:102AB000746F00006E2000007374000061740000E9
:102AC0007573000020630000686100006E670000FD
:102AD000656400000062000075740000746F0000FF
:102AE0006E7300000042000075740000746F0000F7
:102AF0006E73000020760000616C000075650000B8
:102B000073200000757000006461000074650000AF
:102B100064000000707200006F7800000050000038
:102B2000726F0000786900006D6900007479000020
:102B300020760000616C00007565000073200000C5
:102B4000757000006461000074650000640000009E
:102B5000707200006F7800002E6300006F6D00003F
:102B60006D000000446100007461000020720000EC
:102B70006563000065690000766500006420000060
:102B80006F6E000020740000686500002070000077
:102B9000726F0000786900006D69000074790000B0
:102BA000206300006F6D00006D7500006E6900000D
:102BB00063610000746900006F6E00000074000023
:102BC000617000000041000020740000617000008E
:102BD0002069000073200000646500007465000037
:102BE000637400006564000000410000636300003E
:102BF000656C0000657200006F6D00006574000078
:102C00006572000020760000616C000075650000B0
:102C1000732000007570000064610000746500009E
:102C2000640000006D690000630000004669000058
:102C3000726500006420000077680000656E000087
:102C4000206D000069630000726F00007068000072
:102C50006F6E000065200000696E00007465000062
:102C60006E73000069740000792000006973000031
:102C700020610000626F0000766500002074000093
:102C80006872000065730000686F00006C640000EB
:102C9000007300006F7500006E6400002E66000077
:102CA000696E000069730000686500006400000040
:102CB000466900007265000064200000776800002B
:102CC000656E000020740000686500002070000040
:102CD0006C61000079620000616300006B200000FD
:102CE0006F66000020610000207500007365000021
:102CF00072200000696E00006974000069610000C4
:102D00007465000064200000736F0000756E0000A1
:102D1000642000006973000020660000696E0000F6
:102D200069730000686500006400000054650000DD
:102D30006D70000065720000617400007572000023
:102D400065200000766100006C75000065200000C1
:102D5000757000006461000074650000640000008C
:102D6000726300003500000052430000352000006F
:102D70006D6500007373000061670000652000004E
:102D800072650000636500006976000065640000FC
:102D9000006D00006F7400006F720000004D0000B5
:102DA0006F7400006F72000020740000696D0000F5
:102DB0006572000000740000696D0000657200001B
:102DC00030000000546900006D65000072200000B2
:102DD00030000000746900006D6500007231000071
:102DE00000540000696D0000657200002031000091
:102DF00000000000F9910000DA9400000992000040
:102E0000F994000015920000149500002392000030
:102E100031950000329200004F9500006B95000044
:102E2000739500008A9500008F950000A89500001A
:102E3000B2950000DF950000E39500006693000066
:102E4000F5950000129600001696000049960000C5
:102E5000589600006A93000096960000B096000015
:102E6000B4960000C9960000CF960000DB960000E3
:102E7000E2960000EA960000F196000000000000D3
:102E8000000000005F7300007973000074650000AB
:102E90006D2E000072650000626F00006F7400000C
:102EA00000520000656200006F6F00007420000097
:102EB00074680000652000006D6900006372000006
:102EC0006F6300006F6E0000747200006F6C000092
:102ED0006C650000720000005F73000079730000F1
:102EE000746500006D2E00007365000074740000AE
:102EF000696E0000677300002E72000065610000BB
:102F00006400000052650000616400002061000060
:102F10002073000065740000746900006E67000093
:102F200000610000646400007265000073730000BB
:102F300000760000616C000075650000005F000015
:102F40007379000073740000656D00002E7300003B
:102F500065740000746900006E670000732E000045
:102F6000777200006974000065000000577200006D
:102F70006974000065200000612000007365000096
:102F800074740000696E0000670000005F73000049
:102F900079730000746500006D2E000073650000F9
:102FA00074740000696E0000677300002E660000F4
:102FB0006C61000073680000005700007269000037
:102FC0007465000020740000686500002073000034
:102FD00065740000746900006E67000073200000D3
:102FE000696E0000746F0000206600006C610000D4
:102FF000736800000000000045720000726F00005E
:10300000723A000020730000616D0000706C0000D7
:1030100065730000206D00007573000074200000CF
:1030200062650000206900006E2000005B2D00003A
:1030300031320000382C000031320000375D0000D2
:1030400020720000616E000067650000005F0000F4
:103050006C650000647300002E730000657400004E
:1030600000530000657400002074000068650000D3
:10307000206C000065640000006C000065640000C6
:10308000006200007269000067680000746E000052
:103090006573000073000000736F0000756E000020
:1030A000642E000072650000636F0000726400000F
:1030B0000053000074610000727400002072000070
:1030C000656300006F720000646900006E670000B5
:1030D000206F000066200000724E00002E77000076
:1030E00061760000004E0000007300006F75000064
:1030F0006E6400002E7000006C610000790000001A
:10310000537400006172000074200000706C0000B5
:103110006179000062610000636B0000206F0000B5
:1031200066200000704E00002E77000061760000DF
:10313000007300006F7500006E6400002E720000C6
:10314000657000006C61000079000000537400009D
:103150006172000074200000706C00006179000052
:1031600062610000636B0000206F000066200000B9
:10317000724E00002E7700006176000000730000A0
:103180006F7500006E6400002E73000079730000FC
:10319000746500006D00000053740000617200004F
:1031A00074200000706C0000617900006261000012
:1031B000636B0000206F0000662000007379000040
:1031C00073740000656D0000207300006F750000CF
:1031D0006E640000204E0000006C0000656400007A
:1031E000732E000063690000726300006C650000CC
:1031F0000053000065740000206300006972000045
:10320000637500006C6100007220000072690000AC
:103210006E670000206C0000656400007300000011
:103220006C300000006C0000310000006C320000C7
:10323000006C0000330000006C340000006C0000E3
:10324000350000006C360000006C00003700000004
:103250006C650000647300002E7400006F70000045
:103260000053000065740000205200004742000037
:10327000207400006F700000206C00006564000086
:1032800000720000656400000067000072650000C5
:10329000656E0000006200006C75000065000000B3
:1032A0006C650000647300002E6200006F74000003
:1032B000746F00006D2E00007269000067680000E6
:1032C00074000000536500007420000052470000A5
:1032D00042200000626F0000746F00006D2000004B
:1032E0007269000067680000742000006C650000CF
:1032F000640000006C650000647300002E62000032
:103300006F740000746F00006D2E00006C6500008B
:103310006674000000530000657400002052000035
:1033200047420000206200006F7400006F6D0000D3
:10333000206C000065660000742000006C650000D1
:10334000640000006C650000647300002E620000E1
:1033500075740000746F00006E730000005300006D
:10336000657400002062000075740000746F000036
:103370006E730000206C00006564000073000000A4
:103380006C650000647300002E700000726F000016
:10339000782E0000680000005365000074200000D3
:1033A000686F0000726900007A6F00006E740000A0
:1033B000616C000020700000726F000078690000EE
:1033C0006D69000074790000206C000065640000E5
:1033D000730000006C650000647300002E70000034
:1033E000726F0000782E0000760000005365000028
:1033F00074200000766500007274000069630000AC
:10340000616C000020700000726F0000786900009D
:103410006D69000074790000206C00006564000094
:10342000730000006C650000647300002E720000E1
:103430006300000053650000742000007263000008
:10344000206C000065640000006C000065640000F2
:10345000732E0000736F0000756E000064000000A2
:103460005365000074200000736F0000756E00004B
:10347000642000006C650000640000006C650000C2
:10348000647300002E740000656D0000706500001C
:103490007261000074750000726500000053000046
:1034A00065740000206E000074630000206C000052
:1034B00065640000007300006F7500006E6400001A
:1034C0002E6600007265000071000000506C000064
:1034D00061790000206600007265000071750000CF
:1034E000656E000063790000004800007A0000006B
:1034F00064730000007300006F7500006E640000CC
:103500002E77000061760000650000005365000022
:1035100074200000746800006520000070720000D4
:10352000696D000061720000792000007761000081
:1035300076650000206F00006620000074680000BF
:1035400065200000746F00006E65000020670000B9
:10355000656E000065720000617400006F7200000B
:1035600000770000617600006500000070720000C6
:103570006F7800002E6300006F6D00006D2E00005C
:10358000656E0000616200006C650000004500008F
:103590006E610000626C0000652000006F72000028
:1035A0002064000069730000616200006C65000027
:1035B000207400006865000020700000726F000039
:1035C000786900006D6900007479000020630000D4
:1035D0006F6D00006D7500006E6900006361000092
:1035E000746900006F6E00000073000074610000D9
:1035F0007465000000730000642E00006F7000000E
:10360000656E0000004F0000706500006E20000035
:1036100061200000666900006C650000206F0000FA
:103620006E20000074680000652000005344000014
:103630002063000061720000640000006E750000ED
:103640006D6200006572000000730000746100008C
:103650007475000073000000736400002E77000092
:103660007269000074650000005700007269000074
:103670007465000020640000617400006120000097
:10368000746F00002074000068650000206F000067
:10369000706500006E65000064200000666900002F
:1036A0006C650000006400006174000061000000AF
:1036B0007772000069740000746500006E000000FD
:1036C000736400002E720000656100006400000059
:1036D0005265000061640000206400006174000015
:1036E00061200000667200006F6D00002074000011
:1036F00068650000206F0000706500006E650000C6
:1037000064200000666900006C6500000072000023
:103710006561000064000000736400002E73000007
:10372000656500006B00000053650000656B0000DC
:103730002074000068650000206F000070650000C4
:103740006E65000064200000666900006C65000082
:10375000007000006F73000069740000696F000062
:103760006E0000005F720000662E00006E6F0000A9
:103770006465000069640000005300006574000087
:103780002057000069720000656C0000657300003E
:10379000732000004E6F00006465000020490000A7
:1037A000440000006E6F00006465000049440000A2
:1037B00000000000733000002E77000061760000EA
:1037C00000730000322E00007761000076000000D8
:1037D000733300002E770000617600000073000054
:1037E000342E000077610000760000007335000081
:1037F0002E7700006176000000730000362E000076
:103800007761000076000000733700002E7700001B
:103810006176000000000000480D00000D0000006F
:103820003011000007000000EC130000070000004A
:103830000019000007000000781E000007000000CB
:103840000000000000000000781E00000D000000D5
:103850000019000007000000EC1300000700000042
:103860003011000007000000480D000007000000B4
:1038700000000000000000004C04000007000000F1
:103880009808000007000000000000000000000091
:10389000E40C000007000000301100000D000000E3
:1038A000C819000007000000000000000000000030
:1038B0009C27000002000000AB2200000100000075
:1038C0009D1C000002000000FB1800000200000028
:1038D0002D32000001000000322D00000100000028
:1038E0004628000002000000E82600000100000059
:1038F000BF22000002000000FB18000002000000D0
:10390000FF32000001000000C6200000010000009E
:10391000762F0000020000002C2E000001000000A5
:10392000CE2C000001000000FD3900000200000064
:103930000000000000000000C819000005000000A1
:10394000BE0A0000040000000000000000000000AB
:1039500030110000070000007C1500000700000087
:10396000000000000000000030110000070000000F
:103970007C15000007000000C819000007000000C7
:103980000000000000000000222A00002B2C000094
:103990003A3B00003C3D00003E3F00005B5D000004
:1039A0007C7F0000008000009A900000418E0000A3
:1039B000418F000080450000454500004949000056
:1039C000498E00008F900000929200004F990000F5
:1039D0004F55000055590000999A00009B9C00002B
:1039E0009D9E00009F410000494F000055A500002A
:1039F000A5A60000A7A80000A9AA0000ABAC000083
:103A000021AE0000AFB00000B1B20000B3B40000BE
:103A1000B5B60000B7B80000B9BA0000BBBC0000E2
:103A2000BDBE0000BFC00000C1C20000C3C4000092
:103A3000C5C60000C7C80000C9CA0000CBCC000042
:103A4000CDCE0000CFD00000D1D20000D3D40000F2
:103A5000D5D60000D7D80000D9DA0000DBDC0000A2
:103A6000DDDE0000DFE00000E1E20000E3E4000052
:103A7000E5E60000E7E80000E9EA0000EBEC000002
:103A8000EDEE0000EFF00000F1F20000F3F40000B2
:103A9000F5F60000F7F80000F9FA0000FBFC000062
:103AA000FDFE0000FF0000002E2E00002F2E000063
:103AB0002E2F00006D6F00006C6F00006C65000021
:103AC0002F690000326300002F690000326300009C
:103AD0005F70000072690000762E00006800000030
:103AE0002E2E00002F2E00002E2F00006D6F0000E4
:103AF0006C6F00006C6500002F69000032630000ED
:103B00002F6D00006173000074650000725F00009B
:103B1000707200006F7400006F6300006F6C000033
:103B20002E630000000000002E2E00002F2E00004B
:103B30002E2F00006D6F00006C6F00006C650000A0
:103B40002F690000326300002F690000326300001B
:103B50005F70000072690000762E000068000000AF
:103B60002E2E00002F2E00002E2F00006D6F000063
:103B70006C6F00006C6500002F690000326300006C
:103B80002F6D00006173000074650000722E00004C
:103B9000630000002E2E00002F2E00002E2F0000AC
:103BA0006D6F00006C6F00006C6500002F690000F5
:103BB000326300002F690000326300005F70000074
:103BC00072690000762E0000680000002E2E0000B2
:103BD0002F2E00002E2F00006D6F00006C6F000074
:103BE0006C6500002F690000326300002F73000035
:103BF0006C610000766500002E630000000000008C
:103C00002E2E00002F2E00002E2F00006D6F0000C2
:103C10006C6F00006C6500002F740000696D00007F
:103C2000657200002F740000696D0000657200006D
:103C30002E630000000000000100000000000000F2
:103C4000080000000000000040000000000000002C
:103C5000000100000000000052490000464600003C
:103C60000000000000000000574100005645000021
:103C7000666D0000742000001000000000000000CD
:103C80000100000001000000841E00000000000090
:103C9000841E000000000000010000000800000079
:103CA000646100007461000000000000000000007A
:103CB0005F4C00004F470000445500004D5000008D
:103CC0002E23000040210000005F0000544500004A
:103CD000535400004D4F0000442E000023400000CC
:103CE00021000000564D0000434F000044450000F5
:103CF0002E410000424F0000000000002E2E000068
:103D00002F2E00002E2F00006D6F00006C6F000042
:103D10006C6500002F6600006C6100007368000095
:103D20002F6600006C610000736800002E630000C5
:103D3000000000002E2E00002F2E00002E2F00006D
:103D40006D6F00006C6F00006C6500002F69000053
:103D5000326300002F690000326300005F700000D2
:103D600072690000762E0000680000005F7000009D
:103D70006F770000657200006F660000660000004B
:103D8000506F000077650000726F000066660000EB
:103D9000000000002E2E00002F6D00006D6100005D
:103DA00037360000363000002E63000000000000AF
:103DB0005F4200004C570000484C0000564C000089
:103DC0002E440000415400000000000010110000CB
:103DD000141200001300000001160000170000007C
:103DE000038000000F0F00000F0000000200FA0027
:103DF000881F7800E4815700C2022000C13D2300E3
:103E0000E4470200000000006FB997000084EB0057
:103E1000C0022000800F510029003A00003E23001C
:103E2000C4FD2F00F5FF2F0030034200A0834A009D
:103E30004102200080804000B10F5300A18F5B0041
:103E40001F003A00A49F8100B59F8100F801400047
:103E5000B30F5200A38F5A0019003A0086182E00A3
:103E6000F7FF2F000402430085824B00870C2000DF
:103E7000870F5200E08F5A0011003E0044E82100F5
:103E800005002000C49F8900D59F8900A49F890058
:103E9000B59F89008008EB00B11078000008EB00A6
:103EA00030107800C1E229006400500022070200AF
:103EB00000000000E00F500001003A00000478000C
:103EC000080078004F0478000080FA000000060027
:103ED000C202200003002000FC4B04000000000090
:103EE0000200FA00881F7800000478006011B80012
:103EF00008007800FC4B020000000000E48157003D
:103F0000C2022000C1E22900080078007A490200BC
:103F1000000000000000EB00C10220006FB9970014
:103F2000810F5100010032000080EB004F04780047
:103F30000080FA00000006000A00FA00889FBE0018
:103F4000000478000202BE00C2BF9F00D3BF9F00E2
:103F50004402B0000580B000A4BF9F00B5BF9F0021
:103F6000420020000300200008007800FC4B020003
:103F700000000000E00F500016003A00EE815700EC
:103F800042002000EC805700080078007A490200C7
:103F9000000000009FBC9700E48F54000D003A0021
:103FA000820220000300200008007800FC4B020081
:103FB00000000000E00F500006003A00EE815700BC
:103FC00009017800E8805700080078007A4902006B
:103FD000000000004F04BE000080FA000000060050
:103FE000C2EF020000000000FDFF3700A4CE8000F9
:103FF00004000100A0CE88000000060000000000C0
:1040000000000000000000000000000000000000B0
:1040100000000000000000000000000000000000A0
:104020000000000000000000000000000000000090
:104030000000000000000000000000000000000080
:107000000200370031587800030178008201E9005E
:10701000E00F5100FBFF3A000000060002003700BD
:1070200001587800030178008201E900E00F510067
:10703000FBFF3A0000000600889FBE008A9FBE004A
:107040008C9FBE008E1F7800000678000205BE00EF
:107050005C149000EC1490000001EB008A0F5400C7
:107060008B8F5C00380032004C409000E04F5000A5
:1070700024003200EE0220000C07470014C0B300C9
:107080000801BE008E0078001C4090000CA4020095
:107090000000000012002000E00F50002A003A001B
:1070A000404698005C099000EC0990007C08900034
:1070B0008C1090000200400083804800800F540034
:1070C000818F5C000F003100BC4690000B00370040
:1070D0005C089000EC089000080440008984480097
:1070E00014C0B3000801BE008E0078001C40900060
:1070F0000CA40200000000008D46E900E1CF56001C
:10710000F3FF3E000001EB00E00F5500E08F5D0053
:107110000D003200E10220008C80400014C0B3005A
:107120000A01BE001C40900098A30200000000006D
:1071300012002000E00F500003003A005A16980099
:107140006B16980000017800020078004F07780065
:107150004F06BE004F05BE004F04BE0000000600F3
:10716000881F780000047800E10220008880400039
:1071700014C0B3001840900098A302000000000063
:1071800031C0B300E00F500046003A00D122200089
:1071900088804000914078008181FB00C819DD00A3
:1071A000C122200088804000914078008180FB004F
:1071B0008181710021C0B30052A52A00828F510045
:1071C00038003A0078E39000C833DD000600200064
:1071D00068E190008281FB0002002000020373003E
:1071E0008383730048E190000281FB0003002000CC
:1071F000020373008383730058E190004811DD009F
:107200000300200002037300838373000782FB00E6
:1072100084027800060278000401BE006414240091
:107220004505200080407800840F5100858F59006B
:107230001C00320038439100C833DD0006002000F6
:10724000284091008080FB000000200000037300B4
:1072500081837300084091000080FB000100200042
:107260000003730081837300184091004800DD0023
:107270000100200000037300818373000781FB007D
:1072800082017800060178000200BE000400680058
:1072900085806800010070008000EA0000807000B6
:1072A000CF00DE00014078004F04780000000600A7
:1072B00092002000E00F50000C0032008041EB00F3
:1072C00090CF110009003200B0019000818F510071
:1072D00006003A00104090008CA30200000000005D
:1072E00061016000010032003200200002007800DD
:1072F00000000600889FBE008A1F78000004780006
:107300006011B800080078004BFF07008004780087
:10731000E08F54005F003A0030C0B300984F100077
:1073200054003A0058409000E04F500051003200A5
:107330006000B8005014980061149800EA02200020
:107340000805450002202000890078000A00780026
:1073500032FF0700C02220000800400052C5B300E1
:1073600002487800D022200008004000A2CAB300E2
:107370000248780022C5B300626C9800726C9800D5
:107380006F4141000274980013C4B3001374980055
:10739000202120000800400024C7B30004487800E2
:1073A00030212000080040000448780040212000DF
:1073B00008004000034878005021200008004000E9
:1073C0000248780078019000880990006021200030
:1073D00008004000024878007121200088804000A9
:1073E0004810DE008048780080212000080040001E
:1073F000401ADE000500200004487800902120009B
:10740000080040004819DE0002487800580190004A
:10741000E8019000A0212000080040000248780008
:10742000B1212000888040004810DE0080487800AC
:10743000C021200008004000401ADE0005002000A6
:1074400004487800D0212000080040004819DE00E0
:107450000248780014C0B30018099000A8099000F1
:107460008A007800184090000CA402000000000080
:10747000594498000001EB008040EB001840900058
:10748000A4A40200000000008004EA0080847400CC
:10749000CF4CDE00090078004F0578004F04BE0095
:1074A00000000600F6874700889FBE008A9FBE0046
:1074B0008C9FBE008E1F78000244780090017800F7
:1074C0001302FB000403B100E90F520009003E0063
:1074D00093429000A2C3B30082CF520005003A004D
:1074E0000388E800B0002000F0B79F00E00F5200D2
:1074F000E6013A007ECE80008E087800C1002000B0
:10750000F1B79F00E00F5700E00132000041EB00AF
:107510009E4F11000F0032001E4090008CA302000D
:10752000000000008080FB006180600009003A00DC
:10753000F0B79F00E04F5400D4013200E4806000B7
:10754000A3002000F3B79F00D0013A00F1B79F00DD
:10755000CE0137000040EB00004F78001047980044
:1075600066A20200000000008080FB0061806000D5
:1075700032002000F2B79F00C4013A00E04F5400EF
:1075800004003200E4806000A3002000F3B79F00F5
:10759000BE013A006011B8000E007800F0FE07004E
:1075A0006066B800E14F50001A003A000EF09300F8
:1075B000D1002000F1B79F00E04F5000B30132002E
:1075C0007EF19300C811DD00020020006EF09300F0
:1075D0008080FB00000020000001710081817100AB
:1075E0004EF093000080FB000100200000017100BC
:1075F000818171005EF093004800DD0001002000F1
:1076000000067100818671000C01BE000E0078003A
:10761000D3FE070012002000F2B79F00E34F500096
:107620009A013200D3002000F3B79F00E04F5000D2
:1076300096013A00AE789000C808DD001E789000F0
:107640000080FB008080700000202000808F5000B0
:107650008E013A005EC590004855DD004EC0900096
:107660000080FB00000575000B002000E00F5500B6
:10767000E08F5D0012003A005ED59000C855DD0035
:107680000A0020004ED090008080FB000000200007
:1076900000057500818575002ED090000080FB00EC
:1076A0000100200000057500818575003ED0900026
:1076B0004800DD000100200000057500818575008F
:1076C0005A0F98006B0F9800EE78900031479800A1
:1076D0000141E900D0002000F0B79F00E14F5100C8
:1076E0006A013E003E799000A2EF9F002247980079
:1076F000E04F510065013200AFE997000381FB00C4
:107700000200E9000201600060013A000EC1900031
:107710004811DD007E7890000080FB0000007100C1
:10772000E0B79F0040079800000178006F006100FB
:1077300056013A002EC190004811DD001EC0900095
:107740000080FB00000171006114B800E00F5400DC
:10775000E08F5C0014003A001ED190000281FB0013
:1077600003002000C813DD00060020000ED19000A9
:107770008281FB00020020000201730083817300FC
:107780006ECC90000884FB00090020000803710003
:10779000898371007EC990004811DD00030020003C
:1077A00002047300838473005E7B90004833DD0025
:1077B0004E7890000080FB0000037300D30020008F
:1077C000F3B79F00310132000182FB000500200069
:1077D0000401BE000A00BE0086BF9F0054040200E0
:1077E0000000000090B79F00A1B79F000FBB97005B
:1077F0006130B800F0AF9F0081B79F00EFB09700F5
:107800004408DE007FA997008FB197000000410077
:10781000E08049001FB19700AFB19700000141001F
:1078200081814900B2B79F00C3B79F00820F540007
:10783000838F5C00150139000203540083835C00D0
:10784000AFE997000382FB00050020000401BE00A1
:107850000600BE0034040200000000000002BE006A
:10786000E00F5000E08F58000801320016C0B3004E
:1078700050FF2000800F5200E08F5A0005003600B4
:1078800036C0B300EB0F4200E08F5A0001003E000B
:1078900026C0B30062044200E0844A00380F98001A
:1078A000490F98003FB19700CFB197000200460002
:1078B00083804E0030179800411798007FA89700EA
:1078C0008FB097000C0140008D814800720F980026
:1078D00003179800E34F53001E003A00D100200028
:1078E000F1B79F006FB19700E00F5100E7003A0039
:1078F0005ED99000C811DD00020020004ED8900033
:107900008080FB0000002000000071008180710079
:107910002ED990000281FB000300200002007000BD
:10792000838070003ED990004811DD0003002000E4
:1079300002007000838070001017980021179800D3
:107940004248DD00CE40DE00810070004240DD0094
:107950001C003700D0002000F0B79F00EFB0970068
:10796000E08F5000C90032001FB09700AFB0970001
:1079700000014100818149001217980023179800E7
:10798000E24F530003003A000800440089804C0095
:107990000C00370032002000030020000800BE0069
:1079A00086BF9F0054040200000000008100D10047
:1079B0000080D3006104640008004000E0804800BB
:1079C0000FBB9700F01FB0000180B0004709DD0039
:1079D0004900DE0000007100C908DE00D30020006D
:1079E000F3B79F00800F5500818F5D00A70039001D
:1079F0000080EB008080EB0070079800010F98007A
:107A00006000B8005007980061079800E34F5300EA
:107A100093003A000040EB00504798007ED9900058
:107A20004811DD006ED890000080FB00000171005D
:107A300002014600E0814E00120F9800230F9800CB
:107A4000E10220008E80400014C0B3001E40900070
:107A500086BF9F0098A30200000000000FBB9700A4
:107A6000E00F50007E003A00D02220000E004000BF
:107A7000104078008080FB00C808DD00C022200094
:107A80000E004000104078000080FB0080807000F5
:107A900050A52A00808F500071003A001E7190009E
:107AA000C811DD00020020000E7090008080FB00F5
:107AB0000000200000017100818171006E6890005B
:107AC0000080FB0001002000000171008181710035
:107AD0007E6890004800DD00010020000001710078
:107AE000818171002025250011162400800F51008E
:107AF000818F59005A003A00502120000E004000AA
:107B000010417800C811DD00020020004021200053
:107B10000E004000104078008080FB000000200034
:107B20000001710081817100202120000E004000C1
:107B3000104078000080FB0001002000000171006F
:107B400081817100302120000E004000104078003B
:107B50000080FB004800DD000100200000017100F2
:107B6000818171002027270011142600800F510009
:107B7000818F59003A003A00D02120000E004000C9
:107B800010417800C811DD0002002000C021200053
:107B90000E004000104078008080FB0000002000B4
:107BA0000000710081807100A22120000E014100BF
:107BB000124178000281FB000300200002007000E7
:107BC00083807000B22120000E0141001241780034
:107BD0000281FB004811DD0003002000020070005C
:107BE0008380700050079800610798009021200062
:107BF0000E00400010417800C811DD000200200096
:107C0000802120000E004000104078008080FB00A2
:107C100000002000000071008180710062212000BE
:107C20000E014100124178000281FB000300200098
:107C30000200700083807000722120000E0141005C
:107C4000124178000281FB004811DD000300200092
:107C5000020070008380700070079800010F980088
:107C6000064F7800D019EC0080CE880030079800CD
:107C70006000B80050179800611798000040EB00B2
:107C8000404798000000EB00F0B79F007FB09700DE
:107C90004F0778004F06BE004F05BE004F04BE00E0
:107CA0006F01B1000000060000017800B000200064
:107CB0008001E900E00F50000A0032001240780015
:107CC0000082FB00914278000580FB00000052001A
:107CD00004003A000201E8008100E8000300780097
:107CE000F3FF3700000006008001780041CC290036
:107CF000010037008100E800114178000200FB001C
:107D0000E04F510002003200830F5000F9FF3A00AB
:107D100000000600E8874700889FBE008A9FBE00DB
:107D20008C9FBE008E1F7800E1B79F0091067800FF
:107D3000F4C2B300C3C5B300010037008D06E800EC
:107D40001D417800844F5100FCFF3200834F5100E9
:107D5000FAFF320090057800B200200001022000F6
:107D60000B007800ADFC07000005EB000A07780067
:107D70008C0020008A44780002C2B30031CD290073
:107D80006D447F000E07E800824F54003300360038
:107D9000F0C2B300804F540030003200C0C5B300C1
:107DA000804F54002D003200E0C2B300804F5400D9
:107DB000020032008C0F55000A003900E80F56000F
:107DC00045003A00E0C2B300804F540042003A0040
:107DD00020002000804CDD000C057800BC00200055
:107DE000E7FF3700E04F540004003D003940B30086
:107DF0000884FB000808B10061447C000880FB0097
:107E000081BF9F00F2B79F00B7FF07008FB89700B0
:107E10007FB19700E00F50002F003A00F0CBB30085
:107E200000404400F94F500002003E000914A00039
:107E300007003700F0C9B30000404400F94F50007C
:107E400003003E000904A00000CEB300004444003B
:107E500088757D000A05E800C9FF37006FB09700FC
:107E60000E8846008040EB0000C2B300804F5400F3
:107E700001003E0041C0B30060002000E00F55004B
:107E80001600320050CEB3009B4F100002003A00A3
:107E900050C0B300804D7800E80F560002003A0051
:107EA00020002000804CDD008984FB00638064009A
:107EB000E10F500001003A000144A000EC8464008E
:107EC000E48F540001003A000134A000B14D980045
:107ED0000000EB0001003700600020004F07780031
:107EE0004F06BE004F05BE004F04BE008F00B1001C
:107EF00000000600881F780000047800620051002E
:107F0000E0805900380A9000C80A900062025200CE
:107F1000E0825A006011B800840F5000858F58002D
:107F200009003100284190000281FB00030020007D
:107F3000540402000000000038119000C8119000A5
:107F400000014100818149000200BE004F04780019
:107F500000000600889FBE008A9FBE008C9FBE0066
:107F60008E1F7800000678000205BE001800200071
:107F700009002000E10F5100E08F59007A0036001F
:107F80003C089000CC089000800F5100818F590070
:107F9000750031001C407800E24F50002F00320085
:107FA000E34F5000450032000084EB008084EB007A
:107FB000E14F50006C003A008206D10082864600F4
:107FC0004969DE007C0890008C109000020140009E
:107FD000E08148000C00780017FC07000084EB00EB
:107FE0008084EB00E00F50005F003A000D00780045
:107FF000F01FB200E002B0006C4778008D06E80088
:108000004969DE007C0890008C109000020140005D
:10801000E08148000C00780007FC0700E00F5000EA
:1080200051003A000E87FB00FD1FB200ED02B000C8
:108030006CC07E004804DD000E047400610565001C
:10804000020032004444DE0002003700FEFF200040
:108050000E04640009002000430037004859DD0089
:108060004850DE0000007100C858DE007C09900016
:108070008C11900000014100818149000C007800C2
:10808000EDFB07000084EB008084EB00E00F500064
:1080900035003A000A054500FA1FB200EA02B000B6
:1080A0006C447D000884FB000A0546001A409000DD
:1080B0004800DD0000047400E6FF37004959DD0088
:1080C0004750DE0000007100C758DE007C099000B8
:1080D0008C11900000014100818149000C00780062
:1080E000D5FB07000084EB008084EB00E00F50001C
:1080F0001D003A004255DD00FA1FB200EA02B0004E
:108100000A004600204190000281FB00030020008D
:10811000C012DD000400200030419000C811DD00D5
:108120000200200002017200838172001040900062
:108130004800DD0001002000000171008181710014
:108140006C407D000080FB000100200000017100F8
:1081500081817100F0FF2000030060008000780042
:10816000020078000004BE000800BE004F0778003F
:108170004F06BE004F05BE004F04BE0000000600C3
:10818000881F7800000478000000EB0020049800AD
:1081900038019000C801900021002000E10F51003B
:1081A000E08F59003D00320018007800300A90003E
:1081B000C00A9000840F5100858F590037003100AC
:1081C000E00F5100E08F590014003A0031C0B300B5
:1081D00090CF100005003A0010119000A0119000FF
:1081E000E00F5100E08F59000C003A006011B80018
:1081F0005204980063049800400190002100200080
:10820000E00F51002500320010119000A0119000E5
:1082100072049800030C980018003700A0409000EA
:10822000E0CF500010003A001800780049FF070026
:108230000001BE00E10F4000E08F48001400320052
:10824000E10F5000E08F580013003600180078004E
:10825000C008900030089000800F5100818F5900B5
:10826000F1FF39000C0037005204980063049800B5
:1082700020FF070070049800010C9800E302200022
:1082800018804100100C98008000EB0003003700BC
:1082900011002000010037002100200001007800BB
:1082A0004F04780000000600889FBE008A9FBE0031
:1082B0008C9FBE008E1F7800000578000204BE006F
:1082C0000406BE0020002000E10F5100E08F59009D
:1082D000960036003A099000CA099000820F5400B7
:1082E000838F5C00910031009A407800E2CF50000B
:1082F00040003200E3CF500052003200E1CF500086
:1083000088003A008805D100888545004959DE007B
:108310007A0890008A10900002014000E081480035
:108320000A00780044FB0700E00F50007D003A008F
:108330000B017800F21FB2006104640008003200F3
:10834000E002200002004000EA407800EFC0600038
:108350000C80FB004400DD0000C07000010037000D
:108360000C40780002014500606998008B05E80028
:1083700010C0B300404598004959DE007A089000CB
:108380008A10900002014000E08148000A00780055
:1083900029FB0700E00F500062003A00FB1FB2000B
:1083A000E00F540005003200CC68DD004466DE00BA
:1083B0000C867000C46EDE000B003700E102200066
:1083C0008B8040006AC1780001CFB300814061001A
:1083D0004869DD004866DE000C067100C86EDE00EC
:1083E0006F4666000CC670008B054500EC6D98006A
:1083F0004C003700484ADD004840DE0000007200B3
:10840000C848DE007A0990008A11900000014100FE
:10841000818149000A00780007FB0700E00F500047
:1084200040003A0008044400F81FB20088004500EC
:10843000EC689800010478004866DE007C6C9800C7
:10844000380037004949DD004740DE000000710078
:10845000C748DE007A0990008A11900000014100AF
:10846000818149000A007800F3FA0700E00F50000C
:108470002C003A004244DD00F81FB200EE0220005A
:10848000080747008E004500E38540008184E8002E
:10849000194178000281FB0003002000C012DD00BA
:1084A000040020001B417800C811DD0002002000FC
:1084B0000201720083817200514278000483FB0044
:1084C0004833DD000700200006027100878271003A
:1084D0006A417F000281FB0003002000020172005C
:1084E0008381720004002F0003016200030020005A
:1084F000C011DD00020020000C0671008D867100A5
:10850000080445006C6C98004861DE0082487800E1
:108510004069DE0003002000824C7800486EDE00D7
:108520008C4D780011C0B300414598004F0778008A
:108530004F06BE004F05BE004F04BE0000000600FF
:10854000889FBE008A9FBE008C9FBE008E1F780051
:10855000000778000204BE00E00F5100E08F5900D0
:108560000B003A005E069000EE069000E00F560009
:10857000E08F5E00120032003E089000CE089000AE
:10858000800F5600818F5E000F0039000C0037000D
:108590000E0078006FFE0700E10F5000E08F5800DA
:1085A0004D0036003E099000CE099000820F500029
:1085B000838F58004E0039000806BE0002003700C5
:1085C0001C0020000D0020000C05BE0061054500C8
:1085D000E0854D003E089000CE089000800F5500C9
:1085E000818F5D0005003900E10F5600E08F5E00CD
:1085F0003C0036002A0020000B0020000A01BE00CB
:108600000E00780053FE0700E00F5000E08F580086
:108610000A003200E10F4000E08F480034003200D1
:10862000E10F5000E08F5800310032008C0F5500F0
:108630008D8F5D00E5FF3A002A003700F4FF2F0020
:10864000F5FF20000A01BE000E00780016FF0700AB
:1086500000017800E00F510018003A00E00F5400CC
:10866000E08F5C00070032000A02BE000801BE0075
:108670000E0078000CFF070000017800E00F5100A9
:108680000E003A005A0798006B0798007E00900091
:108690008E089000E10F4000E08F48001300320088
:1086A00061005000E080580070079800010F9800AA
:1086B00010C0B300504798000C0037001000200095
:1086C00001002000E10F510009003A000080EB009A
:1086D0008080EB0006003700100020000100200021
:1086E000030037006000B800010037000A00BE0038
:1086F0004F0778004F06BE004F05BE004F04BE0076
:1087000000000600E4874700889FBE008A9FBE00E5
:108710008C9FBE008E1F780000057800010678004F
:10872000AA0690008D06E8004B0020007C00320075
:108730007A0090008A089000E00F5000E08F580007
:10874000770032006F8766006C003A0061004000DD
:10875000E080480070059800010D98005A019000D3
:10876000EA0190001A007800E00F5100E08F5900F4
:1087700004003A0040009000808F56005F003900EE
:1087800067003700A04090008180FB008100E90075
:10879000446ADE008480600058003A00EDFD070066
:1087A0000004BE002B002000E10F5000E08F5800B5
:1087B0005B0036001B002000E10F4000E08F480006
:1087C000570032001A00780030099000C00990006C
:1087D000820F5400838F5C00410039004B00200061
:1087E000E00F56004E0032005A019000EA0190005E
:1087F00053FF07000004BE007B002000E00F500084
:10880000E08F5800460032002B002000E10F50009E
:10881000E08F5800420032001B002000E10F4000B2
:10882000E08F48003E0032006011B8001A00780066
:1088300001FA070000067800E00F560038003A0001
:10884000E10220001A804000022020008C00780005
:10885000F2F907001A0278000801BE00040078004F
:1088600084BF9F00A3FD07000FBA97005012980025
:10887000611298000E0037004B4098006011B8005C
:108880001A007800ECF90700E00F500023003A00CE
:108890001A01780052109000E21090006100400030
:1088A000E080480050119800611198000C46E800E3
:1088B0001A007800A0409000814F5600EEFF39006A
:1088C0000C81FB000300200050129000E012900089
:1088D0000201520083815A005210980063109800E0
:1088E00058059800690598000801BE001A00780034
:1088F00080FD070070059800010D98002D05980077
:10890000E10220001A8040004577DD000E0740009C
:108910001E0D98008005EB00010037001B002000B1
:108920000B0078004F0778004F06BE004F05BE00D1
:108930004F04BE004F00B10000000600889FBE003B
:1089400080047800090078000DFE0700000478001C
:10895000E00F540017003A00790190008909900057
:1089600019007800B4F9070000047800E00F540003
:1089700010003A00190890008040EB0090CF1000E2
:108980000B003200B0489000E880600004003A001C
:10899000A9089000C4FC0700E00F50000500320059
:1089A0008000EB000900780056FF0700E7FF370062
:1089B00048002000080078004F04BE0000000600B8
:1089C0000200FA00889FBE0000047800D1BF9F001B
:1089D00011407800F2C2B300824F50000300320011
:1089E000C2C5B300824F500002003A008100E80087
:1089F000D1BF9F006000B800300498004104980087
:108A00005FB89700F1C1B30090CF100005003E00A1
:108A100008007800DAFD07008000EB00110C9800D8
:108A20002B003700F4044400E6805700090078006A
:108A3000B8FC0700E00F500025003A00080078005D
:108A4000BEFF0700A8089000B1489000E00F50005A
:108A500005003200E40F50001D003A00E480600081
:108A60001A0032001A003700E480600018003A0053
:108A700098089000314890007000600013003200A8
:108A8000515190004811DD00415090000080FB00E2
:108A90000001710003002000C011DD000200200071
:108AA000315A90004822DD00A15890008180FB00DF
:108AB000010272000500200004017100858171002F
:108AC0003204980043049800D7FF3700500020007C
:108AD0004F04BE000080FA0000000600889FBE0020
:108AE0008A1F78008004780009007800A4FD070040
:108AF00000047800E00F54001D003A007901900056
:108B000089099000190078004BF9070000047800EB
:108B1000E00F540016003A00190890001040780049
:108B2000FB4F400016003200E04F500014003200AE
:108B30001100200009007800F2FE0700ECFF37006A
:108B4000190D900002022000880078000A007800C9
:108B500032F90700B2002000A90890000A0078004E
:108B600027F907009900780010C0B300C0409800B2
:108B7000080078004F0578004F04BE000000060092
:108B80007901900089099000190078002AF90700FE
:108B900000047800E00F5400F5FF3A00E8FF3700CA
:108BA000889FBE008A9FBE008C9FBE000006780092
:108BB0000204BE0020002000E10F5100E08F5900A8
:108BC0002F0036003C099000CC0990001DC0B30076
:108BD000820F5400838F5C001F003900280037008B
:108BE0000801BE000C007800DAFC07000005BE009A
:108BF000E00F5000E08F58001C003200E10F5000E1
:108C0000E08F58001B003200E10F4000E08F480069
:108C10001A0032006022B8000801BE000C00780083
:108C2000A1FD0700E00F500015003A007C00900005
:108C30008C089000E10F4000E08F480005003200F2
:108C400061004000E080480070069800010E980026
:108C50005D4698000A04BE003C089000CC089000D5
:108C6000800F5400818F5C00DDFF39000000EB00B5
:108C70000300370020002000010037001000200012
:108C80004F06BE004F05BE004F04BE0000000600A8
:108C9000B2002000E04F500009003A0072CE800080
:108CA000E00F51000100320000497800E08F5000D1
:108CB000010032008048EB0071CE88000001EB001B
:108CC00002007800000006006F02B000889FBE001E
:108CD0008A9FBE008C9FBE008E1F78000007780020
:108CE00081BF9F00000FEB00FF4661007E416100E5
:108CF000A1FD2F008F80400070805700E9F9070028
:108D0000E1FC2F008F804000F1B79F00E00F500082
:108D100004003A008FB89700A0FD2F000F0040001C
:108D200027FF07006FB69700E00F500003003A00DE
:108D3000E00F560001003A00600020008D80FB002B
:108D40007C81600055003200E00F50000A003200C4
:108D5000E40F500003003A00A0FD2F000F00400078
:108D60005EFF07006FB69700E00F500090003A00DA
:108D70000D34A000070037003C49900071016100EC
:108D8000700020008A003A00E4806000800020002B
:108D900087003A00688066004C00320070AF020025
:108DA00000000000604E98004801DE00724E9800FE
:108DB0004009DE0003002000025698004808DE004B
:108DC000105698008040EB00314E9800415E9800AC
:108DD000515E9800615E9800715E980075004600D3
:108DE00074024600FB0246007A03460010417800F8
:108DF0000284FB004844DD00944178000381FB00BD
:108E00000204740009002000C044DD0008002000B6
:108E1000954378000781FB004811DD0096437800F8
:108E20008781FB000301710003002000020474002D
:108E300083847400014B7800814A7800014A7800ED
:108E4000014878005FA8970011C0B3004140980026
:108E5000E00F5400E08F5C001C00320050159000C1
:108E6000E01590000801BE004DFF0700E00F500024
:108E70004F003A005FA8970061045400E0845C0052
:108E800058009800690098000A01BE006AF80700BF
:108E9000E00F50000D00320045003700E00F500099
:108EA00043003A003C4990000281FB00F001610060
:108EB000400020003E003A00E280600003003200E3
:108EC000610161007000200039003A00688066008E
:108ED000010032000D54A0005FAA970054109000CA
:108EE000E4109000500F9800610F98007C0F9800DC
:108EF0004D479800DC509000C808DD004C509000B1
:108F00000080FB000080700001002000C000DD0038
:108F100000002000BC599000C819DD002C599000B9
:108F20000281FB000281710003002000020070003A
:108F30008380700070079800010F98007C599000A2
:108F4000C811DD00020020006C5890008080FB00FA
:108F50000000200000007100818071004C599000D9
:108F60000281FB000300200002007000838070007B
:108F70005C5990004811DD000300200002007000E1
:108F80008380700050079800610798006000B80067
:108F90003007980041079800300F9800410F980063
:108FA000040F780034029000140798000000EB00D2
:108FB0004F0778004F06BE004F05BE004F04BE00AD
:108FC0006F02B10000000600EA874700889FBE00DC
:108FD0008A9FBE008C9FBE008E1F7800000578001F
:108FE0000104780082057800E3B79F008009EB0058
:108FF0009A0090001A007800ADF80700000778008A
:10900000E00F5700B4003A004A429000E04F52008F
:10901000AE00350061026200AE0032005A029000DC
:10902000EA0290003A019000CA0190000202520048
:1090300083825A00615BB800840F5300858F5B0008
:10904000010036008405780088BF9F0000022000E0
:1090500000004500F0B79F008E007800D1B79F0058
:109060000B077800950037003A019000CA01900084
:10907000F01F20000202600074003A001A0078001D
:10908000C91ADE00C718DD004912DE000482700034
:10909000A04590008B45E90084C5650011003A00A9
:1090A000E00F5100E08F590003003A007A00900071
:1090B0008A089000030037001A099000AA0990005E
:1090C000A4FB0700E10F5000E08F58000D003600B0
:1090D000E10F4000E08F480055003200100D98006D
:1090E000210D98001A0678001A099000AA0990002C
:1090F0000C0078007FFB0700E00F5000E08F580065
:1091000004003A004A4090000074A00040459800D6
:109110006E0037000B84FB000900200000044400AF
:1091200081844C00C976DE00220032002C41900080
:109130008B85FB008B8146000281FB00828F5100F2
:10914000010036008B0651000D4278000801BE0078
:109150008FB897001C40900098A302000000000008
:109160004A429000E00F500023003A000404B2008D
:109170000E0032003A089000CA0890000800500023
:10918000898058006169B800820F5000838F5800B1
:10919000060031004900DD008FB8970000804000D4
:1091A00002202000FFB0970095F70700496CDD0012
:1091B000360037003A089000CA089000880F500027
:1091C000898F58001F0032004A4190000204B2000B
:1091D0000E00320014C0B3000001BE00FFB09700C3
:1091E0001C4090000CA40200000000004A429000C5
:1091F000E00F5000030032000474A00044459800C2
:109200000E0037000464A100444598001A0078005D
:1092100014C0B3000801BE00FFB0970010409000DA
:1092200098A3020000000000E00F5000050032008B
:109230004A4090000074A000404598001E002000A5
:1092400025003700380D9800490D98003A0190002C
:10925000CA01900082017800F31FB20000202000B4
:10926000030150000E047800820F57000100360001
:1092700002047800FFB09700838140000801780065
:10928000830078000FB897005DF707000FB89700CC
:109290000800400080BF9F003A019000CA01900082
:1092A00008014100E081490032059800430598001B
:1092B000EFB097009108440008075700E00F5700EF
:1092C00069FF3A005FB79700030037002E002000C7
:1092D000010037007E0020000E0078004F07780064
:1092E0004F06BE004F05BE004F04BE00AF00B100E8
:1092F00000000600EA874700889FBE008A9FBE00E4
:109300008C9FBE008E1F7800000578000104780055
:1093100082057800E3B79F008009EB009A00900077
:109320001A007800E2F7070000077800E00F570006
:10933000D6003A004A409000E04F50005F003500F0
:1093400062006000D00032005A029000EA029000F1
:109350000B034200E0834A00840F5300858F5B00BB
:10936000010031008E05780088BF9F0000022000B8
:1093700000004500F0B79F008E007800D1B79F0035
:109380000B077800B00037003A019000CA01900046
:10939000F01F2000020260008E003A001A027800DE
:1093A000C91BDE00C718DD004913DE00068370000C
:1093B000A44590008B45E90086C5650021003A0070
:1093C000E00F5100E08F59000B003A007A00900046
:1093D0008A089000E00F5000E08F58000D003A001E
:1093E0000001BE000400780055FC070070059800DD
:1093F000010D9800040037001A099000AA09900096
:10940000040078004EFC0700E00F5000E08F580089
:109410008F0032004A429000E10F5000E08F580068
:1094200003003A000474A00044459800230037006C
:10943000E10F4000E08F480010003200100D98004E
:10944000210D98004A4190000204B2001000320041
:109450001A00780014C0B3003A099000CA099000BD
:10946000FFB09700104090000CA402000000000024
:109470004A429000E00F5000030032000474A00044
:10948000444598004F0037000464A100444598000B
:109490001A0678001A099000AA0990000C007800BA
:1094A00094FA0700E00F5000E08F580005003A00E2
:1094B0004A4090000074A000404598002E00200013
:1094C000720037000B84FB000900200000044400F8
:1094D00081844C00C976DE00230032002C419000CC
:1094E0008B85FB008B8146000281FB00828F51003F
:1094F000010036008B0651000D4278000801BE00C5
:109500008FB897001C4090000CA4020000000000DF
:10951000E00F500028003A003A089000CA08900076
:1095200008005000898058006169B800820F50001F
:10953000838F58000A0031004900DD008FB8970082
:109540000080400002202000800078007FB097005B
:10955000ABF607004A4190000264A1004245980022
:10956000496CDD002C0037003A099000CA099000D0
:10957000880F5100898F5900140032003A02900080
:10958000CA0290005A019000EA019000820F520036
:10959000838F5A000D00310014C0B3000801BE00D3
:1095A000FFB097001C40900098A30200000000004C
:1095B000E00F5000050032004A4090000074A00007
:1095C000404598001E00200030003700380D9800FC
:1095D000490D98003A009000CA009000F01FB200B8
:1095E00001202000008150000E047800820F5700F7
:1095F0000100360002047800FFB0970000804000B0
:10960000080178008FB897007DF607004A41900066
:109610000264A000424598000FB89700080040007F
:1096200080BF9F003A019000CA01900008014100EC
:10963000E08149003205980043059800EFB097009B
:109640009108440008075700E00F57004EFF3A000A
:109650005FB797003A019000CA0190005A0090004D
:10966000EA009000800F5100818F590002003600FF
:109670005205980063059800CA4090000154A0006C
:1096800041459800010037007E0020000E00780060
:109690004F0778004F06BE004F05BE004F04BE00C6
:1096A000AF00B10000000600889FBE0000047800F3
:1096B0009800900018007800FDF60700E00F5000B9
:1096C00042003A00C84090008180FB000101780010
:1096D0000202B2003D0032000104B200100032006C
:1096E00001022000888040001800780014C0B300F8
:1096F00038099000C8099000104090000CA40200A6
:10970000000000008000780010002000E08F500072
:109710002E003A00484090000064A10040449800A8
:1097200058099000E80990001800780042F60700F8
:10973000E00F500025003A00F80C90006B804400C8
:109740001054A00028489000C05C98003848900051
:10975000D05C980048489000E05C98005848900021
:10976000F05C980068489000A05C980078489000F1
:10977000B05C980008509000C054980018509000B9
:10978000D054980070AF020000000000E054980030
:109790004801DE00F25498004009DE00030020007A
:1097A000825C98004808DE00905C98004840900079
:1097B0000054A100404498009800780010C0B30005
:1097C000C040980018007800CAF607004F04BE0099
:1097D00000000600881F7800000478000800780068
:1097E000B1FF0700E00F500001003A00000C7800C4
:1097F0004F04780000000600EA874700889FBE00FB
:109800008A9FBE008C9FBE008E1F780000077800E4
:109810000205BE009E0090001E007800A4F607001E
:10982000D0B79F00E00F5000E3003A004E41900097
:10983000E04F5100DE0035005E009000EE00900029
:10984000800F5500818F5D000300360062016100CA
:1098500001003A000005BE003E069000CE069000D2
:109860006000B8003007980041079800E00F5500ED
:10987000E08F5D00940032001E03780026419000C6
:109880000281FB0003002000491CDD00C714DE003C
:10989000890474004914DD00E00F5600E08F5E007B
:1098A0002300320061065600E0865E00610055002C
:1098B000E0805D000801BE0086BF9F003404020006
:1098C000000000000002BE000801BE000C00BE0047
:1098D000E4B79F00F5B79F003404020000000000C9
:1098E0006FB29700FFB297000FBB9700800F520036
:1098F000818F5A000E00390060001400E0801C00C7
:109900000003660001826600840278000602780087
:109910000401BE0032079800430798000205550075
:1099200083855D001E099000AE099000120037008B
:109930007E0190008E099000E00F5100E08F5900E9
:109940000B003A0006007800FDFA07000001BE0097
:10995000E10F5000E08F58004D003200E10F400051
:10996000E08F48007D00320070079800010F9800DA
:10997000120F9800230F9800E00F5100E08F59005C
:109980004E0032002C003700CE409000E280600094
:10999000070032001E007800E9FA07000001BE004F
:1099A000E00F5000E08F580004003A002600370016
:1099B0001E00780067F907000001BE00E10F4100BA
:1099C000E08F490004003A004E4090000074A0006F
:1099D0004047980053003700E10F5100E08F5900D5
:1099E000060036009E007800310A9000C10A9000FF
:1099F000840F5100858F5900050039004E409000BA
:109A00000074A00040479800220020005700370053
:109A1000120F9800230F98003E029000CE02900093
:109A20000402440085824C003407980045079800E2
:109A30000805550089855D00880F5500898F5D00F8
:109A4000D1FF3E00010037000805BE003E02900035
:109A5000CE0290000402450085824D003407980034
:109A6000450798000A027800F41FB20005002000A4
:109A7000E00F5200E08F5A00120032001E00780002
:109A80001CF90700E00F5000E08F580004003A0076
:109A90004E4090000074A0004047980044003700FA
:109AA0004759DD004955DE000A057100C95DDE0039
:109AB0000005450081854D00030037000205BE000A
:109AC000010037000405BE003E009000F01FB20008
:109AD0002A0032003E099000CE099000820F550006
:109AE000838F5D00250032004E4090000004B200DC
:109AF00010003200010220008E8040001E0078001D
:109B000014C0B300104090000CA40200000000003C
:109B1000CE409000E00F5000040032000174A0001D
:109B20004147980010002000220037000164A10086
:109B300041479800010220008E8040001E007800FE
:109B400014C0B3000A01BE001040900098A30200A8
:109B500000000000E00F5000060032004E40900070
:109B60000074A0004047980012002000D2B79F0068
:109B7000110037003A0F98004B0F98003E009000FC
:109B8000CE0090005E019000EE019000820F500028
:109B9000838F58000800360050079800610798002E
:109BA0004E4090000054A00040479800020037004B
:109BB00020002000D0B79F005FB097004F077800CB
:109BC0004F06BE004F05BE004F04BE00AF00B100FF
:109BD00000000600FF4F500002003E008040780069
:109BE000060037008040EB00F2C3B300824F500004
:109BF00002003E0001C4B30080C050000140780064
:109C000000000600889FBE008A1F7800800478004C
:109C1000F24FEC00F2EFB70001C6B300814F5000E5
:109C200001003600F26FEF0021FF20009140780024
:109C3000814C78000904780000C2B30000C14000E4
:109C4000026C780000C6B300804F5100010036005E
:109C5000004C51000985E8000144B000014D780036
:109C600000C6B30080CF50000100360000CD500088
:109C700019407800D7FF0700804C78001840780022
:109C8000D4FF0700004C78001A407800D1FF07008D
:109C9000004D78004F0578004F04BE00000006001C
:109CA000800078000000EB00E48F500009003200D3
:109CB000E88F50000700320010002000E08F5000B5
:109CC00004003A00307F80008000EA0000807000CD
:109CD0004F00DE0000000600889FBE000004BE00AA
:109CE000090444000100370069045400E80F5400DF
:109CF000FDFF3C000100370069044400E00F540000
:109D0000FDFF350008007800E5FF0700E00F500078
:109D1000F3FF3200080078004F04BE000000060088
:109D200001002000E80F5000E08F58002B003E009B
:109D30000060010008003700090037000B00370001
:109D40000E003700110037001300370015003700F0
:109D5000180037001C0037000041EB000C003700F2
:109D60000041EB0001C2B300140037000041EB00DA
:109D700001C2B30001407800110037000041EB0040
:109D80008240780000C2B3000D00370002C2B30069
:109D900082407800F7FF370002C2B3008040EB003A
:109DA000F4FF370002C2B300824078000040EB00AD
:109DB0000300370002C2B3008040EB00024078008D
:109DC00002C004000000000052C0B300F1C0B300A4
:109DD00000C2B30002C00200000000000000060044
:109DE000881F78000004780008007800CCFF070086
:109DF0006140B800E80F5000E08F58003E003E0080
:109E00000060010008003700090037003700370004
:109E10000D00370035003700170037001F003700EE
:109E200030003700310037000000210030003700DB
:109E300040002000F463020000000000F2AA0200CB
:109E4000000000002C00370000102000F463020026
:109E50000000000040002000F46302000000000049
:109E60000041EB0082407800F0C0B30002C0020065
:109E7000000000002000370040002000F4630200D2
:109E80000000000000012000F46302000000000058
:109E9000600F2000704688001700370080ED290011
:109EA000C6B102000000000000047800E00F54007A
:109EB0000E003A00210020008097210054B20200D9
:109EC0000000000021002000A097210054B20200F1
:109ED0000000000008007800C6B102000000000089
:109EE00002003700EA2FEF00EC2FEF0040002000C7
:109EF000F4630200000000004F0478000000060038
:109F00000400FA00881F7800000478000001EB00CC
:109F10006000B800A6C00200000000008043EB0013
:109F2000074378008742780007427800874178002D
:109F3000074178008740780007407800B2BF0200F0
:109F4000000000008040EB0000C1B300BEBE020074
:109F5000000000008040EB0010C1B300BEBE020054
:109F6000000000008040EB0040C1B300BEBE020014
:109F7000000000008040EB0050C1B300BEBE0200F4
:109F8000000000008040EB0020C1B300BEBE020014
:109F9000000000008040EB0030C1B300BEBE0200F4
:109FA000000000008040EB0060C1B300BEBE0200B4
:109FB000000000008040EB0070C1B300BEBE020094
:109FC000000000008040EB0001407800BEBE0200AF
:109FD000000000008040EB0010C0B300BEBE0200D5
:109FE000000000006140B800E80F5000E08F58000A
:109FF00051003E00006001000800370009003700F2
:10A000000E0037000A003700480037000F00370005
:10A010001F003700430037004400370000002100D4
:10A0200043003700FCAA02000000000003003700D4
:10A03000001020000C64020000000000400020001E
:10A040000C640200000000000E00370040002000F9
:10A050000C64020000000000000120000C640200FB
:10A06000000000008040EB00E0C1B300BEBE020073
:10A0700000000000CE28EF00F1BF2F0080CD2000AF
:10A0800010886000AC28EF00AE28EF002A003700EF
:10A0900080ED2900C6B1020000000000E00F500072
:10A0A00020003A00D0BF9F00E0BF9F0021002000A9
:10A0B0006680570054B2020000000000210020001A
:10A0C0006480570054B2020000000000C0CB800042
:10A0D000DFB89700808F500004003A00D0CB80009A
:10A0E000EFB89700808F50000B0032006000B8007E
:10A0F00014B202000000000021002000809721001F
:10A100009CB202000000000021002000A097210066
:10A110009CB20200000000000000EB00C6B102008B
:10A1200000000000AC28EF00AE28EF004000200047
:10A130000C640200000000004F0478000080FA0068
:10A1400000000600FE4FEC0080407800010078001F
:10A15000FEEFB7000100FB00E0CF50000800340024
:10A1600082C2B30082CF50000B00340001C8B3009C
:10A170008000FD00FEEFB7008000FD00000006003B
:10A1800042002000811F7800110009000200D80061
:10A19000CF0078000000EA00000006000400FA008A
:10A1A000889FBE008A9FBE00984380000005EB0098
:10A1B000100020009103200080804000818040003A
:10A1C00002802000E2807800888F50000200340076
:10A1D00000057800010478000000E800E40F50005A
:10A1E000F4FF3400E0CB800062051500220020005F
:10A1F000801F7800110009000200D800800078005C
:10A200004F00780001D5B900C9DA2000890F540049
:10A210000C00340001FA2000810F540007003C00BC
:10A2200088845400809FBE00110009008204D80079
:10A23000800478004F00BE00110037008004EA005F
:10A240000F00370071BB2000810F540004013C0057
:10A25000813EB100810F54000B00340089C12F00F2
:10A260008884440092FF2F00809FBE0011000900E7
:10A270008204D800800478004F00BE00C912B000EC
:10A28000808F540001003400800478008000EA00D0
:10A29000818F540001003D0081047800311F2000AF
:10A2A000810F54000A003C0001FF2000914078001B
:10A2B000E0CF500003003200604588007045880000
:10A2C00007003700AC28EF00AE28EF00040037008D
:10A2D0000A804400704588000A8054006045880068
:10A2E000F0CFBF004240A90014003400F1CFBF00FE
:10A2F000120032006C80570042FE07006FF1970099
:10A30000DFF097004FF0970002C00200000000004D
:10A310005FF19700CFF097006FF097003AC002000E
:10A32000000000004FF19700EFF097005FF09700FA
:10A330001EC00200000000000600370081FF070079
:10A340000001EB00800078000000EB00A6C00200D6
:10A350000000000007FF200097437800E0CF530083
:10A3600016003200EFCFBF007E59B400EFEFB70008
:10A37000FE4F5000020036007EF9EF000400370067
:10A38000E04F500002003A0010C0B3007EF9B70061
:10A39000F5FE2000954278008580FB004309DE0031
:10A3A000C408DE00814378000243780004C2B30091
:10A3B000854178000040EB00070037000743780034
:10A3C00005C2B30005427800854178000741780056
:10A3D0008740780007407800B2BF0200000000000C
:10A3E000DFD7BF000080FB000000EA004F00DE0066
:10A3F0008000EB00E04F500005003200C1932100C7
:10A40000914078008180FB008100E900CF08DE00E8
:10A410003CF9B700E08F500007003200E1CB80002C
:10A420002103B000E1CB8800401F2000808F500046
:10A4300001003400E0CB8800DCD7BF000080FB00C7
:10A440000000EA004F00DE008000EB00E04F50000B
:10A4500005003200B1932100914078008180FB001B
:10A460008100E900CF08DE003BF9B700E08F500023
:10A4700007003200E1CB80002103B100E1CB88006E
:10A4800040ED2F00808F500001003D00E0CB8800A0
:10A4900010C0B300411F2000810F540003003C0096
:10A4A0000040EB008000EB0005003700A193210085
:10A4B000914078008180FB008100E900CF08DE0038
:10A4C0003AF9B700E08F500003003200600020002E
:10A4D00052DE020000000000E00F55000D003A00BF
:10A4E000E08F540060003A00F1CFBF005E003A00F8
:10A4F000401F2000800F54005B00340010C0B300E8
:10A50000F1EFB7007000200052DE020000000000F2
:10A5100001003700F16FEF00100820004145800076
:10A52000808F50000300340051458000808F500020
:10A5300008003C00AC28EF00AE28EF0001C2B300D9
:10A5400080C0B300BEBE02000000000001C2B30024
:10A55000050037008040EB0080C0B300BEBE0200A3
:10A56000000000008040EB00B0C0B300BEBE02009F
:10A5700000000000F0CFBF00020032000040E90000
:10A58000F0EFB700D8ECAB003B003200F1F72F0042
:10A5900080CD200010886000F06FEF0072448000D2
:10A5A0008E28EF000004EB00100020007104200052
:10A5B000808040008181400004802000E481790097
:10A5C000828F5100020034000004780003017800FB
:10A5D0008180400003802000818041008008EB00E2
:10A5E0000000E800E60F5000F0FF340080BB2000C0
:10A5F000800F510020003400F84488009C08ED00D2
:10A60000E20F50001C003E0010C0B300E20F5400E7
:10A61000030032000040EB008000EB000500370033
:10A6200091932100914078008180FB008100E90036
:10A63000CF08DE0039F9B700E08F50000300320088
:10A640007000200052DE020000000000E20F540003
:10A6500009003A0060C0B300F0EFB7000600370011
:10A660008004EB0006FF3700301F2000800F5400ED
:10A67000A8FF3400A8FF37004F05BE004F04BE00FE
:10A680000080FA0000000600EE874700889FBE00A9
:10A690008A9FBE008C9FBE008E1F78000E0078003F
:10A6A0000F077800AE01B10003000900001FEB00A6
:10A6B00000077800A3FE07000041EB00804078000F
:10A6C00002C0020000000000F3CFEC00F3EFB7007F
:10A6D0008080FB00C508DE0002C2B300FA8157008B
:10A6E00082F178007F4060008101E900E78161002C
:10A6F0000041510002427800FA82570084F279004A
:10A700008100E800E78060000041780082F2780074
:10A71000DFEB97004FEB9700BFEA97002FEA970017
:10A720009FE997000FE99700FFE097006FE097001F
:10A73000B2BF020000000000DFD7BF000080FB00B6
:10A740000000EA004F00DE008000EB00E04F500008
:10A7500005003200E1932100914078008180FB00E8
:10A760008100E900CF08DE003EF9B700E08F50001D
:10A770000700320001CC80002103B00001CC88002A
:10A78000401F2000808F50000100340000CC880062
:10A79000DCD7BF000080FB000000EA004F00DE00B5
:10A7A0008000EB00E04F500005003200D193210003
:10A7B000914078008180FB008100E900CF08DE0035
:10A7C0003DF9B700E08F50000700320001CC800057
:10A7D0002103B10001CC880040ED2F00808F500094
:10A7E00001003D0000CC88000ACC8000E00F55003D
:10A7F0005300350098438000A1438000C643800089
:10A80000D24380006116B9006142B9000C064200D3
:10A810008D864A00018040006102B9000C064200AA
:10A820008D864A00B04380006302B900CFA2DE00EB
:10A830000C0642008D864A00060043006102B90002
:10A840000C0242008D824A00D0FF2F000088B90020
:10A85000CF80DE00C3FF2F0003C4B900CFC4DE00E9
:10A860000000440081804C006333B900CFB3DE00A8
:10A870000000430081804B004211DD00CF91DE00DB
:10A8800000064100818649000C0042008D804A008C
:10A890006154B9000801BE00F4B79F0085BF9F0056
:10A8A00054040200000000000E7D2000811F78008B
:10A8B000110009004E08D800CF007800800555002F
:10A8C0006B4588007FB297008FBA97000C0052004A
:10A8D0008D805A000801BE005404020000000000F0
:10A8E000811F7800110009004E08D800CF007800C1
:10A8F000000555007A45880081DA2F00818F5500C8
:10A9000001003D0061458800810F550002003D00B7
:10A9100080DA2F0070458800802520006145800086
:10A92000808F5000010034006045880080252000A1
:10A9300071458000808F5000110034000F003700F7
:10A94000F24380000A91B90044ED2F001100090084
:10A950004419D800000178000A01410062458800CE
:10A96000E04380000A80B900811F780011000900CF
:10A970004408D800CF0078000A00400070458800E5
:10A980001008200041458000808F500003003400F3
:10A9900051458000808F500008003C00AC28EF003B
:10A9A000AE28EF0001C2B30080C0B300BEBE0200FB
:10A9B0000000000001C2B300050037008040EB003A
:10A9C00080C0B300BEBE0200000000008040EB006B
:10A9D000B0C0B300BEBE0200000000004F07780008
:10A9E0004F06BE004F05BE004F04BE00EF00B10091
:10A9F00000000600889FBE0010CC80008000400050
:10AA00008080400000468000E00F500001003D00C3
:10AA10000000EA008080400010468000E00F5000F7
:10AA200001003D000000EA008080400020468000D8
:10AA3000E00F500001003D000000EA0000804000EF
:10AA40004200DE0010CC880018002000ED0F5000FE
:10AA5000010036000004EB0011C0B300EE0F5000FF
:10AA600003003E008040EB000000EB0004003700D4
:10AA700041D9BF000080FB000000E9004F00DE006C
:10AA80008000FD0041F9B7008000FD00E00F50009C
:10AA9000050032000041EB0082407800F0C0B300B6
:10AAA00002C002000000000010CC8000ED0F50003A
:10AAB00011003E00F40FEC00A07F8800E50F50006D
:10AAC00007003400EA0F500001003A00F42FEF00B5
:10AAD0000041EB008240780000C2B3000300370061
:10AAE0000041EB00824078000240780002C0020082
:10AAF000000000000500370092FD07000001EB0098
:10AB00008000EB00A6C0020000000000B0468000FC
:10AB1000E00F500004003200D628EF005000200063
:10AB200052DE020000000000A1438000803E2000B1
:10AB3000808F500017003400B2438000800F510016
:10AB400014003400C2438000800F51001100340013
:10AB5000E2438000800F510003003C00F24380007C
:10AB6000800F51000B003400200820004245800077
:10AB7000800F51000700340052458000800F5100C3
:10AB800004003400AC28EF00AE28EF0018002000CD
:10AB90006600370093438000803E2000C24380005F
:10ABA000808F51000A003C00808F500008003C005C
:10ABB000B4438000800F520005003C00800F51001C
:10ABC00003003C00D4438000800F52004500340055
:10ABD000D04380004500200080037800811F78006A
:10ABE000110009008500D8008003FD00CF00780027
:10ABF0005400200000037800811F78001100090034
:10AC00008401D8000003FD00CF0078008683430054
:10AC1000B6438000809FBE00110009000503D800E4
:10AC2000000378004F00BE008683430000037800D5
:10AC3000811F7800110009000501D8000003FD0004
:10AC4000CF0078008682430000037800811F7800DF
:10AC5000110009000400D8000003FD00CF007800B7
:10AC600086824200801F7800110009008400D8000D
:10AC7000800078004F00780064002000809FBE00B4
:10AC8000110009008401D800800178004F00BE0047
:10AC900083804000A6FF2F00811F7800110009006B
:10ACA0000600D80000037800CF007800068040003E
:10ACB000B6FF2F00809FBE00110009000601D800DA
:10ACC000000378004F00BE000601400002804200F1
:10ACD0000000EA0060458800850251007545880043
:10ACE00012003700E3438000F1438000808F510061
:10ACF00002003C00808F50000A0034004200200017
:10AD0000811F7800110009008201D800CF0078006F
:10AD100060458800110009008200D8007045880055
:10AD200002003700AC28EF00AE28EF00100820002A
:10AD300041458000808F5000030034005145800061
:10AD4000808F50000B003C00AC28EF00AE28EF00D5
:10AD50000041EB008240780000C2B3001EC0020038
:10AD6000000000000041EB008240780000C2B30008
:10AD7000080037000041EB00824078000240780074
:10AD80001EC00200000000000041EB00824078007D
:10AD9000024078003AC002000000000080DA2F0074
:10ADA00061458000808F500001003D0060458800B3
:10ADB00080DA2F0071458000808F500001003D0037
:10ADC000704588008025200061458000808F5000FC
:10ADD0000100340060458800802520007145800016
:10ADE000808F5000010034007045880008407800D2
:10ADF0008000EB00E04F5400050032000194210078
:10AE0000914078008180FB008100E900CF08DE00DE
:10AE100040F9B700E08F50000300320040002000EE
:10AE200056DE02000000000010C0B300E00F540026
:10AE3000030032000040EB008000EB00050037000B
:10AE4000F1932100914078008180FB008100E900AE
:10AE5000CF08DE003FF9B700E08F5000030032005A
:10AE60000080EB0052DE0200000000004F04BE0034
:10AE7000000006000400FA00881F7800004020004F
:10AE8000C16680000080600044003200F1BF2F00E6
:10AE900080CD20001088600097FF20009743780045
:10AEA000E0CF53000C003A0007007800FAEFB7003B
:10AEB00010C0B300F9EFB70007437800874278006D
:10AEC0000742780087417800074178008740780082
:10AED0007F40400015003700FACFBF00E1CF53009C
:10AEE00015003A00E24F50002C003400FD4F500096
:10AEF0002A003C0021C0B3008000FD00F9EFB7003C
:10AF00008000FD000040E800F6EFB700FFC34300FB
:10AF10000043EB00864278000642780086417800C4
:10AF2000064178008740780007407800B2BF0200F1
:10AF30000000000019003700E2CF530017003A006C
:10AF400061FF20009140780080CF500013003D0049
:10AF500071C2B300814F500010003C0030C0B300FC
:10AF6000F9EFB700FEC34300074378008042EB00CF
:10AF700005427800854178000741780087407800D5
:10AF800007407800B2BF02000000000070002000FF
:10AF900052DE020000000000F86FEF00FACFBF00A1
:10AFA00031C6B300814F500002003C000040E80071
:10AFB000FAEFB70020C3B300A1FF20009140780052
:10AFC00080CF50000B003400F96FEF008043EB009E
:10AFD000074378008742780007427800874178006D
:10AFE000074178008740780007407800B2BF020030
:10AFF00000000000FACFBF00E54F500015003A00F6
:10B00000F7CFBF00E14F500009003A00F9CFBF0071
:10B01000E14F50000F003A0020C0B300F7EFB70037
:10B02000000520006045880000FB2F000800370065
:10B03000E24F500007003A00F9CFBF00E14F500047
:10B0400004003A00F7EFB7000005200060458800D3
:10B0500070458800FACFBF00FE4F500012003A0042
:10B06000F9CFBF0071FF200091407800E0CF500081
:10B0700008003A00E24F500006003A0010C0B3004A
:10B08000F7EFB70000052000604588007045880094
:10B0900005003700E24F500003003A00F76FEF0061
:10B0A000AC28EF00AE28EF0080C2B300A1FF200063
:10B0B0009140780080CF500009003A00F9CFBF00DE
:10B0C000E34F500006003A0010C0B300F7EFB7009E
:10B0D0000105200061458800AE28EF00F8EFB700B9
:10B0E0001008200041458000808F5000030034008C
:10B0F00051458000808F50000B003C00AC28EF00D1
:10B10000AE28EF000041EB008240780000C2B3009F
:10B110001EC00200000000000041EB0082407800E9
:10B1200000C2B300080037000041EB008240780005
:10B13000024078001EC00200000000000041EB0049
:10B1400082407800024078003AC00200000000000F
:10B1500088FF200018447800E04F5400220032009D
:10B1600066805700A7FA07004FF99700BFF89700CD
:10B170002FF8970002C00200000000003FF997007E
:10B18000AFF897004FF897003AC0020000000000A7
:10B190002FF99700CFF897003FF897001EC00200E4
:10B1A00000000000F84FEC00F8EFB700F1C7B30063
:10B1B000814F500012003A00F86FEF000041EB00A1
:10B1C00082407800024078003AC00200000000008F
:10B1D0000041EB0082407800024078001EC002006F
:10B1E0000000000006003700D6FB07000041780091
:10B1F000884078000140780002C002000000000092
:10B200004F0478000080FA0000000600CDFB070024
:10B2100000417800804078000040EB0002C002004E
:10B2200000000000DCD7BF000A003200DFD7BF00FB
:10B230000800320040458000AA08B4002200200027
:10B24000110009000200D8006009B000C0CB8800DE
:10B2500010C0B300D17D210091407800E0CF5000B4
:10B2600012003200017E210091407800E0CF5000B2
:10B270000E00320040458000AA08B40022002000E1
:10B28000110009000200D800D0CB8800510920002D
:10B29000810F500002003E00800C2000D0CB8800BF
:10B2A000A0F62F007A39B40002003700E04F5000BA
:10B2B0000D0032008043EB0007437800874278009E
:10B2C000074278008741780007417800874078007E
:10B2D00007407800B2BF020000000000AC28EF0079
:10B2E000AE28EF000000060043458000C2CB80007E
:10B2F000828F510001003100FCEFB700D1CB8000FC
:10B30000818F51000200360010C0B300FCEFB7007F
:10B3100050458000820F500001003100FD6FEF00AA
:10B32000810F50000200360010C0B300FDEFB700DF
:10B33000FCCFBF00D1FF20009140780006003A000A
:10B34000E0CF500008003A008000FD00FBEFB7009E
:10B350008000FD0015003700E14F500002003A0068
:10B36000E0CF500010003200E1CF500004003A005E
:10B37000E04F500002003A00FBEFEF000B003700F7
:10B38000FBCFBF004240A9000200340020C0B30040
:10B3900005003700E04F500002003200E0CFB3005C
:10B3A00001003700A0C0B300FBEFB700B7FF2000DB
:10B3B00097437800E0CF53000B003A00C012200002
:10B3C0006045880070458800074378008742780010
:10B3D00004C2B300874178000741780087407800B5
:10B3E0000440780036003700E1CF53000B003A00EC
:10B3F000C012200060458800AE28EF008043EB00BB
:10B4000007437800874278000742780003C2B30000
:10B41000074178008340780028003700E1CF4300DF
:10B420000A003A00AC28EF00C012200070458800E6
:10B4300007C2B3000043EB00874278000642780061
:10B4400086417800064178001B003700E2CF4300B8
:10B450000D003A0040ED2F0060458800C01220002A
:10B46000704588008043EB0006C2B3008742780035
:10B4700007427800874178000741780087407800CC
:10B48000074078000E003700E2CF53000E003A006C
:10B49000C01220006045880040ED2F0070458800F4
:10B4A0008043EB000743780087427800074278002A
:10B4B0008741780002C2B3008640780006407800D9
:10B4C000B2BF040000000000EACF530004003A00BD
:10B4D000C01220006045880040ED2F0070458800B4
:10B4E0000000060017FB0700004178008040EB00D9
:10B4F00002C0020000000000DDD7BF000080FB009A
:10B500000000EA004F00DE008000EB00E04F50003A
:10B510000500320071942100914078008180FB0089
:10B520008100E900CF08DE0047F9B700E08F500046
:10B5300002003200A0F62F00607F8800E0D7BF0035
:10B540000080FB000000EA004F00DE008000EB00FE
:10B55000E04F5000050032006194210091407800D6
:10B560008180FB008100E900CF08DE0046F9B700CA
:10B57000E08F50000200320060092000607F8800E8
:10B58000DCD7BF000080FB000000EA004F00DE00B7
:10B590008000EB00E04F5000050032005194210084
:10B5A000914078008180FB008100E900CF08DE0037
:10B5B00045F9B700E08F500007003200607F80003F
:10B5C000E00F500002003200EC2FEF0002003700C5
:10B5D000A0F62F00EA2FB400DFD7BF000080FB00E9
:10B5E0000000EA004F00DE008000EB00E04F50005A
:10B5F0000500320041942100914078008180FB00D9
:10B600008100E900CF08DE0044F9B700E08F500068
:10B6100007003200607F8000E00F5000020032001F
:10B62000EC2FEF000200370060092000EA2FB40081
:10B630000000EB00C17D210091407800E0CF500078
:10B6400004003200DFD7BF000080FB000000EA00EA
:10B650004F00DE008000EB00E04F5000050032009C
:10B6600031942100914078008180FB008100E90045
:10B67000CF08DE0043F9B700E08F50000100320030
:10B68000EA2FEF000000EB00017E210091407800DE
:10B69000E0CF500004003200DDD7BF000080FB0087
:10B6A0000000EA004F00DE008000EB00E04F500099
:10B6B0000500320021942100914078008180FB0038
:10B6C0008100E900CF08DE0042F9B700E08F5000AA
:10B6D00001003200EC2FEF0050468000E00F5000D8
:10B6E0004800320001022000810F5000300032007B
:10B6F00014003C00E60F50003C00320006003C0005
:10B70000E40F50002F0032003B003C00E20F5000DD
:10B710003B003A0026003700ED0F500036003200A3
:10B7200003003C00E80F500035003A0027003700C6
:10B73000F00F50002D003200F10F500030003A00A1
:10B740002000370001052000810F50001800320052
:10B7500008003C00E3805000810F500019003200C7
:10B760008100E800810F500020003200110220000B
:10B770000500370051052000810F500011003200F4
:10B7800004003C00E4805000810F50001C003A008F
:10B790000E00370061052000810F500013003200B9
:10B7A0008100E800810F500015003A0012003700B8
:10B7B000607F8000E00F500007003A006009200021
:10B7C00008003700A0F62F0009003700607F8000D6
:10B7D000E00F500002003200EC2FEF0008003700AD
:10B7E000A0F62F00EA2FB400050037006009200002
:10B7F000607F880002003700EC2FEF00EA2FEF0097
:10B80000CA28EF0080252000517F8000808F5000E3
:10B8100001003400507F880080DA2F00517F8000C3
:10B82000808F500001003D00507F8800802520005F
:10B83000617F8000808F500001003400607F8800AD
:10B8400080DA2F00617F8000808F500001003D0072
:10B85000607F8800517F8000607F80000101400090
:10B860006245880000805000704588000000060096
:10B8700000102000F46302000000000000202000FF
:10B88000F46302000000000000012000F4630200E5
:10B890000000000040002000F463020000000000EF
:10B8A00010002000F46302000000000000012000EE
:10B8B000F463040000000000EE4FEC00EEEFB70070
:10B8C00041C6B300814F50002200360050C6B3007D
:10B8D000EEEFB700DED7BF000080FB000000EA00FB
:10B8E0004F00DE008000EB00E04F5000050032000A
:10B8F00081932100914078008180FB008100E90064
:10B90000CF08DE0038F9B700E08F50001100320098
:10B91000207F80007AF90700407F8000E00F500010
:10B9200002003A000040210015003700217F80000E
:10B93000810F500004003A000000EB0028F90700D6
:10B94000E42FEF000300370025F90700E80FF800A7
:10B95000E40FF900C6ED020000000000E00F500007
:10B9600004003A0042BC02000000000070006000C9
:10B9700006003200207F800061F9070000402000AF
:10B980000C64020000000000B9FF3700207F800037
:10B9900001002000E70F5000E08F58005D003E00DE
:10B9A00000600100070037005400370054003700E2
:10B9B000540037005700370053003700530037005A
:10B9C00053003700DCD7BF000080FB000000EA0016
:10B9D0004F00DE008000EB00E04F50000500320019
:10B9E00071932100914078008180FB008100E90083
:10B9F000CF08DE0037F9B700E08F500004003200B6
:10BA00008080EB00407F8000B3F80700407F880013
:10BA1000DDD7BF000080FB000000EA004F00DE0021
:10BA20008000EB00E04F50000500320061932100E0
:10BA3000914078008180FB008100E900CF08DE00A2
:10BA400036F9B700E08F5000040032008080EB0030
:10BA5000407F8000A0F80700407F8800DFD7BF004C
:10BA60000080FB000000EA004F00DE008000EB00D9
:10BA7000E04F5000050032005193210091407800C2
:10BA80008180FB008100E900CF08DE0035F9B700B6
:10BA9000E08F50000400320011002000407F800041
:10BAA0008DF80700407F8800E0D7BF000080FB00D2
:10BAB0000000EA004F00DE008000EB00E04F500085
:10BAC0000500320041932100914078008180FB0005
:10BAD0008100E900CF08DE0034F9B700E08F5000A4
:10BAE0000400320011002000407F80007AF8070037
:10BAF000407F8800407F800089F83700A7F9370031
:10BB0000E1FA3700BBFB3700DAFC3700BFFD370036
:10BB100074FE070000000600307F88000000EB0084
:10BB2000AFF80700307F8000E00F500002003200C5
:10BB3000E82FEF000300370010002000407F88004E
:10BB400077F80700B0462000F4630400000000000E
:10BB50000040200004640200000000008000780023
:10BB60000080EB00E08F500001003200207F800059
:10BB700000000600E1C58000E08F50001300320095
:10BB8000C2D8EC00C2F8B700FF4F500004003400E8
:10BB9000E3806000E1C5880000CEB300C2F8B700C2
:10BBA000E0C58000E00F500008003200218C210029
:10BBB000914078008100FB0001003B008100EA0019
:10BBC000E0C0B300BEBE02000000000010C0B30021
:10BBD000E1C58000E08F5000030032000040EB0020
:10BBE0008000EB0005003700E189210091407800DA
:10BBF0008180FB008100E900CF08DE009EF8B700DD
:10BC0000E08F5000040032008040EB00E0C0B30041
:10BC1000BEBE02000000000000000600889FBE00BB
:10BC20000000EB0002C2B300C17D2100E1417800B9
:10BC3000618C2100E0CF510007003200E141780023
:10BC4000E3C141008370780082CF510003003600C9
:10BC50008270780001003700837078000000E800EF
:10BC6000E40F5000F0FF3400C8D8BF000B003200D2
:10BC70000802200039022000818C210091407800C8
:10BC800008407800BEBE0200000000000804E80082
:10BC9000890F5400F8FF34001C003700618C21002C
:10BCA00091407800E0CF50000300320010C2B30092
:10BCB000BEBE020000000000718C2100914078009F
:10BCC000E0CF50000300320020C2B300BEBE02002D
:10BCD00000000000918C210091407800E0CF5000DE
:10BCE0000300320000C2B300BEBE0200000000002C
:10BCF000A18C210091407800E0CF50000300320079
:10BD000030C2B300BEBE0200000000000000EB0025
:10BD1000618C210091407800E0CF500004003A008F
:10BD2000C8D8BF000080FB000000E9004F00DE0023
:10BD30008000EB00E04F500005003200618A2100D6
:10BD4000914078008180FB008100E900CF08DE008F
:10BD5000A6F8B700E08F5000040032008040EB00EE
:10BD600010C2B300BEBE0200000000000000EB00E5
:10BD7000718C210091407800E0CF500004003A001F
:10BD8000C8D8BF000080FB000000E9004F00DE00C3
:10BD90008000EB00E04F500005003200518A210086
:10BDA000914078008180FB008100E900CF08DE002F
:10BDB000A5F8B700E08F5000040032008040EB008F
:10BDC00020C2B300BEBE0200000000000000EB0075
:10BDD000918C210091407800E0CF500004003A009F
:10BDE000C8D8BF000080FB000000E9004F00DE0063
:10BDF0008000EB00E04F500005003200418A210036
:10BE0000914078008180FB008100E900CF08DE00CE
:10BE1000A4F8B700E08F5000040032008040EB002F
:10BE200000C2B300BEBE0200000000000000EB0034
:10BE3000A18C210091407800E0CF500004003A002E
:10BE4000C8D8BF000080FB000000E9004F00DE0002
:10BE50008000EB00E04F500005003200318A2100E5
:10BE6000914078008180FB008100E900CF08DE006E
:10BE7000A3F8B700E08F5000040032008040EB00D0
:10BE800030C2B300BEBE0200000000004F04BE007E
:10BE9000000006005AD9BF000080FB000000E90046
:10BEA0004F00DE008000EB00E04F50000500320044
:10BEB000C18A2100914078008180FB008100E90067
:10BEC000CF08DE00ACF8B700E08F5000040032006D
:10BED0008040EB00D0C1B300BEBE020000000000F5
:10BEE0005AD9BF00050032005A79EF0001C2B300F1
:10BEF000D0C1B300BEBE020000000000000006007A
:10BF0000881F7800CE58EC00CEF8B700EA4F5000FA
:10BF100023003A00CE78EF0031468000500920001F
:10BF2000808F500006003C008040EB0060C2B300F0
:10BF3000BEBE02000000000001C2B30015003700C1
:10BF400080112000808F50000600340001C2B30031
:10BF50006E404000BEBE0200000000008040EB00CA
:10BF60000C0037006109B100C508DD00220820007F
:10BF7000110009008200D800800078000144780098
:10BF800060C2B300BEBE02000000000001C2B300E8
:10BF900088C0500070C2B300BEBE020000000000A6
:10BFA0004F04780000000600889FBE00292480000E
:10BFB000E884640041003200488C21001844780075
:10BFC000E04F54000E003A008840780050C0B300A3
:10BFD000BEBE0200000000008840780060C0B300D0
:10BFE000BEBE0200000000008840780070C0B300B0
:10BFF000BEBE02000000000010C0B300C4F8B700CD
:10C00000C5D8BF0012002000010032000001FB0073
:10C0100071C0B300EA0F510007003C00230020006C
:10C02000801F7800110009000301D800800078000B
:10C030004F0078008140E80000C04000C5F8B7001C
:10C0400041C6B300814F500015003400C358EC00C6
:10C05000C3F8B70011C0B3008000FD00C5F8B700F9
:10C060008000FD00E34F500001003A00C378EF006C
:10C07000388C210018447800E04F540008003A0042
:10C080008840780070C0B300BEBE0200000000000F
:10C090008840780060C0B300BEBE0200000000000F
:10C0A000C3D8BF0065404000518C2100914078000A
:10C0B000BEBE020000000000B000370080458000D6
:10C0C000B208B400883E20000880B900A8F820001B
:10C0D000809FBE00110009004888D8000004780045
:10C0E0004F00BE00C4D8BF0027003200090078000E
:10C0F000C4F8B70050182000800F54000A00360022
:10C1000001C2B30050C0B300BEBE02000000000078
:10C1100001C2B30060C0B300BEBE02000000000058
:10C1200001C2B3001500370080162000800F5400B4
:10C130000600360001C2B30050C0B300BEBE02000C
:10C140000000000001C2B3000800370040152000C5
:10C15000800F54000C00360001C2B30050C0B30081
:10C16000BEBE0200000000008940780060C0B3003D
:10C17000BEBE0200000000008940780070C0B3001D
:10C18000BEBE02000000000010C0B3005118200025
:10C19000810F540003003E000040EB008000EB00E4
:10C1A00005003700218A2100914078008180FB0042
:10C1B0008100E900CF08DE00A2F8B700E08F500050
:10C1C0000C00320001C2B30050C0B300BEBE02007A
:10C1D0000000000001C2B30060C0B300BEBE020098
:10C1E0000000000001C2B30070C0B300BEBE020078
:10C1F0000000000071E92F008880400010C0B300EB
:10C20000F78F5000030036000040EB008000EB0089
:10C2100005003700118A2100914078008180FB00E1
:10C220008100E900CF08DE00A1F8B700E08F5000E0
:10C230000C00320001C2B30050C0B300BEBE020009
:10C240000000000001C2B30060C0B300BEBE020027
:10C25000000000008040EB0070C0B300BEBE0200D2
:10C2600000000000B1EA2F008880400010C0B30039
:10C27000EE8F5000030036000040EB008000EB0022
:10C2800005003700018A2100914078008180FB0081
:10C290008100E900CF08DE00A0F8B700E08F500071
:10C2A0000C00320001C2B30050C0B300BEBE020099
:10C2B000000000008040EB0060C0B300BEBE020082
:10C2C000000000008040EB0070C0B300BEBE020062
:10C2D0000000000010C0B30041152000810F540081
:10C2E000030036000040EB008000EB000500370043
:10C2F000F1892100914078008180FB008100E900F4
:10C30000CF08DE009FF8B700E08F50000800320031
:10C310008040EB0060C0B300BEBE02000000000021
:10C320008040EB0070C0B300BEBE02000000000001
:10C3300040152000800F540010003E00C558EC004E
:10C34000C5F8B700E34F500004003A0001C2B30043
:10C3500050C0B300BEBE020000000000C5D8BF0040
:10C36000E54F5000050034008040EB0050C0B300A2
:10C37000BEBE020000000000C578EF004F04BE0002
:10C3800000000600DCD7BF000080FB000000EA00D0
:10C390004F00DE008000EB00E04F5000050032004F
:10C3A000B18A2100914078008180FB008100E90082
:10C3B000CF08DE00ABF8B700E08F5000030032007A
:10C3C0002000200052DE020000000000DDD7BF0088
:10C3D0000080FB000000EA004F00DE008000EB0060
:10C3E000E04F500005003200A18A21009140780002
:10C3F0008180FB008100E900CF08DE00AAF8B700C9
:10C40000E08F5000030032002000200052DE0200C6
:10C4100000000000DED7BF000080FB000000EA0043
:10C420004F00DE008000EB00E04F500005003200BE
:10C43000918A2100914078008180FB008100E90011
:10C44000CF08DE00A9F8B700E08F500003003200EB
:10C450003000200052DE020000000000DFD7BF00E5
:10C460000080FB000000EA004F00DE008000EB00CF
:10C47000E04F500005003200818A21009140780091
:10C480008180FB008100E900CF08DE00A8F8B7003A
:10C49000E08F5000030032002000200052DE020036
:10C4A00000000000E0D7BF000080FB000000EA00B1
:10C4B0004F00DE008000EB00E04F5000050032002E
:10C4C000718A2100914078008180FB008100E900A1
:10C4D000CF08DE00A7F8B700E08F5000030032005D
:10C4E0002000200052DE02000000000000000600D4
:10C4F000889FBE008A9FBE008C1F78000000EB0062
:10C50000E3862100C2852100910320008080400045
:10C510008180400004802000E48078000002400018
:10C52000E3027A00818F520001003D0081317A00E0
:10C53000E08F50000500320000024000E2027A0065
:10C54000818F52000100340001317A000000E800C0
:10C55000E60F5000ECFF340040458000E1C380004E
:10C56000808F500001003D00E0C3880050458000EE
:10C57000F1C38000808F500001003D00F0C38800AF
:10C580000004EB000C0220006BEE290008014400BF
:10C59000C0852100E00079009003200008004000E1
:10C5A000000040000380200063007800E386210043
:10C5B00063057900010555000100500001003B00B2
:10C5C0000000EB000C80B900809FBE001100090044
:10C5D0004A08D800000578004F00BE00EB447C00FC
:10C5E0008A40780009407800BEBE020000000000CA
:10C5F000E20F540005003A008944E8008A407800C0
:10C6000009407800BEBE0200000000000804E800F7
:10C61000E60F5400DDFF3400E2C380004045800097
:10C62000E00F500001003D000000EB000802200078
:10C630000880B900811F7800110009004208D80065
:10C64000CF0078008040780060C1B300BEBE020019
:10C6500000000000F3C3800052458000080078000D
:10C66000E00F510001003D000001EB000090B90017
:10C67000811F7800110009004308D800CF0078001E
:10C680008040780070C1B300BEBE02000000000010
:10C690004F0678004F05BE004F04BE0000000600A4
:10C6A000889FBE0020468000F40F50003D003C00F3
:10C6B0001146800000468000467502000000000020
:10C6C00022002000110009000200D800037D200094
:10C6D00003014000F1F92000C8012000810F510042
:10C6E0001C0036000277210002024000B801200041
:10C6F000810F52001700360004712200040240002E
:10C70000A8012000810F520012003600046B2300A4
:10C710000402400098012000810F52000D003600F5
:10C7200088012000F5D52600850F520009003E0043
:10C73000830150006C044400818F510005003600D5
:10C7400002005000F8012000810F500001003E005F
:10C750006604440029468000E08F540001003D003B
:10C760008904EA00F48414008984440001003B0039
:10C770008004EB0060C68000E00F5000030035002D
:10C780008040EB00BEBE020000000000894078003F
:10C7900008407800BEBE02000000000068C68800A5
:10C7A0000700370060C68000E00F5000030035002E
:10C7B0008040EB00BEBE020000000000CCB8EF00DD
:10C7C0004F04BE000000060067006000C800DD00E6
:10C7D000F2058000F08F2F00000061000100700062
:10C7E000F00588000000060001C68000E08F5000C0
:10C7F00002003A008AC0A9009AC0A8000100700097
:10C8000000C6880000000600C018B6000000060040
:10C810008AC0A800000006000080EA00C018B60028
:10C8200000C6880001003A009AC0A9000000060076
:10C830001000FA00889FBE008A9FBE00D4D8BF00B7
:10C84000E14F500055023A00C6ED02000000000022
:10C85000E00F500004003A0042BC0200000000005B
:10C86000F00060002500320000002100EAFF070010
:10C870000001EB006000B800A6C00200000000004C
:10C880008043EB0007437800874278000742780036
:10C89000874178000741780087407800074078009A
:10C8A000B2BF0200000000008043EB0007437800A5
:10C8B0008742780007427800874178000741780076
:10C8C000874078000740780056C002000000000052
:10C8D000AC28EF00AE28EF0042BC020000000000D0
:10C8E0000002B2000200320082BD0200000000001F
:10C8F000385C02000000000041023700238D210057
:10C9000093417800E1CF510008003200E2CF51009E
:10C9100009003200E0CF51000B003A00010178001D
:10C92000F10020000002200005003700010178001E
:10C93000010220000100370002022000F000200068
:10C94000A6C0020000000000D3D8BF00E14F4000A5
:10C950001F003A00CF58EC00CFF8B700FC4F500052
:10C960000A003A0007C2B300074378008742780004
:10C9700007427800874178000741780087407800B7
:10C980000740780056C002000000000080C3B300DA
:10C99000F18C21009140780080CF50003B003600A0
:10C9A000CF78EF008043EB000743780087427800A0
:10C9B0000742780087417800074178008740780077
:10C9C0000740780056C00200000000002F0037002A
:10C9D000A250020000000000A2500200000000006F
:10C9E000A250020000000000000478008843780094
:10C9F000084378008842780008427800884178002F
:10CA000008417800884078000840780056C002004D
:10CA100000000000238D210093417800E1CF5100F8
:10CA20000A003200E2CF51000E003200E0CF510088
:10CA300011003A00C545DD00C55DDE006F44B90058
:10CA40004545DE00834478000B0037006F40B90095
:10CA5000C505DE004544DD004545DE008044EB00B1
:10CA6000050037006F40B900C505DE004544DD0014
:10CA7000C544DE000045EB000981FB008A80FB0015
:10CA80000B80FB00A6C0020000000000D3D8BF004E
:10CA90000000FB00CF80DE0061004000E080480025
:10CAA000E30F5000E08F5800B9013E000060010024
:10CAB000030037006B003700D100370093013700C7
:10CAC000DCD7BF000080FB000000EA004F00DE0062
:10CAD0008000EB00E04F500005003200A18B2100E8
:10CAE000914078008180FB008100E900CF08DE00E2
:10CAF000BAF8B700E08F500001003200D278ED00A4
:10CB0000DFD7BF000080FB000000EA004F00DE001E
:10CB10008000EB00E04F500005003200918B2100B7
:10CB2000914078008180FB008100E900CF08DE00A1
:10CB3000B9F8B700E08F500001003200D278EC0065
:10CB4000DDD7BF000080FB000000EA004F00DE00E0
:10CB50008000EB00E04F500005003200818B210087
:10CB6000914078008180FB008100E900CF08DE0061
:10CB7000B8F8B700E08F500001003200D278EC0026
:10CB8000E0D7BF000080FB000000EA004F00DE009D
:10CB90008000EB00E04F500005003200718B210057
:10CBA000914078008180FB008100E900CF08DE0021
:10CBB000B7F8B700E08F500001003200D278ED00E6
:10CBC000D2D8BF0009003B0042BC020000000000B8
:10CBD000610060000200320020C0B3000100370095
:10CBE00010C0B300D2F8B7000A003700E14F500080
:10CBF0000400340042BC020000000000610060003C
:10CC0000F8FF3200D2D8BF00E24F500001003400DC
:10CC1000D278EF00DED7BF000080FB000000EA0002
:10CC20004F00DE008000EB00E04F500005003200B6
:10CC3000618B2100914078008180FB008100E90038
:10CC4000CF08DE00B6F8B700E08F50005001320088
:10CC5000D2D8BF00D3F8B70010C0B300D5F8B700E2
:10CC60004B013700DCD7BF000080FB000000EA006A
:10CC70004F00DE008000EB00E04F50000500320066
:10CC8000518B2100914078008180FB008100E900F8
:10CC9000CF08DE00B5F8B700E08F50000300320087
:10CCA000D178EC00ACB6020000000000DFD7BF0076
:10CCB0000080FB000000EA004F00DE008000EB0077
:10CCC000E04F500005003200418B21009140780078
:10CCD0008180FB008100E900CF08DE00B4F8B700D6
:10CCE000E08F500003003200D178ED00ACB60200B6
:10CCF00000000000D1D8BF0002003B00D178EF0057
:10CD000004003700E84F50000200340080C0B30038
:10CD1000D1F8B700118D2100914078008100FB000F
:10CD2000F1AA88000040EB00618210008080FB00C7
:10CD300081014200C219DD0081804000F882570065
:10CD40000181420003097800E08F510001003D009D
:10CD50000009EB000040E800E74F5000F3FF360009
:10CD60008FEB97002FEB9700CFEA97006FEA9700C1
:10CD70008FF197002FF19700CFF097006FF0970099
:10CD8000B2BF0200000000000000EB00E17D2100C6
:10CD900091407800E0CF500004003200D5D8BF00A9
:10CDA0000080FB000000E9004F00DE008000EB0087
:10CDB000E04F500005003200318B21009140780097
:10CDC0008180FB008100E900CF08DE00B3F8B700E6
:10CDD000E08F5000EE003200D3F8EF008043EB000C
:10CDE000074378008742780007427800874178003F
:10CDF000074178008740780007407800BD00370081
:10CE000060458000E00F500067003200E0D7BF00AF
:10CE10000080FB000000EA004F00DE008000EB0015
:10CE2000E04F500005003200218B21009140780036
:10CE30008180FB008100E900CF08DE00B2F8B70076
:10CE4000E08F500003003200D078EC00ACB6020056
:10CE500000000000DDD7BF000080FB000000EA00FA
:10CE60004F00DE008000EB00E04F50000500320074
:10CE7000118B2100914078008180FB008100E90046
:10CE8000CF08DE00B1F8B700E08F50000300320099
:10CE9000D078ED00ACB6020000000000018D21004A
:10CEA00091407800E0CF500019003500FFCF5000CE
:10CEB000100034007FC150008043EB00074378002E
:10CEC000874278000742780087417800F1C1B300BB
:10CED00007407800B2BF02000000000020C3B3008A
:10CEE000018D21009140780080CF50002600340051
:10CEF000190037008043EB00074378008742780031
:10CF00000742780087417800074178001B0037000E
:10CF1000FFCF400012003D00F7C1B30016CEB300B2
:10CF2000014353008042EB000542780085417800C0
:10CF3000054178008540780005407800B2BF0200C6
:10CF400000000000E0CCB300018D2100914078008A
:10CF500080CF50000C003D00D0F8B7000A00370029
:10CF60008143EA000043EB008642780006427800E5
:10CF700086417800064178008640780006407800B7
:10CF8000B2BF020000000000D0D8BF000000FB00CC
:10CF9000011020008080400071AB8800011020004B
:10CFA0000080500080AB8800DCD7BF000080FB0011
:10CFB0000000EA004F00DE008000EB00E04F500070
:10CFC00005003200018B2100914078008180FB0038
:10CFD0008100E900CF08DE00B0F8B700E08F500014
:10CFE0000B003200614580000108B10061458800F6
:10CFF00000F82F00AE28B40010E82F00808F5000FA
:10D0000003003D000000E90060458800704588008D
:10D01000DFD7BF000080FB000000EA004F00DE0009
:10D020008000EB00E04F500005003200F18A210043
:10D03000914078008180FB008100E900CF08DE008C
:10D04000AFF8B700E08F50000B0032006145800060
:10D050000108B0006145880000082000AE28B40037
:10D06000F0172000808F5000030034000000E8001B
:10D0700060458800704588000000EB00E17D2100DC
:10D0800091407800E0CF500004003200D5D8BF00B6
:10D090000080FB000000E9004F00DE008000EB0094
:10D0A000E04F500005003200E18A210091407800F5
:10D0B0008180FB008100E900CF08DE00AEF8B700F8
:10D0C000E08F50003200320060458000E00F5000D9
:10D0D0000B003A00D3F8EF0080437800004378005B
:10D0E000804278000042780080417800004178005A
:10D0F00080407800B2BF020000000000240037002A
:10D10000AC28EF00AE28EF002100370042BC02003F
:10D11000000000000002B20002003A007ABD0200E6
:10D12000000000000000EB00E17D2100914078004C
:10D13000E0CF500004003200D5D8BF000080FB00D3
:10D140000000E9004F00DE008000EB00E04F5000DF
:10D1500005003200D18A2100914078008180FB00D7
:10D160008100E900CF08DE00ADF8B700E08F500085
:10D170000700320042BC0200000000000002B200C2
:10D180000200320082BD020000000000D3F8EF0070
:10D19000DED7BF001A003A0016003700DDD7BF0007
:10D1A00016003200E0D7BF0014003200D558EC0062
:10D1B000D5F8B70041C6B300814F500010003600CB
:10D1C0008140E800814F500009003A0010C0B300D0
:10D1D000D4F8B700004020008FFD0700D3F8EF001F
:10D1E0005ED5BF00D1F8B7006ED5BF00D0F8B7004C
:10D1F00060C6B300D5F8B70001003700D578EF005E
:10D200004F05BE004F04BE000080FA00000006007B
:10D210003600F800809FBE00829FBE00849FBE0043
:10D22000869FBE003400F80000002000A0018800A6
:10D230008AC0A900C078AB00010032004DFA070097
:10D24000C0B8AB000100320057FB0700C038AB008C
:10D250000100320071FA0700C018AB000100320073
:10D2600048FC0700C058AB0001003200A0FC0700DA
:10D27000C0D8AB000100320006FB0700C118AB00AC
:10D280000100320006FD0700C138AB00010032008A
:10D290001BFB07000040200001C6800000806000EA
:10D2A000020032005C5C02000000000000802000F0
:10D2B00001C680000080600002003200D49E02009F
:10D2C000000000000000210001C680000080600016
:10D2D0000100320056FD07003400F9004F03BE0084
:10D2E0004F02BE004F01BE004F00BE003600F900E5
:10D2F00000400600E28B210012417800C098AB008C
:10D300001800320071468000E08F50000B003200A0
:10D310000080FB00810F5000030034004300DE005A
:10D32000804F510003003900E04F510006003200E9
:10D330000240E900BEF8B700030037008000FD009E
:10D34000BEF8B7008000FD00E18B2100914078001D
:10D35000814F510003003200E0C1B300BEBE0200A5
:10D360000000000000000600C18B2100E00F50000B
:10D3700003003D0067006000910870000000060097
:10D380000080EA0091086000000006000200FA0038
:10D39000F0BF9F0001017800CF80DE00E40F500055
:10D3A000E08F580010003E000060010004003700CC
:10D3B0000500370006003700070037000800370077
:10D3C000120888000E003700620888000C00370041
:10D3D000720888000A003700D20888000800370069
:10D3E000E2088800060037008F81E9004210200023
:10D3F000014D200000E02900F61F0200000000009F
:10D400000080FA00000006000200FA00F0BF9F0052
:10D41000EA0F500019003E00120020000010DD004D
:10D4200082412000020160000D003A0000017800F6
:10D430006220B20003003A006100600015003A006B
:10D440000E003700E1806000C308DD008008800026
:10D450000030A10001007000800888000D00370036
:10D46000E1806000C308DD00F00880000030A1000A
:10D4700001007000F0088800060037008F81E90085
:10D4800042102000A146200000E02900F61F020003
:10D49000000000000080FA00000006000200FA0010
:10D4A000F0BF9F0001017800CF80DE00EA0F50003E
:10D4B000E08F580034003E00006001000A00370091
:10D4C00011003700180037001F0037002600370012
:10D4D0002D0037002C0037002B0037002A003700C2
:10D4E0000900370018003700630161004410DD00B7
:10D4F00022088000F1FC2F00010161000001710091
:10D500002208880026003700630161004410DD0016
:10D5100082088000F1FC2F00010161000001710010
:10D52000820888001E003700630161004410DD009E
:10D5300092088000F1FC2F000101610000017100E0
:10D540009208880016003700630161004410DD0076
:10D55000F2088000F1FC2F00010161000001710060
:10D56000F20888000E003700630161004410DD00FE
:10D5700002098000F1FC2F0001016100000171002F
:10D5800002098800060037008F81E9004210200060
:10D59000214A200000E02900F61F020000000000E0
:10D5A0000080FA00000006000200FA00F0BF9F00B1
:10D5B000401ADE0005002000E90F50000300320091
:10D5C000EA0F500007003A000300370062088800A5
:10D5D0007408880009003700D2088800E408880031
:10D5E000060037008F81E90042102000A14F200083
:10D5F00000E02900F61F0200000000000080FA0091
:10D6000000000600E80F5000020034000000D000C7
:10D61000710050000000060080007800100020001B
:10D62000E88F500001003C000000EB000000060005
:10D630000200FA00889FBE008A1F7800C0BF9F00CA
:10D6400000047800EC0F540006003600E881570013
:10D6500042102000E115200000E02900F61F020022
:10D660000000000008007800E6FF070000057800D1
:10D67000A98321004250DD00008044009000780022
:10D680000110A1000100A000010878000800780046
:10D69000E1FF0700E00F5000040032000A00E8003C
:10D6A0004200DD00008044001000A0004F0578001B
:10D6B0004F04BE000080FA0000000600D1FF070002
:10D6C0004200DD000080E8008183210061007800D5
:10D6D00061006000000006000200FA00889FBE00A2
:10D6E000D0BF9F000104780080047800EC8F5400C4
:10D6F00004003600E681570042102000E1192000A6
:10D700000C00370009007800BEFF07004200DD0072
:10D710000080E80081832100610078000000D100D2
:10D720006140600006003A00E68157003210200098
:10D73000211A200000E02900F61F0200000000006E
:10D740006148B900EA0F5000E08F58002A003E00FF
:10D75000006001000A0037000F0037001400370096
:10D76000190037001E003700230037002200370061
:10D770002100370020003700070037001200370073
:10D780004F44DD002008800000F0A1000800700078
:10D79000200888001C0037004F44DD00800880000E
:10D7A00000F0A10008007000800888001600370013
:10D7B0004F44DD009008800000F0A10008007000D8
:10D7C00090088800100037004F44DD00F00880000A
:10D7D00000F0A10008007000F00888000A0037007F
:10D7E0004F44DD000009800000F0A1000800700037
:10D7F0000009880004003700E6815700421020002D
:10D80000511C2000CBFF37004F04BE000080FA00FF
:10D81000000006008000EB00AFFF37001100200081
:10D82000ADFF37000200FA00F0BF9F00CF80DE009E
:10D83000EA0F5000E08F580018003E000060010021
:10D840000A0037000C0037000D0037000F003700CA
:10D850001000370011003700100037000F003700AC
:10D860000E00370003003700070037000208880069
:10D870001000370043088800320888000D00370088
:10D88000520888000B003700B3088800A2088800FF
:10D8900008003700C2088800060037008F81E900C1
:10D8A00042102000D11E200000E02900F61F0200D7
:10D8B000000000000080FA00000006002F04B00005
:10D8C000889FBE008A9FBE008C9FBE008E1F78007E
:10D8D000D0A79F00E2A79F00F3A79F0081AF9F0002
:10D8E0006000B8006011B800909F9F00A19F9F004A
:10D8F000B29F9F00C39F9F000E0078000F07780023
:10D900006E04B100C1E1290007000900311F780051
:10D91000000778005FA69700EC0F56000500360060
:10D92000A3FC2F008F814100421020002110200015
:10D930000E0037000C00780032FF070080007800EE
:10D94000C208DD008180E80082832100E280780047
:10D950008100D100E1C0600007003A00A3FC2F0065
:10D960008F814100321020006110200000E029006A
:10D97000F61F0200000000008FA89700E08F500003
:10D9800013003200E38F500011003200E68F500088
:10D990000F003200E98F50000D003200E18F40008F
:10D9A00025003200E28F400023003200E38F400068
:10D9B00021003200E48F40001F00320003FD2F00E1
:10D9C0008F81410052102000B1102000E7FF370086
:10D9D0006FA19700FFA19700929F9F00A39F9F00B8
:10D9E0000001EB00B29F9F00C29F9F00820678005B
:10D9F000698710000E003700A400200005002000F9
:10DA00006033B8001F989700AF9897003F99970030
:10DA1000CF9997006004020000000000909F9F00D3
:10DA2000A19F9F00B29F9F00C39F9F008D06E800AB
:10DA30008E8F5600F0FF3500E80F5600A1003C0025
:10DA40008040EB000C0078006FFE07000FA99700E4
:10DA5000E00F5100880035001F9C9700AF9C970095
:10DA60003F9D9700CF9D970088EF020000000000C7
:10DA700090B79F00A1B79F008003EB00B7B79F004E
:10DA80000000EB00C0B79F001FB29700AFB2970035
:10DA90003FB39700CFB397000440E10005C8E10011
:10DAA00006D0E10007D8E1001F0039001F98970059
:10DAB000AF9897003F999700CF999700D0AF9F00FC
:10DAC000E1AF9F00F2AF9F0083B79F0088EF020095
:10DAD000000000000004BE004FB597008A057800E2
:10DAE00004F02F00F50F20006033B8000800BE00DE
:10DAF0000A01BE0060040200000000005FAA970057
:10DB0000EFAA97007FAB97008FB397000020E1004A
:10DB100001A8E10002B0E10003B8E10002003E000C
:10DB20004FB697000600370023FB2F008F8141007E
:10DB300012102000D11120008CFF37000C06E800E5
:10DB40001F989700AF9897003F999700CF9997003B
:10DB500090B79F00A1B79F00B2B79F00C3B79F00C7
:10DB600088EF0200000000004261DD00A3FB2F00EF
:10DB70008F814100028141001202BE00D4B79F0094
:10DB8000E5B79F008002EB00F5B79F000003EB00B4
:10DB900086BF9F000004BE000A0020000B0020008A
:10DBA000F4FF2F00050020006033B8000800BE001D
:10DBB0000A01BE0060040200000000005FB297008E
:10DBC000EFB297007FB397008FBB9700600402000D
:10DBD000000000001FB29700AFB297003FB397005C
:10DBE000CFB397000020E10001A8E10002B0E100FE
:10DBF00003B8E100D1FF3E001F989700AF9897004F
:10DC00003F999700CF99970090B79F00A1B79F00C9
:10DC1000B2B79F00C3B79F0088EF0200000000006A
:10DC20000004BE000FBD97008A0578005FB2970020
:10DC3000EFB297007FB397008FBB97000800BE003C
:10DC40000A01BE0060040200000000000203BE00E2
:10DC50000002BE001FB09700AFB097003FB1970021
:10DC6000CFB1970082050200000000000205BE004F
:10DC70000004BE000C0037006FA09700FFA09700C3
:10DC8000E10F4000E08F580005003600C3FC2F0074
:10DC90008F814100121020007112200033FF3700E5
:10DCA0000286EA000004BE008C0078005FA09700A6
:10DCB000FAFD0700880078005FA09700B3FD070019
:10DCC0008C00370011C0B3000C007800CEFD0700B7
:10DCD0008FA89700E08F50007D0035001F9C9700B3
:10DCE000AF9C97003F9D9700CF9D970088EF020063
:10DCF00000000000D0B79F00E1B79F008003EB0059
:10DD0000F7B79F000000EB0080BF9F005FB2970055
:10DD1000EFB297007FB397008FBB97000440E100FC
:10DD200005C8E10006D0E10007D8E1002000390075
:10DD30001F989700AF9897003F999700CF99970049
:10DD4000D0AF9F00E1AF9F00F2AF9F0083B79F006D
:10DD500088EF0200000000000004BE000FBD970025
:10DD60008A05780004F02F00F5FF2F00F60F200041
:10DD7000070020000800BE000A01BE006004020087
:10DD8000000000005FAA9700EFAA97007FAB970002
:10DD90008FB397000020E10001A8E10002B0E1008C
:10DDA00003B8E10002003E000FBF970006003700F5
:10DDB00023FB2F008F81410012102000A1132000AF
:10DDC000EAFE37000E07E8001F989700AF9897000B
:10DDD0003F999700CF999700D0B79F00E1B79F0078
:10DDE000F2B79F0083BF9F0088EF02000000000091
:10DDF0000001BE004270DD00A1FB2F008F804000BB
:10DE0000008040001006BE000C00BE00540402005A
:10DE1000000000000004BE000005EB008A05780049
:10DE20000802BE000A03BE005FB09700EFB0970083
:10DE30007FB197008FB997008205020000000000B3
:10DE4000F4FF2F00F5FF2F006033B8000400E1005D
:10DE50000588E1000690E1000798E100D9FF3E0047
:10DE60000800BE000A01BE0090B79F00A1B79F0046
:10DE7000B2B79F00C3B79F001F9C9700AF9C97004D
:10DE80003F9D9700CF9D970088EF020000000000A3
:10DE90000002BE004FB39700860378000800BE0062
:10DEA0000A01BE0082050200000000000C02BE0054
:10DEB0004FB49700080378008803780082050200B9
:10DEC000000000000205BE000004BE000300370091
:10DED0000187EA006FA49700FFA497008E007800E6
:10DEE0005FA097006DFD07000801BE005FA09700CE
:10DEF000ADFD07006011B8005FA0970049FE070064
:10DF00004F0778004F06BE004F05BE004F04BE000D
:10DF10002F04B100000006000200FA00F0BF9F00CD
:10DF2000CF80DE00EA0F5000E08F58001F003E0057
:10DF3000006001000A0037000B00370010003700B6
:10DF4000110037001700370018003700170037009E
:10DF50001600370015003700060037000C003700A8
:10DF60000008800001003700300880000100200018
:10DF70001400370032088000400880000600370097
:10DF800050088000F9FF3700A0088000F7FF370035
:10DF9000A2088000B00880008000780002007800AD
:10DFA00008003700C0088000F0FF37008F81E900CB
:10DFB000421020005121200000E02900F61F02003D
:10DFC000000000000080FA00000006000400FA00D3
:10DFD000E0BF9F00F1BF9F0001017800E10F5100F9
:10DFE000040036008F81E900621020009122200099
:10DFF0003E0037006FB89700CF80DE00EA0F500078
:10E00000E08F580036003E00006001000A00370033
:10E0100012003700190037002100370028003700B0
:10E020002F0037002E0037002D0037002C0037005E
:10E030000900370019003700610161000201410049
:10E04000200880000010A100020070002008880055
:10E0500005A1A9002800370013A1A90061016100F2
:10E0600002014100800880000010A1000200700041
:10E070008008880011A1A9001F003700610161001C
:10E0800002014100900880000010A1000200700011
:10E090009008880013A1A9001700370021A1A9004A
:10E0A0006101610002014100F00880000010A10040
:10E0B00002007000F00888001FA1A9000E003700C0
:10E0C0006101610002014100000980000010A1000F
:10E0D000020070000009880021A1A9000600370095
:10E0E000E4815700421020001126200000E02900A2
:10E0F000F61F0200000000000080FA000000060089
:10E100000200FA00F0BF9F0001017800CF80DE001E
:10E11000EA0F5000E08F58002F003E000060010021
:10E120000A00370010003700160037001C003700C7
:10E13000220037002800370027003700260037006C
:10E140002500370008003700150037006101610025
:10E150004611DD00200880000060A1000200700070
:10E160002008880022003700610161004611DD00AF
:10E17000800880000060A100020070008008880014
:10E180001B003700610161004611DD00900880002E
:10E190000060A100020070009008880014003700A1
:10E1A000610161004611DD00F00880000060A100FF
:10E1B00002007000F00888000D0037006101610066
:10E1C0004611DD00000980000060A100020070001F
:10E1D00000098800060037008F81E9004210200006
:10E1E0004129200000E02900F61F02000000000085
:10E1F0000080FA00000006000400FA00889FBE00BC
:10E200008A1F7800B0BF9F0001057800C2BF9F0041
:10E2100080047800EC8F540004003600EA81570037
:10E2200042102000812A2000070037004FBC9700D1
:10E230000800E900E60F500006003600E8815700AC
:10E2400022002000912A200000E02900F61F020091
:10E250000000000009007800EAFC07004200DD0031
:10E26000828321000A3178006148B900EA0F50002A
:10E27000E08F58003C003E00006001000A003700BB
:10E28000130037001C003700240037002D00370032
:10E2900035003700340037003300370032003700D4
:10E2A0001500370027003700670464004C40DD008C
:10E2B00028058000F1FF28000104640000047400B8
:10E2C000280588008460A9009460A8002A0037000F
:10E2D000670464004C40DD0038058000F1FF280031
:10E2E00001046400000474003805880084E0A9007B
:10E2F00094E0A80020003700670464004105800016
:10E3000080FF2F000080600008047000480588002E
:10E310008500A9009500A800170037006704640075
:10E320004C40DD0088058000F1FF280001046400F6
:10E3300000047400880588008760A9009760A80021
:10E340000D003700670464009105800080FF2F00F6
:10E350000080600008047000980588008780A9008C
:10E360009780A80004003700EA815700421020007F
:10E37000D12E2000B4FF37004F0578004F04BE00B7
:10E380000080FA00000006000200FA00F0BF9F00C3
:10E39000CF80DE00EA0F5000E08F58002A003E00D8
:10E3A000006001000A0037000F003700140037003A
:10E3B000190037001E003700230037002200370005
:10E3C00021003700200037000D003700180037000B
:10E3D000A00480004300DE00610060009460A8009B
:10E3E0008460A8001E003700A00480004700DE0003
:10E3F0006100600094E0A80084E0A80018003700E5
:10E40000A00480004800DE00610060009500A800C4
:10E410008500A80012003700B00480004B00DE0029
:10E42000610060009760A8008760A8000C003700BA
:10E43000B00480004C00DE00610060009780A800FE
:10E440008780A800060037008F81E9004210200075
:10E45000F133200000E02900F61F02000000000058
:10E460000080FA00000006000200FA00F0BF9F00E2
:10E47000CF80DE00EA0F5000E08F58001E003E0003
:10E48000006001000A0037000C0037000E00370062
:10E490001000370012003700170037001600370051
:10E4A0001500370014003700070037000C00370054
:10E4B000200480004300DE000B00370020048000B1
:10E4C0004700DE0008003700200480004800DE001E
:10E4D00005003700300480004B00DE0002003700EA
:10E4E000300480004C00DE00610060000080FA0013
:10E4F00000000600060037008F81E900421020006E
:10E500001137200000E02900F61F02000000000083
:10E510000200FA00F0BF9F0001017800CF80DE000A
:10E52000EA0F5000E08F580038003E000060010004
:10E530000A003700110037001A00370021003700A9
:10E540002800370031003700300037002F00370037
:10E550002E0037001300370022003700200480000F
:10E560004300DE0061006000610161004311DD00D5
:10E57000210480000130A100070037002004800042
:10E580004700DE0061006000610161004711DD00AD
:10E59000210480000170A1008280700021048800A5
:10E5A00020003700200480004800DE006100600089
:10E5B000610161004811DD00210480000180A1009B
:10E5C000F5FF3700300480004B00DE006100600082
:10E5D000610161004B11DD003104800001B0A10038
:10E5E00007003700300480004C00DE00610060004E
:10E5F000610161004C11DD003104800001C0A10007
:10E600008280700031048800060037008F81E900A5
:10E6100042102000613B200000E02900F61F0200AC
:10E62000000000000080FA00000006000200FA006E
:10E63000F0BF9F00CF80DE00EA0F5000E08F58004F
:10E640001B003E00006001000A0037000C0037008C
:10E650000E0037001000370012003700140037009A
:10E660001300370012003700110037000700370091
:10E670000C0037009460A9008460A90012003700E4
:10E6800094E0A90084E0A9000F0037009500A900DC
:10E690008500A9000C0037009760A9008760A900D9
:10E6A000090037009780A9008780A900060037007D
:10E6B0008F81E90042102000913F200000E02900F6
:10E6C000F61F0200000000000080FA0000000600B3
:10E6D0000600FA00889FBE008A9FBE008C9FBE0085
:10E6E000F0B79F008106780000057800EC0F550018
:10E6F00004003600F281570042102000210C200057
:10E70000100037000A00780082BF9F0093BF9F006F
:10E71000BCFB0700000678004264DD000880E800CA
:10E720008183210061027800614262000FB9970085
:10E730009FB9970006003A00F2815700221020008E
:10E74000610C200000E02900F61F0200000000001C
:10E75000AB83210008844500980478000910A000CC
:10E760000900A100090C78000A00780082BF9F0010
:10E7700093BF9F00A8FB07000FB997009FB99700B0
:10E78000E00F5000060032000C00E8004200DD00FF
:10E79000008045001000A1001820A00002003700F2
:10E7A0000920A100090C78007FB0970082BF9F006C
:10E7B00093BF9F009DFF07008D0078000FB9970061
:10E7C0009FB997007FB097003CFC07008000EB00EA
:10E7D0007FB09700FDFD07008000EB007FB0970041
:10E7E00047FE07004F06BE004F05BE004F04BE00A7
:10E7F0000080FA00000006000200FA00F0BF9F004F
:10E80000CF80DE00EA0F5000E08F58001B003E0072
:10E81000006001000A0037000B0037000C003700D1
:10E820000D0037000E0037001400370013003700CA
:10E8300012003700110037000300370006003700D0
:10E84000210880000700370081088000050037009C
:10E850009108800003003700F108800001003700B4
:10E8600001098000C408DE00E3806000000420008D
:10E87000E28F500007003A000D0037008F81E90059
:10E88000421020009142200000E02900F61F020003
:10E890000000000000102000E38F50000400320050
:10E8A00080002000E18F50000100320010002000A5
:10E8B0000080FA00000006003600F800809FBE00CD
:10E8C000829FBE00849FBE00869FBE003400F80079
:10E8D00000002000A00188000000EB00C1C1800002
:10E8E000010001008460A9003400F9004F03BE005C
:10E8F0004F02BE004F01BE004F00BE003600F900BF
:10E90000004006003600F800809FBE00829FBE00D7
:10E91000849FBE00869FBE003400F80000002000E7
:10E92000A001880084E0A90010002000E1C180005F
:10E93000010001003400F9004F03BE004F02BE0089
:10E940004F01BE004F00BE003600F9000040060037
:10E950003600F800809FBE00829FBE00849FBE00EC
:10E96000869FBE003400F80000002000A00188004F
:10E970008500A900F0C1800066006000E60F50002D
:10E9800003003A0090002000E1C18000020037003F
:10E990002000200001C28000010001003400F900C5
:10E9A0004F03BE004F02BE004F01BE004F00BE002D
:10E9B0003600F900004006003600F800809FBE00D7
:10E9C000829FBE00849FBE00869FBE003400F80078
:10E9D00000002000A00188008760A900300020000E
:10E9E00021C28000010001003400F9004F03BE0085
:10E9F0004F02BE004F01BE004F00BE003600F900BE
:10EA0000004006003600F800809FBE00829FBE00D6
:10EA1000849FBE00869FBE003400F80000002000E6
:10EA2000A00188008780A90030C2800066006000D5
:10EA3000E60F500003003A00A000200021C2800031
:10EA4000020037004000200041C2800001000100A8
:10EA50003400F9004F03BE004F02BE004F01BE005C
:10EA60004F00BE003600F9000040060090089000FC
:10EA7000E001900001814000630179008100E9001C
:10EA80001108980002007800000006000200FA0059
:10EA9000889FBE008004780001047800E08F540055
:10EAA00003003A0000002800000064005C0037000A
:10EAB00000002400E00F54005600320008027800E5
:10EAC00001003D000802EA0009007800E08F5400D0
:10EAD00001003D000900EA00CF80DE00668157009A
:10EAE000811F7800110009004488D80001097800CE
:10EAF000CF0078005FB9970003002000C011DD004F
:10EB000002002000809FBE00110009004499D80037
:10EB1000000178004F00BE008000780002007800FD
:10EB20000181CF00E00F51000300320004022000F9
:10EB300002025200040037000082CF00E00F5200B2
:10EB40000100320070021200EC02520009003B008A
:10EB5000C22820000300200054040200000000002E
:10EB6000440BDD004C00DE0000007300CC88DE00AA
:10EB70002400370012002000030020000403780066
:10EB80000603E900030033000201410083814900CC
:10EB9000FBFF3700020050008380580068025200DB
:10EBA0000402E900030033008180D1000080D3001B
:10EBB000FBFF3700FF0060004580DE00C32ADD0058
:10EBC000050140000200410046FA28006600780076
:10EBD00003022000018251000482B9000201E80012
:10EBE00002014100660079000180B9000000420086
:10EBF00081804A00811F7800110009004308D80075
:10EC0000CF007800E00F540002003D000100280012
:10EC100000805000E08F540001003C000000EA003A
:10EC20004F04BE000080FA0000000600889FBE006E
:10EC30008A9FBE008C1F780000017800E00F510011
:10EC40000C003D0001002C00810F510003003D002D
:10EC500000002800000041000400370010002800D8
:10EC6000810F51002C0032000200EA001A0020003F
:10EC70000B00370001002400810F51000300340015
:10EC8000000028000200500004003700F0FF2700B9
:10EC9000810F510020003200020078000005EB00D7
:10ECA000C780DE0000017800F207B20081814000D9
:10ECB00020EA2800E08579000C08200002065600B2
:10ECC0008100E8008180400060807800CF80DE0015
:10ECD000CF91DE0054040200000000000004BE00DA
:10ECE0006162B9006159B9000400BE005404020019
:10ECF0000000000008004000898048004909DD004C
:10ED00004700DE0000007100C788DE00E00F5500FC
:10ED1000010032000000EA004F0678004F05BE00F7
:10ED20004F04BE0000000600010024000100400066
:10ED3000BEFF37000100240001003700C288DE005A
:10ED4000808F5000FDFF3C00000178000000EB00C8
:10ED500007003700808140000080D100830F510000
:10ED6000020035000301510001004000C288DE00AE
:10ED7000E08F5000F7FF3A0000000600889FBE00B9
:10ED80008A9FBE0080027800010078008001EB00BD
:10ED90004A00200059002000180037000A01B8007E
:10EDA000811F7800110009004999D800CF00780030
:10EDB0000001EB00820178000D0037008203410062
:10EDC0008783420017037800040242000482420055
:10EDD00014047800880553004240A9000300340061
:10EDE000880B7800060A7800130020000201E80072
:10EDF00000024100810F5200F0FF3900E10F500086
:10EE0000E6FF3E00E08F5100E9FF3A004F05BE00EB
:10EE10004F04BE0000000600889FBE008A1F7800D5
:10EE2000000478000800780010FF07000005780053
:10EE3000080078000DFF07008004780008007800C3
:10EE40000AFF07008000EB0007003700C8019000B0
:10EE50000A0145000982440064B179000A05E8000E
:10EE60008904E8008100E800808F5000F7FF390036
:10EE70004F0578004F04BE0000000600889FBE00CA
:10EE80008A1F78000004780008007800F7FE070069
:10EE90008004780008007800F4FE07000005780080
:10EEA00008007800F1FE07008000EB000A0545002D
:10EEB00005003700C8019000098144006AB179005B
:10EEC0008904E8008100E800808F5000F9FF3900D4
:10EED0004F0578004F04BE0000000600889FBE006A
:10EEE0008A9FBE000004780008007800DFFE07005B
:10EEF0000005780008007800DCFE07008004780038
:10EF000008007800D9FE0700800578000800780026
:10EF1000D6FE0700C80090008B85450061817D000A
:10EF20008000EB0009003700C80290008A0145000C
:10EF30008381420009824400048242009409410016
:10EF40000A05E8008904E8008100E800808F50008D
:10EF5000F5FF39004F05BE004F04BE00000006005B
:10EF6000889FBE008A9FBE000004780008007800D9
:10EF7000BEFE07008005780008007800BBFE070091
:10EF80000005780008007800B8FE070080047800CB
:10EF900008007800B5FE07008000EB000D00370088
:10EFA000480190008B8145008301410009824400A3
:10EFB000040241008A024500050141001402780064
:10EFC000920942008B05E8000A05E8008904E80080
:10EFD0008100E800808F5000F1FF39004F05BE002E
:10EFE0004F04BE0000000600889FBE008A9FBE003E
:10EFF00000047800080078009CFE07008005780077
:10F000000800780099FE07000005780008007800E5
:10F0100096FE0700800478000800780093FE070041
:10F020008000EB000D003700480190008B81450007
:10F03000830141000A024500040241008982440024
:10F040000501410014027800920952008B05E80086
:10F050000A05E8008904E8008100E800808F50007C
:10F06000F1FF39004F05BE004F04BE00000006004E
:10F07000889FBE008A9FBE000004780008007800C8
:10F080007AFE0700800578000800780077FE070008
:10F09000000578000800780074FE070080047800FE
:10F0A0000800780071FE07008000EB000C003700BC
:10F0B000480290008B824500898144000A01450086
:10F0C000E4817900640179000299B90002B27A0002
:10F0D0008B05E8000A05E8008904E8008100E800E3
:10F0E000808F5000F2FF39004F05BE004F04BE0074
:10F0F00000000600889FBE008A9FBE008C9FBE0055
:10F100008E1F7800000478000800780057FE070082
:10F11000800578000800780054FE0700000578009C
:10F120000800780051FE070080047800080078008D
:10F130004EFE0700800678000006EB001C0037003A
:10F14000C80090000A004500610078000981440071
:10F1500061017900CF91DE00E00F5100E08F59008E
:10F160000B0032000A05E8008904E8000B8745001F
:10F170000E874000CF80DE00820602000000000003
:10F18000000F78008B05E8000C06E8000800370047
:10F1900023002000730498007001440071002900CE
:10F1A000080078006ECF0200000000000200370067
:10F1B0008D0F5600E2FF39004F0778004F06BE0062
:10F1C0004F05BE004F04BE0000000600889FBE0031
:10F1D0008A9FBE00000478000800780023FE070024
:10F1E000800578000800780020FE07000005780000
:10F1F000080078001DFE07008004780008007800F1
:10F200001AFE07008000EB000F0037004801900055
:10F210008A014500E28179000A05E80089824400FC
:10F220008904E8000B8245000402410062817A00F3
:10F23000830F51000100340003017800020A7800B6
:10F240008B05E8008100E800808F5000EFFF390057
:10F250004F05BE004F04BE0000000600889FBE00A0
:10F260008A9FBE000004780008007800FFFD0700B8
:10F270008005780008007800FCFD07000005780094
:10F2800008007800F9FD0700800478000800780085
:10F29000F6FD07008000EB000F00370048019000EA
:10F2A0008A014500E28179000A05E800898244006C
:10F2B0008904E8000B8245000402410062817A0063
:10F2C000830F510001003D0003017800020A78001D
:10F2D0008B05E8008100E800808F5000EFFF3900C7
:10F2E0004F05BE004F04BE0000000600889FBE0010
:10F2F0008A9FBE008C1F7800000478000800780008
:10F30000DAFD07000006780008007800D7FD070046
:10F310008005780008007800D4FD0700000578001B
:10F3200008007800D1FD070080047800080078000C
:10F33000CEFD07008001EB0014003700C8009000EC
:10F340000B814500610279008B05E8000A01450048
:10F35000E10279000A05E8000981440061017900B1
:10F360008904E800820F520004003C000501780087
:10F37000840F510001003D00040178000C0246009A
:10F3800082307A000C06E8008301E800808F51008B
:10F39000EAFF39004F0678004F05BE004F04BE005B
:10F3A00000000600889FBE008A9FBE008C9FBE00A2
:10F3B0000004780008007800ACFD070080047800A5
:10F3C00008007800A9FD0700800678000800780092
:10F3D000A6FD0700000678004805900008007800A8
:10F3E000A2FD07000001780002014100EA05790052
:10F3F000080078009DFD070000057800000220004D
:10F40000808F550005003C000D0378008C007800CB
:10F410008003EB006011B8000F0037004800900037
:10F420008984440089044000800CEB0014003700FC
:10F4300001804000650278008100E800060043007A
:10F44000650078000603E8000482B900020142006A
:10F4500083814A008703E800C80290008A8F530026
:10F46000F3FF3900898444008B05E9000300330071
:10F470008381D1000281D300FBFF370082B27C0080
:10F480004F06BE004F05BE004F04BE000000060040
:10F49000889FBE008A9FBE008C1F78000004780001
:10F4A0000800780071FD07008004780008007800EB
:10F4B0006EFD070000067800080078006BFD07006D
:10F4C000800578000800780068FD070000057800D6
:10F4D0000800780065FD070000017800E00F51008A
:10F4E000250032004802900009804400E4017800C1
:10F4F0000903E8006118B9000C06460003327E00DB
:10F500008B8445004802900003B27C001700200065
:10F510001000370086014300E48179000603E8000B
:10F520000C024200948F510001003D00030A780054
:10F530004802900009024200948F510001003400FB
:10F54000030A7800611AB9000000420081804A0075
:10F550008703E80048029000828F5300EDFF3900D6
:10F560000A0545000A054200030020008206020049
:10F5700000000000000D78004F0678004F05BE0027
:10F580004F04BE0000000600889FBE008A9FBE0098
:10F59000000478000800780034FD0700800578003A
:10F5A0000800780031FD07000005780008007800A9
:10F5B0002EFD070080047800080078002BFD07006E
:10F5C00000027800E00F5200160032000B017800B4
:10F5D0008000EB0005002800F0FF27000A05450029
:10F5E000898444004803900082014100E68179004B
:10F5F0000201E800808F510002003D0001337D00D0
:10F6000003007800858F510003003400C802900089
:10F6100081B27C00830278008100E800848F500072
:10F62000F0FF39004F05BE004F04BE000000060089
:10F63000889FBE0000047800080078000BFD0700DA
:10F64000800478000800780008FD0700800078003A
:10F65000898444004800900009004000C7FD07006D
:10F660004F04BE0000000600E8874700889FBE00E8
:10F670008A9FBE008C9FBE008E1F78000005780018
:10F680000A007800F9FC0700000778000A007800FB
:10F69000F6FC0700800678000A007800F3FC0700FB
:10F6A000000678000A007800F0FC0700800578006A
:10F6B0000A007800EDFC0700800378000003EB00EF
:10F6C0002A003700CA0090000D80460061027800D1
:10F6D0000C004600610078000B8145006104790050
:10F6E000CFC4DE00E00F5400E08F5C001700320052
:10F6F0008D06E8000C06E8008B05E8000E014700C7
:10F7000002814000E2B79F00CF80DE00CFA2DE0082
:10F710000401BE00F6B79F0087BF9F00540402009B
:10F72000000000000801BE00820602000000000088
:10F730006FB19700000978000E07E8007FB39700CB
:10F740000603E8008FBB9700080037002300200065
:10F750007305980070014500710029000A007800C7
:10F760006ECF02000000000002003700870F530038
:10F77000D4FF39004F0778004F06BE004F05BE008A
:10F780004F04BE008F00B10000000600889FBE003D
:10F790008A9FBE008C9FBE008E1F780000047800F8
:10F7A00008007800B1FC07008005780008007800A8
:10F7B000AEFC07000005780008007800ABFC0700ED
:10F7C0008004780008007800A8FC07000007780093
:10F7D0000006EB000C003700C80690000A00450048
:10F7E0006D0078000A05E80089804400ED8078000B
:10F7F0008904E800A5FC07008B80450080B67800EE
:10F800008B05E8000C06E8008E0F5600F2FF390069
:10F810004F0778004F06BE004F05BE004F04BE00E4
:10F8200000000600889FBE008A9FBE008C9FBE001D
:10F8300000047800080078008CFC070000057800C0
:10F840000800780089FC0700800478000800780030
:10F8500086FC0700000678008005EB0009003700F1
:10F86000C8069000098044006D0078008904E80013
:10F87000EEFC07008A00450080B678000A05E80023
:10F880008B05E8008C8F5500F5FF39004F06BE0050
:10F890004F05BE004F04BE0000000600889FBE005A
:10F8A0008A9FBE008C9FBE0000047800080078008C
:10F8B0006EFC070000057800080078006BFC07006C
:10F8C000800478000800780068FC070000067800D3
:10F8D0008005EB0009003700C8069000098044004D
:10F8E0006D0078008904E8000FFD07008A004500DC
:10F8F00080B678000A05E8008B05E8008C8F55007B
:10F90000F5FF39004F06BE004F05BE004F04BE0094
:10F9100000000600EE874700889FBE008A9FBE0059
:10F920008C9FBE008E1F7800000778000E007800C4
:10F930004EFC0700E0B79F000E0078004BFC07006C
:10F94000000478000E00780048FC0700CE04900008
:10F9500088004400698678000804E8000804440030
:10F9600069037C000000400069047800080078000A
:10F9700086BF9F00ECFC07000005780008007800B7
:10F98000AAFC070000047800EFB097000180400057
:10F9900000804400D0B79F00CFE6DE00CFD5DE0068
:10F9A0000A01BE000C00BE0054040200000000006A
:10F9B000B0B79F00C1B79F000FBB9700CFB3DE0069
:10F9C000CFC4DE000801BE000600BE0086BF9F0057
:10F9D000F7B79F0054040200000000000002BE00C0
:10F9E0003FB09700CFB097000402500085825800C6
:10F9F000C128DD004F22DE0004827000CFAADE00A5
:10FA00005FB1970004097800EFB197000300E800A8
:10FA10004E07900000004000000747000A01BE00AA
:10FA20000FBB9700FFB397000600BE00540402000E
:10FA3000000000000005BE000801BE000C00BE0072
:10FA400054040200000000000A0040008B804800BF
:10FA50004109DD004F00DE0000007100CF88DE00AC
:10FA6000000F78004F0778004F06BE004F05BE001C
:10FA70004F04BE00EF00B10000000600889FBE00EA
:10FA80008A9FBE008C9FBE000004780008007800AA
:10FA9000F6FB07000005780008007800F3FB07007C
:10FAA0008004780008007800F0FB0700000678006A
:10FAB0008005EB0009003700C8069000098044006B
:10FAC0006D0078008904E8009AFC07008A00450070
:10FAD00080B678000A05E8008B05E8008C8F550099
:10FAE000F5FF39004F06BE004F05BE004F04BE00B3
:10FAF00000000600889FBE008A9FBE008004780038
:10FB000009007800D9FB070000047800090078009C
:10FB1000D6FB07000005780009007800D3FB07003A
:10FB20008005780009007800D0FB0700800178008C
:10FB3000490190008B854500E2837D008000EB0049
:10FB4000070037008100E800838F50000400360072
:10FB500008044400080141000009EB004F00370091
:10FB60000A8040000000400062007800E00F500072
:10FB7000F4FF3A00010078000B0037008100E80034
:10FB8000838F50000800360008044400E00F500046
:10FB90003A0032000000E900870F500037003900BA
:10FBA0000000D1003C0037000A82400004024200FD
:10FBB00062027A00E00F5200F0FF32000003EB0017
:10FBC00006007800060278008402780003003700FF
:10FBD0008502E800838F52000B00310081844200CF
:10FBE000809FBE00110009008384D8008104780042
:10FBF0004F00BE008A84440089844400E2847C0073
:10FC0000E08F5400F2FF3A0084845200808F540049
:10FC100003003400048242000483D100090078000C
:10FC2000838F520005003900110037000402E800FC
:10FC3000830F5200020039000D00370005027800E2
:10FC400081024200809FBE00110009008382D8001B
:10FC5000810278004F00BE008A8242008582420005
:10FC6000E2827A00E08F5200D7FF3A00EFFF3700C0
:10FC700008044400870F500003003D0008044100C1
:10FC8000008CEB00050037008100430011000900E3
:10FC90008380D8008000FD0000317C004F05BE004D
:10FCA0004F04BE0000000600B0CE88000000060031
:10FCB00050252600B1CE80000088B9009261230053
:10FCC00000004100B0CE880000000600889FBE0002
:10FCD0008A9FBE008C1F780000047800080078001E
:10FCE00062FB070080047800080078005FFB0700D3
:10FCF000800578000005EB0007003700098044000C
:10FD00004806900000064600E9FF0700000E780054
:10FD10008904E8000A05E8008B0F5500F7FF390059
:10FD20004F0678004F05BE004F04BE0000000600DD
:10FD3000AA24AB000D003200328280009240900075
:10FD400000C8B30080CF500007003A0080828000D6
:10FD50009040900040C8B30080CF500002003A00AD
:10FD60006840400010419800AA24A9000008200023
:10FD70005024880000000600010321009140780013
:10FD800000C8B30080CF50002F003A0000CCB30071
:10FD90005CF0B70033D0BF00E24F500008003200E3
:10FDA000E34F500017003200E14F500025003A00A9
:10FDB00000122100D0828800200120001D003700A1
:10FDC00032D0BF000080FB0000004000E11B21009A
:10FDD000E1007800D1828800D0828000801F780006
:10FDE000204090005EF0B7004F007800D082800085
:10FDF000801F7800304090005FF0B7004F0078001F
:10FE00000000060032D0BF00E24F50000B003E0061
:10FE100032D0BF000080FB0000004000011C210028
:10FE2000E1007800D1828800D08280001040780004
:10FE30000080FB00F0828800000006005C70EF008C
:10FE4000000006005C70EF00000006003870EF0054
:10FE50003970EF0030D0BF007F006000E10F50002C
:10FE60000B003200E20F50000B003200E00F500098
:10FE70001B003A005CF0A8003810A8001084800035
:10FE8000E10F500016003A003830A8001400370087
:10FE90005CF0A800120037005CF0A80034D0BF006E
:10FEA0000500330034D0BF006F0060000000400048
:10FEB000A10421000400370034D0BF006F006000AF
:10FEC0000000400001052100610078001040900012
:10FED000640060000200320010C0B30038F0B700C8
:10FEE0005CF0AB000500320080032100D082880066
:10FEF0005C10A80020C0B3005EF0B7000000060050
:10FF0000F082800081C0B300E70F50000A003E007D
:10FF1000F182800056D0BF0002003A0010C0B3004A
:10FF20000400370056D0BF00E14F500002003A00F5
:10FF300020C0B30056F0B7000180FB005E30B50072
:10FF4000808280000148780080032100408388007F
:10FF50005C10AB00070032000F003700D082800039
:10FF6000428380003059780042838800D082880024
:10FF70008140E900E0CF5000F8FF3A0000000600A1
:10FF8000D08280004283800030597800428388000C
:10FF9000D08288008140E900E0CF5000F8FF3A00AD
:10FFA00000000600881F780080828000100478001E
:10FFB0004E44DE00614464005050AA00008280007C
:10FFC000E80F50000A003A0032D0BF000080FB006A
:10FFD000B0248800B0248000E00F500002003200FE
:10FFE000000120000100370040002000008288004E
:10FFF00058D0BF00E14F500011003A0080032100AB
:020000040001F9
:100000008182800090009800BDFF070061052100FB
:100010009140780080828000E2CF500002003A00D8
:1000200041C8B3000400370081CCB300E04F540056
:100030000100320081C8B30011409800120037005F
:1000400062D0BF000F003B0065D0BF000080FB0006
:100050006106210091407800C808DD000080700032
:100060000700320065D0BF000080FB006106210060
:1000700091407800C808DD00008070000000010099
:1000800062F0A9005870EF004F04780000000600ED
:100090000080FB000181FB000000400000014100E6
:1000A0004311DD00030021000301410012F0A10013
:1000B000E0CF500002003A00A10421000100370007
:1000C000010521008230780012E0A10064014100A6
:1000D00012E0A000000006000001EB00228488006E
:1000E000820078004007200048EE02000000000077
:1000F0008284A9000001200000248800000006007E
:100100008284A800000120005024880010002000F4
:10011000208488000001EB008000EB0050072000E5
:1001200048EE0400000000000200FA00881F78007A
:1001300032D0BF00E14F50000B003A0030D0BF007A
:100140007F40600008003A005CF0A80031D0BF009A
:10015000E34F500003003A00100020001084880094
:10016000010037008230EF0032D0BF008E003A002D
:1001700030D0BF007F406000E24F50008A003A005C
:1001800034D0BF006F4060008700320034D0BF0021
:100190006F006000E20F500083003C00018280008D
:1001A00000022000808F50007F003A005CF0A80021
:1001B00034D0BF000A00330034D0BF006F006000AD
:1001C00000004000A1042100E1007800E1BF9F0091
:1001D00034D0BF006F006000210721000900370004
:1001E00034D0BF006F006000000040000105210016
:1001F000E1007800E1BF9F0034D0BF006F006000D5
:10020000E1062100614478006140640004003A0086
:100210004FF897000024A100C0FF9F0003003700A3
:10022000CFF897000124A000C1FF9F0034D0BF0089
:100230000500330034D0BF006F00600000004000B4
:10024000A10421000400370034D0BF006F0060001B
:1002500000004000010521006FB99700823078004E
:1002600031D0BF00E34F500018003A006FB897003C
:100270008000EB00908F10000E003D0034D0BF00D6
:10028000050033004103210091407800EF806000B9
:10029000220721000400370041032100914078002B
:1002A000EF806000E206210062C078000014A00028
:1002B00000F17800EFB897001141900040C8B300FA
:1002C0000040710090409800370037004FF99700C8
:1002D0000224A200C2FF9F00EFB8970011409000D7
:1002E0000001EB00910F110008003D000074A10017
:1002F0000064A000904098002200200050002000E0
:1003000048EE020000000000020037000064A00078
:10031000904098004FF897000024A200C0FF9F0073
:100320006244640006003A006FB89700024028005B
:100330001001610001002800810F510017003A00F0
:1003400034D0BF0005003300410321009140780004
:10035000EF806000220721000400370041032100E4
:1003600091407800EF806000E206210062C07800D2
:100370000014A10000F17800EFB897001140900040
:10038000B043B200904098002200200050002000AE
:1003900048EE02000000000003003700904090008B
:1003A000B143B200114098004F0478000080FA0079
:1003B000000006005CF0A800AC24EF00AE24EF00C3
:1003C0000040EB00020021008081FB0001002100C1
:1003D000C219DD00830141008009EB00B3117800F0
:1003E0000040E800EB4F5000F7FF36009424A800CF
:1003F0004470EF009424A900688040008082880047
:10040000318288004182880032D0BF0042F0B700BC
:1004100042D0BF0002003A00000120000600370071
:1004200012002000210421001000200048EE0200EC
:10043000000000000002200000828800000006008A
:1004400030D0BF000046B20035003A0031D0BF00C6
:100450000080FB0001002000EB0F5000E08F5800EF
:100460002F003E000060010013003700130037002A
:100470002B00370011003700290037000600370035
:100480000900370021003700090037000700370056
:100490000B003700140037005CF0A800800020003B
:1004A000008288000000060033FE3700C1FF3700DD
:1004B000200421000600370064FE37001AFF3700D1
:1004C00034D0BF000080FB00410421000100400047
:1004D000D08288005C10A80010C0B3005EF0B700A6
:1004E0005CF0A800000006005CF0A80034D0BF005B
:1004F0000080FB0041042100821F780022032100BC
:10050000927078004F017800000006000001EB00B7
:100510008000EB002000200048EE020000000000F8
:10052000000006009EC0A9008EA4EF008AA4EF0080
:10053000AA24EF00AC24EF00AE24EF00200020003E
:1005400030258800A824EF008644A900F009200087
:1005500080248800602488008804A800010021000D
:100560004808DE00C02488000040EB000081FB004A
:100570004211DD00028140000009EB0032117800D9
:100580000040E800EB4F5000F8FF36009424A8002C
:100590009624EF0094A4A9009424A90080002000D0
:1005A00009003700502488005C70EF006270EF0093
:1005B00031062100914078006370EF004106210070
:1005C000914078006470EF0051248000E880600062
:1005D000F4FF3A0010002000C0838800D083880018
:1005E000E1838800F183880021848800014078003D
:1005F00005052100A40421000081FB0082014100C7
:1006000003834200000BEB00830142008009EB00F2
:10061000E3062100817179002307210081717900AF
:100620000040E800E24F5000F3FF36008000210058
:1006300080828800D000200050258800000321001F
:100640001080880080C0B30000F0B70040C8B3003D
:1006500001F0B7004270EF004030EF0000000600EC
:10066000C0838000E00F500024003A0011002000F9
:10067000C1838800D0838000E00F50001F003A0043
:10068000D18388008205210012417800E24F510099
:1006900006003A00818280008048780080CCB30058
:1006A00081828000904098000000060082052100B1
:1006B00012417800E14F510010003A000084880098
:1006C00080C0B3003282800000497800348280000C
:1006D000030321001302980042C8B300124298009D
:1006E0000184880041828000804878004182800037
:1006F0009300980000C8B3009040980000000600E6
:10070000308280009040780063D0BF000080FB0002
:1007100042062100124178004811DD0000007100FE
:100720000181FB00800F51000300360031062100DB
:100730009140780064D0BF0063D0BF000080FB0010
:1007400042062100124178004811DD0000007100CE
:100750008181FB0003005000320621001241780025
:1007600063F0B7004800DE00420621001241780025
:1007700064F0B7000040EB001600370002062100CD
:10078000124178000281FB0013062100934178009A
:10079000C819DD000082FB00028171008303210083
:1007A00063597A0003062100934178000001FD009F
:1007B00060F0B7000001FD004811DE0013062100C3
:1007C000934178000001FD0061F0B7000001FD00D9
:1007D0000040E800814F5000E8FF390063D0BF00BF
:1007E0000080FB004106210091407800C808DD0030
:1007F00000807000418280000E00320080C0B30093
:100800008048780040828000810321001100980018
:1008100001002400328280009280600002003A00D1
:1008200081CCB3000100370081C8B30011409800AB
:100830000000060080C0B30080487800418280003C
:10084000000321009000980040C8B3009040980039
:1008500065D0BF000080FB00610621009140780058
:10086000C808DD00008070000700320065D0BF00BE
:100870000080FB006106210091407800C808DD007F
:10088000008070000000010062F0A900B0838000C9
:10089000E00F500001003A0071FF07000000060061
:1008A00058D0BF00E24F500001003A0094FF3700DB
:1008B0005870EF0000848000E00F500009003A00FB
:1008C00080C0B3004182800080487800418280006F
:1008D0000003210090009800C0C8B3009040980029
:1008E000000006008030EF00000006007C30EF00C2
:1008F0007E30EF0058D0BF00E24F500005003A00B4
:1009000080C0B3004182800080487800418280002E
:100910001200370036D0BF000080FB0071032100B9
:1009200091407800C808DD0000807000F2828000ED
:10093000820F50000700310036D0BF000080FB005E
:100940007103210091407800C808DD00008070002C
:10095000F08288006AFD0700818280008003210008
:100960009000980080CCB3009040980000000600F2
:1009700094A4A9005CF0AB0017003A0062D0BF005D
:1009800009003B0020C0B30058F0B700F08380009E
:10099000E00F500001003A00D4FF07007A30EF006A
:1009A0007830EF000000060080C0B3004182800074
:1009B0008048780041828000000321009000980068
:1009C000C0C8B30090409800684050008182800009
:1009D000904098000000060030D0BF000C003B00A3
:1009E00010C0B30058F0B700E0838000E00F500063
:1009F00001003A00BDFF07007A30EF007830EF00C9
:100A0000B0838000E00F500011003A0014FF37005F
:100A100020C0B30058F0B70080C0B300418280000E
:100A200080487800418280000003210090009800F7
:100A300040C8B300904098007A30EF007830EF0063
:100A4000B0838000E00F500001003A0004FF07006F
:100A500000000600881F78005670EF000004EB00CD
:100A6000B8838800E8838800F883880008848800B9
:100A70000800780058F0B700818280001140900093
:100A80000074A10090409800010521001124A200EB
:100A900082828000124090000074A10010419800F2
:100AA0001124A20041828000114090000074A10036
:100AB00090409800080078005CF0B700F882880049
:100AC0000800780062F0B70063D0BF00080078002B
:100AD00063F0B70064D0BF000004FD0064F0B7000D
:100AE0000004FD0056FE070008017800820078002F
:100AF0003000200048EE0200000000009CFF0700CC
:100B00004F04780000000600D0C2B30086F0B700A2
:100B10006CD0BF00B00FB20020003A00C106210027
:100B2000914078008181FB00C219DE004219DD008E
:100B30000400210084004100318288004182880045
:100B40004850AA006402790002C023000202620039
:100B500002402300820F52000F003A0091029000E1
:100B60000082FB00020321009542780005717A00A3
:100B7000110290000402E800940098000040E80090
:100B8000E74F5000F5FF3600C219DD0020002100BC
:100B900002B07900AFFF370041FF37006CD0BF00D3
:100BA000B00FB200E80F500001003A00FDFC070052
:100BB00000000600889FBE008A1F7800004478006D
:100BC000814478000985FB0068006500030032005D
:100BD0008040EB00084078002DFD070064056500AB
:100BE0000300320011C0B3000840780028FD070060
:100BF0000884FB0008044400A04A200009707C001F
:100C00004F0578004F04BE0000000600E04F500082
:100C10000C003A0080C0B300418280008048780018
:100C2000418280000003210090009800C0C8B300FA
:100C30009040980068405000818280009040980069
:100C4000000006008180FB000080FB0000004000E7
:100C5000008040004300DD0004002100040140004A
:100C60009241900041C8B30081C1710013419800C6
:100C70006400400004004000104190008140710079
:100C80001140980000000600804278000582FB00B9
:100C9000E0CF5000030032000402420000052100B2
:100CA0000200370004024200A004210060007A0024
:100CB000E00F500015003200120098000348780041
:100CC000104190000244B200124098009041900000
:100CD00082C8B30002C17100124098000581FB0078
:100CE000E0CF500005003200020141000105210063
:100CF000010141001224A20000000600020141008F
:100D0000A1042100010141001224A20000000600FC
:100D100094A4AB00180032000080FB0000004000EB
:100D200001052100E10278001501BE000404200045
:100D30000201620003002000828ABE00E102780006
:100D40000204200003002000951A690095926900B2
:100D5000010140001224A200E1017800134190003B
:100D60000244B20092419800E100780011409000E6
:100D70000440680090409800000006000000EB006E
:100D8000A0248800602488000082880000000600FB
:100D900000828000E00F500010003A00A02488007C
:100DA000602488002100200031258800402588002B
:100DB0008644A900F009200080248800602488006F
:100DC0009EC0A800010037009404A8009404AB0062
:100DD000FDFF3200100020000082880000000600A5
:100DE000627E2400F10F200012C8600012419000C2
:100DF00012409800827E2400928160002340980077
:100E00001241900032409800A27E2400928060003F
:100E1000414098001241900052409800917F240078
:100E20009140780061409800A17F240091407800B3
:100E300071409800B17F24009140780001489800EB
:100E4000C17F24009140780011489800C17E2400A1
:100E50009140780021489800D17E2400914078008C
:100E600031489800E17E2400914078004148980084
:100E7000F17E24009140780051489800017F2400C1
:100E80009140780061489800117F240091407800DB
:100E900071489800417F24009140780001509800EB
:100EA000517F24009140780011509800317F240038
:100EB0009140780021509800717F24009140780083
:100EC00031509800817F2400914078004150980073
:100ED00000000600889FBE008A9FBE008C9FBE0057
:100EE0000004BE000C4020000D002000000646005B
:100EF00081864E00FAFF2F00FB0F2000080037000C
:100F00000800BE0072C70200000000008A0F5000F7
:100F10008B8F580007003A0062044400E0844C00C4
:100F20008C0F54008D8F5C00F5FF39000000EB0042
:100F300001003700100020004F06BE004F05BE0024
:100F40004F04BE00000006000001EB00110221006A
:100F5000000120001AEF02000000000081012000C3
:100F6000607E240026EF02000000000062EF020015
:100F7000000000008000780010002000E27F2400C4
:100F8000928F5000010032000000EB0000000600CC
:100F90002E00FA0023FD2F008F814100D202200095
:100FA000BCC7020000000000100020009FA89700AE
:100FB000E38F5000010032000000EB000080FA00D7
:100FC000000006001600FA00889FBE008A9FBE003F
:100FD0007E044000E08448000A4020000B0020000E
:100FE0000005450081854D000A003700FE8157004D
:100FF000520120000800BE00BCC702000000000033
:101000000FE897006100600006003A006E0444009B
:10101000E0844C008A0F54008B8F5C00F3FF390092
:101020006044B8000800BE004F05BE004F04BE007B
:101030000080FA00000006001600FA00889FBE003B
:101040008A9FBE008C1F7800000678000205BE0053
:101050008C017800D20220000A00BE00BCC702004A
:10106000000000000C6890000040E800006E98004E
:101070007E044500E0844D00004020000100200077
:101080000A0540008B854800CA00370003FE2F0088
:101090008F814100520120000800BE00BCC7020041
:1010A00000000000CC6090006FE0970000C070006E
:1010B00040669800DC6090007FE0970000C0700000
:1010C00050669800EC6090000FE8970000C0700038
:1010D00060669800FC6090001FE8970000C07000F8
:1010E00070669800CFF097008180FB002C61900023
:1010F0000281FB003C6090004800DD0002007000AF
:1011000000804000206698004800DE0030669800AD
:10111000BFF097008180FB000C6190000281FB0012
:101120001C6090004800DD0002007000008040005C
:10113000006698004800DE0010669800AFF0970047
:101140008180FB006C5990000281FB007C5890006C
:101150004800DD000200700000804000605E9800E2
:101160004800DE00705E98009FF097008180FB00D1
:101170004C5990000281FB005C5890004800DD0053
:101180000200700000804000405E98004800DE00D1
:10119000505E98008FF097008180FB002C599000E2
:1011A0000281FB003C5890004800DD000200700006
:1011B00000804000205E98004800DE00305E98000D
:1011C000FFE897008180FB000C5990000281FB0032
:1011D0001C5890004800DD000200700000804000B4
:1011E000005E98004800DE00105E9800EFE897006F
:1011F0008180FB006C5190000281FB007C509000CC
:101200004800DD0002007000008040006056980039
:101210004800DE0070569800DFE897008180FB00F0
:101220004C5190000281FB005C5090004800DD00B2
:101230000200700000804000405698004800DE0028
:1012400050569800CFE897008180FB002C51900009
:101250000281FB003C5090004800DD00020070005D
:1012600000804000205698004800DE00305698006C
:10127000BFE897008180FB000C5190000281FB00C9
:101280001C5090004800DD0002007000008040000B
:10129000005698004800DE00105698004C49900017
:1012A0000281FB00DC499000C819DD00028071005A
:1012B0006C4990000281FB00FC499000C819DD00D8
:1012C000828071002FB1970002004000E08048004A
:1012D000404E98004801DE00524E9800614E980042
:1012E0004808DE00704E98000C4990000281FB0017
:1012F0009C499000C819DD00028071002C499000C3
:101300000281FB00BC499000C819DD008280710099
:101310001FB1970002004000E0804800004E980096
:101320004801DE00124E9800214E98004808DE0069
:10133000304E98004C4190000281FB00DC4190004F
:10134000C819DD00028071006C4190000281FB0031
:10135000FC419000C819DD00828071000FB1970038
:1013600002004000E0804800404698004801DE004E
:1013700052469800614698004808DE007046980082
:10138000AFE897008180FB002C4190000281FB00B8
:101390003C4090004800DD000200700000804000EA
:1013A000204698004800DE00304698006E04440055
:1013B000E0844C008A0F54008B8F5C0033FF3900AF
:1013C0004F0678004F05BE004F04BE000080FA00B3
:1013D000000006003200FA00889FBE008A9FBE000F
:1013E0008C1F78000004BE00E00F5100E08F590010
:1013F00008003A000E0078000F0778008E03B10055
:1014000015000900001FEB00005FEB0000077800EB
:101410000300370080FC2F000F00400006FF07008C
:1014200030002000C0A79F000800BE00A9FE0700F2
:10143000E00F5000030032000800BE001AC802008E
:10144000000000000005EB00CC02200051FC2F0042
:101450008F8040008105E8001000370081FC2F00DC
:101460008F8040000A804000B0407800C1C79F00D4
:10147000B0407800D1C79F00904D78002FA1970011
:10148000BFA197000800BE0056C80200000000007F
:1014900062044400E0844C00630545008C0F550055
:1014A000EEFF36004F0678004F05BE004F04BE0029
:1014B0000080FA000000060000C023001100200098
:1014C000B3FE0700E00F500014003A0000002400B3
:1014D00011002000AEFE07006011B800E00F5000C0
:1014E000080032000000240011002000B5FE0700B3
:1014F000E00F5000E08F580028003A00020024005E
:101500001300200000C0230011002000B1FF0700DD
:10151000E0C12300110020000000060000C02300ED
:1015200011002000A7FE0700E00F5000E08F5800D8
:101530001A003A00000024001100200094FE070069
:10154000E00F500008003A0002C023001300200002
:1015500000002400110020009EFF0700E00124008D
:1015600011002000000006000000240011002000EF
:1015700094FE0700E00F5000E08F580007003A008B
:10158000020024001300200000C0230011002000EE
:1015900090FF0700E0C123001100200000000600BA
:1015A0001A00FA00889FBE008A9FBE008C1F780038
:1015B0000005EB00F028200081458000808F50005E
:1015C0002E003400BCFF07000004BE000BFE2F00FD
:1015D0008F8545000B00780001FE0700D0FD2F002D
:1015E0000F0040000006E8000E0037008A8045002A
:1015F00031407800C0DF9F0031407800D0DF9F008D
:10160000114E78006FA99700FFA997000800BE004F
:1016100056C802000000000062044400E0844C0050
:1016200063054500F40F5500F0FF3600020024006A
:1016300013002000820F5400838F5C0006003A00E4
:1016400002C02300130020000800BE0061FF070055
:101650001A002000090037001A002000044024006E
:1016600015002000840F5400858F5C0003003A00B1
:1016700000C023001100200056FF07000A00780078
:101680004F0678004F05BE004F04BE000080FA00F0
:1016900000000600303F8200E10F400002003200EF
:1016A000617E24008008E800A85D020000000000C0
:1016B000E00F500006003D00717F240011407800CB
:1016C000E14F40000A0032008048E800080037007F
:1016D000E8004000627E2400E2C07800E1CF4000D4
:1016E000030032008140E800680141000171780088
:1016F0008464AB000F003200C6ED02000000000061
:10170000E00F500006003200403F8200E10F400031
:1017100008003200817E24008008E80000000600F6
:10172000503F8200E10F400002003200A17E240001
:101730008008E800000006000080FB00C300DE0017
:10174000927F240002814000C308DD0001005000A8
:10175000110020000008DD001249700000000600A2
:1017600061052000810F50000B0039008100E80066
:10177000810F500004003600F0804000810F5000BF
:1017800005003A000200370070C0B300EAFF3700DE
:1017900000C1B300E8FF070000000600210620009A
:1017A000810F500011003E008180E900810F500040
:1017B0001D003100F1032000810F500007003E00A2
:1017C000E6805000810F500015003100A002B100EA
:1017D000E40F50001C003E000F0037000005B10070
:1017E000E50F500018003E000D00370051062000A4
:1017F000810F500004003E008100E900810F50007D
:101800000D0031000A00370061062000810F5000F2
:101810000D003A000A003700F0C0B300070037009F
:1018200080C0B30005003700E0C0B30003003700FC
:1018300090C0B3000100370010C1B300BEFF3700F5
:1018400000C1B300BCFF070000000600010020003B
:101850007B005000E0805800EF0F5000E08F5800F0
:101860001F003E00006001000F0037000E0037002F
:101870000D0037000E0037000F0037000E00370054
:101880000D003700080037000D0037000E0037004C
:101890000D0037000E0037000D0037000C00370038
:1018A0000F0037000C003700A0C0B300090037005C
:1018B000D0C0B30007003700C0C0B3000500370038
:1018C00020C1B30003003700B0C0B30001003700EF
:1018D00030C1B30098FF370070C1B30096FF070016
:1018E00000000600B2CD8000C3CD80006100410041
:1018F000E0804900B0CD8800C1CD880002302A00C8
:1019000023002000820F5000838F580007003A0008
:10191000B639EF00B839EF00817F2400114078001C
:10192000E14F4000010032008048E800000006005E
:101930000001EB0011022100000120001AEF02005B
:101940000000000081012000607E240026EF0200DC
:101950000000000062EF020000000000F03F8A007B
:101960000000060020C0B30073FF3700B419EC007C
:10197000A0CD880001A62E00810F500002003A0081
:10198000B439EF0043FF070000000600889FBE0047
:101990008A1F780060778000717780008004EB00F8
:1019A00018002000EAFF2F00910F100033003600CE
:1019B000740037008800440001004000100055000A
:1019C00001002000F00F5000E08F580022003E0080
:1019D00000600100100037000F0037000E003700D4
:1019E0000D0037000C0037000B0037000C003700EB
:1019F000190037000C0037000B0037000C003700CF
:101A000015003700100037000B0037000C003700BE
:101A10000F0037000E003700F0C0B3000D00370094
:101A200080C0B3000B003700E0C0B30009003700EE
:101A300000C1B3000700370010C1B3000500370034
:101A400070C0B3000300370040C1B300010037008D
:101A500050C1B30038FF07008800E800010078009B
:101A6000EE0EB4000001780062807800808F540090
:101A700001003100800478000884E800707780005D
:101A8000900F5400CBFF39003A0037007177800087
:101A900008004400610078004C01DE0003002000D3
:101AA000ED0F5100E08F590030003E000260010050
:101AB0000D0037002D003700190037000D003700EA
:101AC0000F003700110037001300370027003700E0
:101AD00026003700140037001100370016003700C9
:101AE000200037001A003700890F54001F0039000A
:101AF000240037000A00600028FF07001B003700A1
:101B00000A00600016FF0700180037000A00600096
:101B100022FF0700020037000A00600010FF0700E4
:101B20000884E800140037004400DD004480DE0033
:101B300008004000070037000800E80000004000EF
:101B40006100780015FF0700630444000A003700B5
:101B50000A006000808F5400040031008004780087
:101B6000020037000A00600038FF07000804E800A0
:101B700001003700FAFF200060778000800F5400DA
:101B8000C2FF39004F0578004F04BE000000060078
:101B9000D17E240011407800E14F40000100320066
:101BA0008048E80079FF3700E7FC0700E00F5000AD
:101BB00003003A00607E24000C0009000018EB00CE
:101BC0004027AB000300320010C0B300DAFE07006C
:101BD0004027A900807F24008040EB0090CF1000B8
:101BE00004003A00313F8200005A2000808F5000EC
:101BF000060036006AFE0700E00F500003003200C6
:101C0000607E24000C0009000018EB00C17E240057
:101C100011407800E14F4000010032008048E800A8
:101C2000000006001C00FA00889FBE008A9FBE00CC
:101C30008C1F7800000678005C019000EC01900099
:101C40000C007800FC4B02000000000008C02300DC
:101C500019002000FA3F24001B0020000800BE00ED
:101C600072C7020000000000E0AF9F00F1AF9F00CC
:101C7000A3FD2F008F81410032002000C1FD2F0005
:101C80008F8040000C0078007A49020000000000BC
:101C90005FA89700E30F500025003A00620444005B
:101CA000E0844C008A0F54008B8F5C00EBFF360001
:101CB00000FE2F000F00400049FC0700A3FD2F008D
:101CC0008F8141005201200001FE2F008F804000D3
:101CD0000C0078007A49020000000000607E2400B9
:101CE0000C0009000018EB0000C0230011002000C8
:101CF00078FC0700E00F50000400320000C0230011
:101D0000110020001AC8020000000000000024009A
:101D1000110020006FFC0700E00F500004003200AB
:101D200000002400110020001AC80200000000007A
:101D30004F0678004F05BE004F04BE000080FA0039
:101D4000000006008000EB000A003700018140001F
:101D5000A001900002814100920178004C1ADE003F
:101D6000EA0F520002003A000390A1000309780034
:101D70008100E80010019000828F5000F3FF3900CD
:101D800000000600881F780000047800611BB8007E
:101D90000002EB00F10F5300E08F5B0066003E0095
:101DA00006600100110037001200370013003700F1
:101DB0001400370015003700160037001C003700EC
:101DC0003200370033003700340037003500370069
:101DD000380037003C0037003F0037004200370032
:101DE00045003700490037004C003700020ADD008B
:101DF00051003700028ADE004F0037000102410027
:101E00004D003700028250004B0037000192B900AC
:101E100049003700E00F510007003200000278004F
:101E2000110009008200D8000002FD0042003700C6
:101E3000E00F51000F003A0020CB2800E00F5000C7
:101E4000040032008200780008007800B28C0200A2
:101E5000000000002300200073049800700144007B
:101E600071002900080078006ECF02000000000019
:101E700024003700801F7800110009008200D8007C
:101E8000010278004F0078002B003700010271003A
:101E900029003700010269002700370001026100B4
:101EA0002500370014002000828F500015003A00F2
:101EB00021003700028168000202EA00020172007C
:101EC0004F12DE001C00370014002000828F5000EB
:101ED00019003C000B00370014002000828F5000D6
:101EE00015003D000700370014002000828F5000CD
:101EF000110035000300370014002000828F5000CD
:101F00000D0034000002EB000B003700140020002D
:101F1000E08F50000300320007003700E08F5000D0
:101F2000040032000202EA00020272004F22DE00C8
:101F30000100370001027800040078004F047800A7
:101F400000000600E18F5000040032000500390057
:101F5000E28F500007003A0004003700E00F500005
:101F600005003D000000EA00000006000080EA00D5
:101F7000000006000000EB00000006008000EB00FF
:101F80000108980071009800211898002001900025
:101F900001097800300190000201410040009000EA
:101FA0000407040000000000200190009201780066
:101FB00010002000090037000002400062027A0091
:101FC000810F520004003A000000E80000004000C9
:101FD00062007800000006000080E800830F5000D7
:101FE000F5FF3900000005000600FA00889FBE00DA
:101FF0008A1F780000047800A8009000080890006C
:1020000000014000E10479004C49DE00030020009B
:10201000EE0F5100E08F5900F1003E000260010018
:102020000E0037001100370019003700220037007A
:102030002D003700380037004B003700750037009F
:102040007E0037008E00370091003700B700370060
:10205000C8003700D0003700DA0037007800900061
:102060000000A10070049800DD003700E800900037
:10207000180890000000E800100C980000004000D4
:10208000C44CDD00C4CCDE0089307800BE003700CF
:10209000E8019000180990000201E800120C980075
:1020A000020141000000E8000000400061007800EB
:1020B00080317900540037006801900018089000C2
:1020C0000000E800100C980000004000F1FF200024
:1020D00081846400C800900089844400E1847C000D
:1020E00009317800A800370018089000F1FF20009F
:1020F000818464004801900089844400E8019000D4
:1021000080004000E380780001B17C000000E9001D
:10211000100C98009C0037000001E800020141000B
:10212000E10179001809900002014100E8009000E7
:102130000281400092007800838F50000300390034
:10214000A0BF9F00B3BF9F0015003700F0FF200025
:1021500080846400898040004800900081804000B5
:1021600060897800280037000001E8000201410082
:102170006101790068029000980890008101E900EF
:1021800083814100E481790081804000E48078000F
:10219000828F500013003900A0BF9F00B2BF9F0084
:1021A000C1BF9F0020002000700498006300200041
:1021B0006C81570061002900080078006ECF020092
:1021C0000000000020CB2800E00F50008400320007
:1021D0008000EB0008007800B28C020000000000D4
:1021E0007F003700F0FF2000808464008980400079
:1021F000480090008180400003B0780018089000EB
:102200000080E900100C9800080890000080E800A9
:102210005F003700180D90000A0545006800900027
:102220000A05400089007800F10FB2001A0078001A
:1022300044FF0700000D780053003700E8009000CD
:1022400018089000000140000000E9000000400074
:102250008981FB0061017900E100780008007800C5
:10226000C8FE0700980890008100E900110C980052
:10227000680190008180400000B178004200370082
:10228000C44CDD00C4CCDE000080440040003700B8
:10229000E800900018089000000140000000E900EC
:1022A000000040008981FB0061017900E1007800B5
:1022B00008007800B3FE0700980890008180E900CC
:1022C000110C980088089000E00F500005003200C3
:1022D0000930B2002200200003302000838F540018
:1022E00006003A00A80190000101E8000201410047
:1022F00063017900E00F500005003200818040004A
:1023000028009000810040001190A00003003700D9
:1023100081804000818041001190A1000808900058
:1023200002014000020C98002D0037000081E800F7
:1023300002014100E10179000000E80000004000D6
:102340006101780002014100480090000201400054
:10235000F1FF200081806400838141000800780043
:102360006ECF0200000000000808900063004000EB
:1023700007003700F1FF200081806400080078002A
:102380005EB4020000000000080890000000E800B1
:10239000000C980012003700680190009808900027
:1023A0008100E800110C980081804000810041000C
:1023B0008008E800F0FF200080846400090C980089
:1023C0000700370018089000680190008000400066
:1023D000E2807800010C98000000E900100C9800E1
:1023E0004F0578004F04BE000080FA000000060090
:1023F0000000FA00889FBE008A9FBE008C9FBE002E
:1024000080047800810578000F0678000B007800C2
:10241000140702000000000000047800E3064400F6
:10242000650044000000A100808747000C0578008B
:1024300020CB2800E00F5000040032008B00780011
:1024400009007800B28C020000000000200020008B
:10245000F004980009089000000D780028459800C5
:1024600063004500080178008B007800F406020044
:10247000000000008D0178000A0178009100290019
:10248000090078006ECF0200000000008C07780081
:102490004F06BE004F05BE004F04BE000080FA008C
:1024A000000006008000EB000B0037006A8140004E
:1024B000020141006001790080099000830F510002
:1024C00004003A00F00090000110A0007100980094
:1024D000100005008100E80020199000828F500054
:1024E000F2FF390000000500889FBE000004BE0016
:1024F000780090000020A00070049800E08F540045
:102500000D0032000300370008007800B6FE070017
:102510008904E9007800900065006000E50F500034
:1025200009003A00E08F5400F7FF3A000600370038
:1025300008007800ACFE070078009000650060009D
:10254000E50F5000FAFF3200780090000020A10053
:10255000700498004F04BE0000000600A01990000F
:102560000041EB00EF8F510006003E006A81410000
:1025700002014100013079008301E800231898002E
:1025800012C0B3000240780000000600010178008C
:102590008000EB00120037006A8240000402420013
:1025A00060027A00820F52000C003A000301E90039
:1025B0002218980006003700EA814000038241009B
:1025C000EB81400083814100633278008100E800A4
:1025D000828F5000F8FF3900100005008100E800EC
:1025E000A0199000838F5000EBFF39000000050018
:1025F0008000EB0021189800000006000400FA009B
:1026000080089000E1BF9F00F0009000F1BF9F00A4
:102610004300200064815700A10029006ECF020012
:10262000000000000080FA0000000600889FBE0045
:102630000004BE00780090000020A0007004980004
:10264000E08F54001B0032000700370008007800BC
:1026500094FF0700E00F50000E003A0008007800D9
:1026600061FE07008904E9007800900065006000C1
:10267000E50F500013003A00E08F5400F3FF3A00DA
:10268000100037000800780086FF0700E00F5000B8
:1026900006003200780090000010A000700498003E
:1026A00008007800D5FF070009003700080078000F
:1026B0004DFE07007800900065006000E50F5000B7
:1026C000F0FF3200780090000020A1007004980014
:1026D0004F04BE0000000600F0019000618161001F
:1026E0000B003200E28161000001EB00828F51009B
:1026F00007003A0020199000E00F5100020032005C
:10270000CAFF07000100370077FF07001200200012
:102710000200780000000600889FBE0000047800D8
:102720000800780020FE070080047800E08F540045
:102730001300320078009000610060000600320053
:102740007001440023002000810029000800780067
:102750006ECF020000000000090C98000080EB0022
:10276000100C9800F80090000100A000710498007F
:10277000E280600002003200080078009FFF07003E
:10278000090078004F04BE00000006000600FA00B1
:10279000881F78000004780000002A00808F500015
:1027A00004003A0040002000920F100097003E0005
:1027B0009300370010012A00808F500006003A0075
:1027C00050002000C0BF9F002300200068815700F8
:1027D000C10029005F003700E08F51008B003200FC
:1027E00012007800980F500088003A000280E8003C
:1027F0000302E900F2FF2500F3FF2F000101410071
:10280000E0814900EF0F5100E08F59007F003E004A
:10281000026001000F0037001B0037002A0037005C
:10282000350037003A0037003F00370035003700E9
:102830003F0037004B0037004E0037005000370094
:102840005500370062003700650037006800370028
:102850006B003700900178000402E9008000EB0073
:102860000700370003814000020141002803900067
:102870008100E80081824000E0827A00053379001F
:10288000848F5000F7FF390020002000700498006A
:10289000080078002BFD0700E0E72A00E00F500059
:1028A00003003200080078007EAE02000000000045
:1028B0008080EB000800780097FF0700E00F5000D1
:1028C00052003A000F003700780090000010A1007D
:1028D000700498000800780048FF070080DC28009A
:1028E000E00F50004900320008007800C88D020057
:1028F0000000000045003700780090000010A000A4
:1029000070049800080078003CFF07003F00370083
:1029100078009000610060003C0032000800780000
:10292000B1FD0700F7FF370020002000F4FF37005B
:1029300090007800D1BF9F000800780007FF0700D3
:102940000080FB00E0BF9F0043002000668157002D
:10295000B1002900080078006ECF020000000000DE
:102960002A003700900078000800780007FF070071
:1029700026003700080078001DFF070023003700FD
:102980001001900090007800080078009CCF0200B1
:10299000000000001D003700900178000402E900EB
:1029A0008000EB0007003700038140000201410076
:1029B000480390008100E80081824000E0827A00B4
:1029C00005337900848F5000F7FF39000F0037007E
:1029D000080078006EB40200000000000B00370011
:1029E0000800780032B40200000000000700370041
:1029F0000800780052B40200000000000300370015
:102A000008007800E8CF0200000000004F047800C2
:102A10000080FA000000060092007800E08F50006D
:102A20000600350060FD070013002000E00F500095
:102A3000120032008001EB0010003700130020006C
:102A4000F4FF2900848F50000C0036001201900022
:102A50008001EB000402E800848F50000700320080
:102A600071024200848F500004003200900169001E
:102A70000300EA0083017000CF19DE000300780034
:102A80000000060090089000E001900001814000E5
:102A9000630179008100E9001108980002007800C4
:102AA000000006000002EB0002712200A5002000D9
:102AB000811F7800110009000280D8008001780091
:102AC00001007800CF007800E08F510004003A0048
:102AD000E00F520002003A00E10F510003003A00FB
:102AE00004C3B30084D8410014002000809FBE00BE
:102AF000110009000581D800000178004F00BE00D8
:102B0000E00F5100EAFF3A000100780000000600E3
:102B1000E4FF0700E1C2B3000148780071C7B300C9
:102B200001687800F6C0500001687800F5C04000E8
:102B3000016878008040EB0011409800000006001A
:102B4000889FBE008A1F780000047800C8049000A7
:102B500008007800CBFF070000004000E90478007F
:102B60004805900008007800C6FF070000004000FC
:102B7000EA007800EF8F540008003200E08F540024
:102B80000600350070022000808F540003003C00D6
:102B900009407800BEBE0200000000004F0578002A
:102BA0004F04BE00000006000E00FA00881F7800E7
:102BB0008E0078000F0778000E01B10005000900B3
:102BC000001FEB00005FEB000107780001C7B300B6
:102BD00081F79F0040049000AAFF0700000040001A
:102BE00068047800100020000C640200000000005F
:102BF0009EDD0200000000000000EB00E10F440039
:102C000004003200EF80570008007800C0FF070082
:102C10007080570038DE0200000000004F0478008A
:102C20000080FA00000006000E00FA00881F7800FD
:102C30008E0078000F0778000E01B1000500090032
:102C4000001FEB00005FEB000107780021C7B30015
:102C500081F79F00400490008AFF070000004000B9
:102C600068047800E10F440003003A00D0B002008D
:102C70000000000009003700100020000C64020072
:102C800000000000EF80570008007800A0FF070058
:102C90007080570070B00200000000004F04780000
:102CA0000080FA00000006000E00FA00881F78007D
:102CB0008E0078000F0778000E01B10005000900B2
:102CC000001FEB00005FEB000107780021C7B30095
:102CD00081F79F00400490006AFF07000000400059
:102CE00068047800100020000C640200000000005E
:102CF0009EDD0200000000000000EB00E10F440038
:102D000004003200EF8057000800780080FF0700C1
:102D10007080570038DE0200000000004F04780089
:102D20000080FA00000006000E00FA00881F7800FC
:102D30008E0078000F0778000E01B1000500090031
:102D4000001FEB00005FEB000107780031C7B30004
:102D500081F79F00400490004AFF070000004000F8
:102D600068047800100020000C64020000000000DD
:102D70009EDD0200000000000800780052DE020024
:102D80000000000080007800E08F50000600320054
:102D9000EF805700080078005DFF07007080570043
:102DA00038DE0200000000004F0478000080FA00C6
:102DB00000000600E6874700889FBE008A9FBE008D
:102DC0008C9FBE008E1F780000047800C80490001D
:102DD000080078002BFF070000004000E90478009D
:102DE000480590000800780026FF0700000040001A
:102DF0006A057800C80590000800780021FF0700E8
:102E000000004000EB0578004806900008007800BC
:102E10001CFF0700000040006C067800C806900008
:102E20000800780017FF070000004000ED0678005A
:102E3000480790000800780012FF070000004000DB
:102E40006E077800C800900008007800F1B79F0076
:102E50000CFF070000004000FFB0970061037800FE
:102E6000C800900008007800F1B79F0086BF9F005F
:102E700004FF070000004000FFB0970061047800E5
:102E8000001020000C64020000000000884378005D
:102E90000FBB97008E4278000D4278008C4178007D
:102EA0000B4178008A40780009407800B2BF0200E8
:102EB000000000004F0778004F06BE004F05BE001F
:102EC0004F04BE006F00B10000000600889FBE00E6
:102ED0008A9FBE0000047800C804900008007800B3
:102EE000E8FE070000004000E90478004805900073
:102EF00008007800E3FE0700000040006A05780043
:102F0000C805900008007800DEFE070000004000C1
:102F10006B0178008A4078000940780002C0020006
:102F2000000000004F05BE004F04BE000000060078
:102F3000889FBE008A9FBE0000047800C8049000ED
:102F400008007800CFFE070000004000E904780088
:102F50004805900008007800CAFE07000000400005
:102F60006A057800C805900008007800C5FE0700D3
:102F7000000040006B0178008A407800094078002A
:102F80001EC00200000000004F05BE004F04BE003E
:102F900000000600889FBE008A9FBE0000047800E3
:102FA000C804900008007800B6FE0700000040004A
:102FB000E90478004805900008007800B1FE070099
:102FC000000040006A057800C805900008007800FD
:102FD000ACFE0700000040006B0178008A407800DA
:102FE000094078003AC00200000000004F05BE0012
:102FF0004F04BE0000000600889FBE008A9FBE00EE
:103000008C1F780000047800C80490000800780045
:103010009CFE070000004000E9057800C80490000D
:103020000800780097FE070000004000690578005E
:10303000C80490000800780092FE070000004000DD
:10304000E904780048069000080078008DFE07002B
:10305000000040006C047800200020000C64020096
:10306000000000008B40780000C2B300BEBE02002A
:10307000000000008A40780030C2B300BEBE0200EB
:10308000000000008940780010C2B300BEBE0200FC
:10309000000000008840780020C2B300BEBE0200DD
:1030A000000000004F0678004F05BE004F04BE0030
:1030B00000000600E6874700889FBE008A9FBE008A
:1030C0008C9FBE008E1F780000047800C80490001A
:1030D000080078006BFE070000004000E90478005B
:1030E000480590000800780066FE070000004000D8
:1030F0006A057800C80590000800780061FE0700A6
:1031000000004000EB0578004806900008007800B9
:103110005CFE0700000040006C067800C8069000C6
:103120000800780057FE070000004000ED06780018
:10313000480790000800780052FE07000000400099
:103140006E077800C800900008007800F1B79F0073
:103150004CFE070000004000FFB0970061037800BC
:10316000C800900008007800F1B79F0086BF9F005C
:1031700044FE070000004000FFB0970061047800A3
:10318000400020000C64020000000000884378002A
:103190000FBB97008E4278000D4278008C4178007A
:1031A0000B4178008A4078000940780056C0020040
:1031B000000000004F0778004F06BE004F05BE001C
:1031C0004F04BE006F00B10000000600889FBE00E3
:1031D0008A1F780000047800C80490000800780076
:1031E00028FE070000004000E90478004805900030
:1031F0000800780023FE0700000040006A04780001
:10320000400020000C6402000000000089407800AB
:1032100060C1B300BEBE020000000000884078001C
:1032200070C1B300BEBE0200000000004F05780070
:103230004F04BE0000000600881F78004004900084
:1032400010FE070000004000680478000004200021
:103250000C6402000000000088407800D0C1B30078
:10326000BEBE0200000000004F047800000006000F
:10327000881F78004004900002FE07000000400014
:1032800068047800000120000C64020000000000C7
:1032900088407800E0C1B300BEBE0200000000001C
:1032A0004F04780000000600889FBE008A1F780047
:1032B00000047800C804900008007800F1FD0700C1
:1032C00000004000E90478004805900008007800FC
:1032D000ECFD0700000040006A0478000020200098
:1032E0000C640200000000008940780060C2B30056
:1032F000BEBE0200000000008840780070C2B3002B
:10330000BEBE0200000000004F0578004F04BE0062
:1033100000000600889FBE008A1F78000004780025
:10332000C804900008007800D6FD070000004000A7
:10333000E90478004805900008007800D1FD0700F6
:10334000000040006A047800100020000C640200B5
:10335000000000009EDD02000000000088007800F0
:103360000900780074DE0200000000004F057800BC
:103370004F04BE0000000600889FBE0000047800D5
:10338000C804900008007800BEFD0700000040005F
:10339000008044008000EB00F30F2000D2082000E2
:1033A000018240000402400005082000148242000F
:1033B000830F520005003600C17F29000800780005
:1033C000F891020000000000050037008100E800CD
:1033D000828F5000F2FF34009CED020000000000DC
:1033E0004F04BE0000000600881F780040049000D3
:1033F000A4FD07000000400068007800E00F5000C6
:1034000003003200F2AA02000000000002003700B0
:10341000FCAA0200000000004F0478000000060033
:103420000E00FA00889FBE008A1F78000004780012
:10343000C80490000800780092FD070000004000DA
:1034400069057800080078008EFD07008004780088
:103450000E0078000F0778004E01B100050009004A
:10346000001FEB00005FEB000007780051C7B300BE
:10347000C1EF9F00E10F450008003A000000EB009B
:10348000C6B102000000000048009000898444009A
:1034900089044000800CEB0014003700F3805700D3
:1034A0000A0078007FFD0700E1C2B3000148780000
:1034B00041C6B30001687800E3C05000016878009D
:1034C000F3C04000016878008040EB001140980094
:1034D00089844400480090008904400074805700AB
:1034E000C6B1020000000000800C78004F05780093
:1034F0004F04BE000080FA0000000600889FBE0056
:103500008A9FBE0000047800C8059000080078007B
:103510005CFD0700800478000800780059FD070072
:10352000000578000800780056FD0700800078004C
:103530000A054500480090000A05400081804000CF
:1035400089844400098045009CB20200000000000C
:10355000000DD1004F05BE004F04BE000000060064
:10356000889FBE008A9FBE0000047800C8059000B6
:103570000800780043FD0700800478000800780008
:1035800040FD070000057800080078003DFD0700B9
:10359000800078000A054500480090000A054000B8
:1035A00081804000898444000980450054B20200B3
:1035B00000000000000DD1004F05BE004F04BE000A
:1035C00000000600889FBE0000047800C804900038
:1035D000080078002BFD070000004000E904780097
:1035E0000800780027FD07008000780081804000F7
:1035F00048049000010444006148B9000000400004
:103600008180480014B2020000000000000C780025
:103610004F04BE0000000600881F780040049000A0
:1036200018FD0700000040006800780058BC020048
:10363000000000009EBD0200000000004F04780062
:1036400000000600889FBE000004EB00890E2000E9
:10365000803E2000CEEF0200000000000804E800D9
:10366000890F5400FAFF36004F04BE000000060028
:1036700001C2B30080C0B300BEBE02000000000063
:10368000F0FF07008040EB0080C0B300BEBE020028
:103690000000000001C2B30090C0B300BEBE020033
:1036A00000000000E7FF07008040EB0090C0B3007F
:1036B000BEBE02000000000001C2B300A0C0B30003
:1036C000BEBE020000000000DEFF07008040EB00ED
:1036D000A0C0B300BEBE02000000000001C2B300E3
:1036E000B0C0B300BEBE020000000000D5FF07005E
:1036F0008040EB00B0C0B300BEBE0200000000007E
:1037000001C2B300C0C0B300BEBE02000000000092
:10371000CCFF07008040EB00C0C0B300BEBE02007B
:103720000000000001C2B300D0C0B300BEBE020062
:1037300000000000C3FF07008040EB00D0C0B300D2
:10374000BEBE02000000000001C2B30020C0B300F2
:10375000BEBE020000000000BAFF07008040EB0080
:1037600020C0B300BEBE02000000000001C2B300D2
:1037700030C0B300BEBE020000000000B1FF070071
:103780008040EB0030C0B300BEBE0200000000006D
:1037900001C2B30040C0B300BEBE02000000000082
:1037A000A8FF07008040EB0040C0B300BEBE04008D
:1037B0000000000001C2B30020C2B300BEBE020080
:1037C000000000009FFF07008040EB0020C2B30014
:1037D000BEBE02000000000001C2B300014078003C
:1037E000BEBE02000000000096FF07008040EB0014
:1037F00000C2B300BEBE02000000000001C2B30060
:1038000030C2B300BEBE0200000000008DFF070002
:103810008040EB0030C2B300BEBE020000000000DA
:1038200001C2B30010C2B300BEBE0200000000001F
:1038300084FF07008040EB0010C2B300BEBE04004E
:103840000000000001C2B300C0C1B300BEBE020050
:10385000000000007BFF07008040EB00C0C1B30008
:10386000BEBE02000000000001C2B30040C2B300AF
:10387000BEBE02000000000072FF07008040EB00A7
:1038800040C2B300BEBE02000000000001C2B3008F
:1038900050C2B300BEBE02000000000069FF070076
:1038A0008040EB0050C2B300BEBE0200000000002A
:1038B00001C2B300F0C1B300BEBE020000000000B0
:1038C00060FF07008040EB00F0C1B300BEBE020005
:1038D0000000000001C2B30080C1B300BEBE020000
:1038E0000000000057FF07008040EB0080C1B300DC
:1038F000BEBE02000000000001C2B30090C1B300D0
:10390000BEBE0200000000004EFF07008040EB003A
:1039100090C1B300BEBE02000000000001C2B300AF
:10392000A0C1B300BEBE02000000000045FF0700BA
:103930008040EB00A0C1B300BEBE0200000000004A
:1039400001C2B300B0C1B300BEBE0200000000005F
:103950003CFF07008040EB00B0C1B300BEBE0400D6
:103960000000000001C2B30000C1B300BEBE0200EF
:103970000000000033FF07008040EB0000C1B300EF
:10398000BEBE02000000000001C2B30010C1B300BF
:10399000BEBE0200000000002AFF07008040EB00CE
:1039A00010C1B300BEBE02000000000001C2B3009F
:1039B00040C1B300BEBE02000000000021FF0700AE
:1039C0008040EB0040C1B300BEBE0200000000001A
:1039D00001C2B30050C1B300BEBE0200000000002F
:1039E00018FF07008040EB0050C1B300BEBE0200CC
:1039F0000000000001C2B30020C1B300BEBE02003F
:103A0000000000000FFF07008040EB0020C1B30062
:103A1000BEBE02000000000001C2B30030C1B3000E
:103A2000BEBE02000000000006FF07008040EB0061
:103A300030C1B300BEBE0400000000008040EB00B7
:103A400050C0B300BEBE020000000000C5FF07006A
:103A500001C2B300D0C1B300BEBE0200000000002E
:103A6000F8FE07008040EB00D0C1B300BEBE0200EC
:103A70000000000001C2B300E0C1B300BEBE0200FE
:103A800000000000EFFE07008040EB00E0C1B30043
:103A9000BEBE02000000000001C2B30050C0B3006F
:103AA000BEBE020000000000E6FE07008040EB0002
:103AB00050C0B300BEBE02000000000001C2B3004F
:103AC00060C0B300BEBE020000000000DDFE0700C3
:103AD0008040EB0060C0B300BEBE020000000000EA
:103AE00001C2B30070C0B300BEBE020000000000FF
:103AF000D4FE07008040EB0070C0B300BEBE0200E1
:103B0000000000004FFF07002AFF070001C2B300BA
:103B100060C2B300BEBE020000000000C9FE070084
:103B20008040EB0060C2B300BEBE02000000000097
:103B300001C2B30070C2B300BEBE020000000000AC
:103B4000C0FE07008040EB0070C2B300BEBE0200A2
:103B50000000000001C2B3000040EB00BEBE020046
:103B600000000000B7FE07008040EB000140780035
:103B7000BEBE02000000000001C2B300E0C0B300FE
:103B8000BEBE020000000000AEFE07008040EB0059
:103B9000E0C0B300BEBE02000000000001C2B300DE
:103BA00010C0B300BEBE020000000000A5FE07006A
:103BB0008040EB0010C0B300BEBE02000000000059
:103BC00001C2B30060C1B300BEBE0200000000002D
:103BD0009CFE07008040EB0060C1B300BEBE020047
:103BE0000000000001C2B30070C1B300BEBE0200FD
:103BF0000000000093FE07008040EB0070C1B3009E
:103C0000BEBE02000000000099FE37008BFF0700D7
:103C100001C2B30020C0B300BEBE0200000000001D
:103C200001C2B30000C1B300BEBE0200000000002C
:103C300001C2B30010C1B300BEBE0200000000000C
:103C400001C2B30040C1B300BEBE020000000000CC
:103C500001C2B30020C1B300BEBE020000000000DC
:103C600001C2B30030C1B300BEBE020000000000BC
:103C700001C2B3000040EB00BEBE02000000000025
:103C800001C2B30010C0B300BEBE020000000000BD
:103C900001C2B300E0C1B300BEBE020000000000DC
:103CA00001C2B30070C2B300BEBE0200000000003B
:103CB00001C2B30080C1B300BEBE0200000000001C
:103CC00001C2B30090C1B300BEBE020000000000FC
:103CD00001C2B300A0C1B300BEBE020000000000DC
:103CE00001C2B300B0C1B300BEBE020000000000BC
:103CF00001C2B300C0C1B300BEBE0200000000009C
:103D000001C2B30040C2B300BEBE0200000000000A
:103D100001C2B30050C2B300BEBE020000000000EA
:103D200001C2B300F0C1B300BEBE0200000000003B
:103D300001C2B300D0C1B300BEBE0200000000004B
:103D400001C2B30060C1B300BEBE020000000000AB
:103D500001C2B30070C1B300BEBE0200000000008B
:103D600001C2B30080C0B300BEBE0200000000006C
:103D700001C2B300D0C0B300BEBE0200000000000C
:103D800001C2B300E0C0B300BEBE020000000000EC
:103D900000802000F46302000000000010002000FA
:103DA0007ADF04000000000031468000910CB10071
:103DB000A0122000808F500005003E00BA19A80014
:103DC0008040EB0063405000BEBE020000000000D7
:103DD00080458000B208B400813E20000180B90017
:103DE000A2F82000811F7800110009004288D80045
:103DF000CF007800C018B10011022000810F5000E0
:103E000005003E008040EB00D0C0B300BEBE020003
:103E100000000000BA39A800914380005138B10079
:103E2000A0C12000808F500005003E008040EB00C4
:103E300000C1B300BEBE020000000000BA59A800D5
:103E4000A14380005138B100A0C12000808F5000F4
:103E500005003E008040EB0010C1B300BEBE020072
:103E600000000000BA79A800B14380005138B100C9
:103E7000A0C12000808F500005003E008040EB0074
:103E800040C1B300BEBE020000000000BA99A80005
:103E9000C14380005138B100A0C12000808F500084
:103EA00005003E008040EB0020C1B300BEBE020012
:103EB00000000000BAB9A800D14380005138B10019
:103EC000A0C12000808F500005003E008040EB0024
:103ED00030C1B300BEBE020000000000BAD9A80085
:103EE000E14380005138B100A0C12000808F500014
:103EF00005003E008040EB0001407800BEBE02009D
:103F000000000000BAF9A800F14380005138B10068
:103F1000A0C12000808F500005003E008040EB00D3
:103F200010C0B300BEBE020000000000BB19A80014
:103F3000414580005106B100E0312000808F5000E3
:103F400005003E008040EB0060C1B300BEBE020031
:103F500000000000BB39A800514580005106B100A7
:103F6000E0312000808F500005003E008040EB00D3
:103F700070C1B300BEBE020000000000BB59A80023
:103F800050468000E00F500003003A004046800099
:103F9000E00F5000050032008040EB00D0C1B300BC
:103FA000BEBE020000000000BB79A8008002200015
:103FB00061468000808F50000C00340080468000F5
:103FC000810C2000810F500008003400B112200045
:103FD000810F500005003C00BB99A8008040EB0019
:103FE000E0C1B300BEBE020000000000BBB9A800E3
:103FF0008040EB00C0C1B300BEBE02000000000064
:10400000BBD9A8008040EB0050C2B300BEBE020086
:1040100000000000C0428000E00F5000110032009C
:104020008040EB0090C1B300BEBE02000000000063
:104030008040EB00B0C1B300BEBE02000000000033
:104040008040EB0040C2B300BEBE02000000000092
:104050008040EB00F0C1B300BEBE020000000000D3
:10406000BBF9A800D0428000E00F500005003200EC
:104070008040EB0080C1B300BEBE02000000000023
:10408000BC19A800E0428000E00F5000050032009B
:104090008040EB00A0C1B300BEBE020000000000E3
:1040A000BC39A800B8ED020000000000E00F50008D
:1040B000050032008040EB00E0C0B300BEBE02004D
:1040C00000000000BC59A800C008EC00E20F50003E
:1040D0000B003E00C208EC00E20F500008003E005A
:1040E00020468000F40F5000050034008040EB00B3
:1040F00080C0B300BEBE020000000000BC79A80072
:10410000F0FF2F00F1002000D2CD8000E3CD800031
:10411000800F5100818F590008003A008040EB0069
:1041200020C0B300BEBE02000000000001C2B30008
:1041300030C0B300BEBE020000000000BE19EC009B
:10414000F0CD8800710C2000810F500002003E006D
:104150008100E8006145880072F32F0000014100F2
:10416000610C2000810F510002003E0081F32F00FE
:1041700061458800F2E62F0000014100610C20003B
:10418000810F510003003E00AC28EF008180E80061
:104190007145880072DA2F0000014100610C200097
:1041A000810F510002003E0081F32F00714588000D
:1041B000F2CD2F0000014100E1182000810F5100D5
:1041C00002003E00AE28EF0000000600014B200078
:1041D000810F500001003A00BE39EF0000000600D8
:1041E0000080FB00401388006002AB00FEFF32003D
:1041F0004013800000000600401F200010CE880001
:1042000000C0EB00F6FF070000C0EB00F4FF070062
:10421000E14F40000300320011CE8000E08F5000DB
:10422000F9FF3A0000000600CDC2A80000C0EB0074
:10423000EBFF3700CDC2A900EFFF070011002000FF
:10424000E14F400002003200F7FF07008000EB0062
:104250000100780000000600CDC2A800C9C2A90074
:10426000B0132000101388006422EF0061E2A80060
:1042700000000600EFFF0700EBFF0700C9C2A8001F
:1042800061E2A900DE19A80000000600889FBE00B8
:1042900080047800010478004006200000CE8800E9
:1042A00000C0EB00CEFF070080417800E1CF410065
:1042B00004003A0002CE8000E00F5100F8FF3A00FF
:1042C000220037000001EB00E2CF41001F003A005E
:1042D000F20F2000421388006002AB00FEFF3200A4
:1042E00041138000090078000158780042138800CB
:1042F0006002AB00FEFF32004113800001587800DD
:10430000421388006002AB00FEFF320041138000C0
:1043100001587800421388006002AB00FEFF3200B3
:104320004113800001487800640454000200320008
:104330008004E800E7FF370000C0EB00A8FF07009B
:1043400000C0EB00A6FF070012002000020078006A
:104350004F04BE0000000600889FBE008A1F780040
:104360008004780001447800A3FF07000001EB00FF
:10437000E14F400019003A000840780098FF07001C
:1043800012002000E34F44001400320008202000F7
:104390000905E8001940780091FF07008984E800CA
:1043A0001A4078008EFF07000884E900F8FF3A0001
:1043B00000C0EB008AFF070000C0EB0088FF070089
:1043C00000C0EB0086FF07007F00600012002000A5
:1043D000E50F50000100320008017800020078006B
:1043E0004F0578004F04BE0000000600889FBE0005
:1043F0008A1F7800004578000204BE00E04F550097
:1044000006003D006011B80070C3B300F7FF07005D
:10441000E14F50002A003E000A74A10082FF07000D
:1044200084FF07008000780000C0EB00E08F5000A0
:10443000230032000A4078000064A00068FF0700F3
:104440004848DE000100200065FF07004048DE000C
:104450000100200062FF07004849DD004840DE00FF
:1044600000007100C848DE005DFF070008407800CA
:104470005BFF070050C9B300E04F55000400320055
:104480006E405000E84F55000100320010C0B300EC
:1044900053FF0700EC4F550002003A0000C0EB004C
:1044A0004FFF0700A8C0B30000C0EB004CFF07009F
:1044B000E04F500002003D000844E900FAFF3A00D6
:1044C0004F0578004F04BE00000006000400FA000B
:1044D000889FBE008A1F78008040780010C0B3001B
:1044E000E0CF500088003A00511680000000240000
:1044F000008060008300320057FF070061E2A900DE
:104500001113800030FE2F00008060004001B300D6
:104510001013880011138000C0FF2F00008060007E
:104520000000A0001013880061E2A800A9C0B30039
:1045300000C0EB002AFF07008944E900FCFF3A00B5
:104540006011B80009407800A8FF07000045780016
:1045500009447800E14F550059003A00803E2000A0
:1045600000CE8800A21A20000300200080C0B30003
:104570009EFF0700E14F500033003A0000C0EB00FF
:1045800017FF07008880FB00804178006A81570090
:1045900003F178000844E800E34F5400F7FF3600C9
:1045A0000044EB000FF89700E14F500044003A0040
:1045B000A0CAB3009FF8970080CF500040003A0097
:1045C00000CE8000E00F5000060032000200200004
:1045D0000300240090CAB30084FF0700E04F50009E
:1045E000F7FF3A0008CE8000E00F5400340032009C
:1045F0006011B800A0C3B3007CFF07000044EB00CB
:10460000884F50002E003A0000C0EB00F4FE070077
:104610008980FB00804178006A81570003F17800AF
:104620008944E800E3CF5400F7FF3600EFF097002D
:104630000180FB000004B20048C0B300200032003B
:10464000C8C0B3001E0037006011B80090CAB300A4
:1046500066FF070028C0B30099CAB300E14F5000BD
:10466000020036000A4478008844780000CE8000BA
:10467000E00F5000050032006011B80009407800DA
:104680005AFF0700E04F5000F8FF3A0000CE8000CC
:10469000E00F50000700320002202000030020003D
:1046A00000C1B30051FF0700E04F500003003A0083
:1046B0000300370000447800010037000044EB009D
:1046C0000880FB0020CE8800D7FE0700E04F540092
:1046D0000B003200DE19A90061E2A900111380006D
:1046E00030FE2F00008060008001B30010138800AE
:1046F000300020006222B70061E2A800010037000C
:10470000DCFE0700DED9BF004F0578004F04BE0075
:104710000080FA00000006008040780010C0B3005E
:10472000E0CF500001003A00DED9BF0000000600D3
:10473000889FBE008A1F78008104780004447800B6
:1047400044002000E04F50002F003A00E04F54009A
:104750002D003200DED9BF0061006000340020006F
:1047600029003A00C479AB0004003A004918DD0082
:10477000C711DE00830170004911DD00E14F5400D4
:104780000B003A0010C1B30018FF07000045780085
:10479000E04F550018003A00012020000900780081
:1047A000BAFE0700E00F500012003A001200370076
:1047B00020C1B3000DFF0700E04F50000E003A008B
:1047C0000120200009007800B0FE0700E00F500033
:1047D000040032000844E900020032000920B00061
:1047E000F7FF37006011B800C0C0B300FFFE07003C
:1047F000010037000A4478008BFE07000882FB00A6
:104800000402EA004F22DE00040078004F05780021
:104810004F04BE0000000600889FBE008A9FBE00B5
:10482000810578000204BE000445780042002000A3
:10483000E04F500040003A00E04F55003E0032008B
:10484000DED9BF0061006000320020003A003A006B
:10485000DED9BF00640060002200200036003A006C
:1048600020CE8000E800600004003A00C948DD0066
:10487000C744DE00898470004944DD00E14F5500E3
:104880000C003A000801BE0080C1B300D7FE07004B
:1048900000447800E04F540023003A00E1CFB30019
:1048A0000B007800ACFE0700E00F50001B003A0040
:1048B0001D00370066006000040032000A81FB0022
:1048C0000300200070C9B300C8FE07000801BE0045
:1048D00090C1B300C5FE0700E04F500012003A003F
:1048E000C1CFB3000B0078009BFE0700E00F500023
:1048F000040032000A45E900020032000B20B0003B
:10490000F7FF3700D1CFB3000000EB0092FE0700A5
:10491000E00F500003003200030037000845780024
:10492000010037001AC0B3003FFE07000A81FB00F8
:104930000201EA004F11DE00020078004F05BE00C0
:104940004F04BE00000006001000FA00889FBE0061
:104950008A9FBE0080417800014078008204780080
:1049600048002000E0CF5100D4003A00E19D210032
:1049700091407800E180600038002000CF003A00CC
:104980000080FB0001002000EE0F5000E08F580077
:10499000C8003E00006001000E0037001300370021
:1049A000480037004A003700C2003700C100370016
:1049B000C0003700BF003700BE003700BD00370021
:1049C0008E00370091003700930037009A003700BF
:1049D000A800370017FE070018002000E00F500065
:1049E000B500320010FE0700860037006011B800E5
:1049F00090C0B3007DFE070018002000E04F50007B
:104A0000AD003A0001012000788057001FFE07002A
:104A1000E00F5000A80032000FE897008080FB00F4
:104A2000C608DE000FF09700E1CF50000B003A00FF
:104A30001FF197000281FB00080141004800DD00E2
:104A400000014100030020004A18DD00C610DE000E
:104A5000810070004A10DD003C0037000080FB0040
:104A60004600DE00FFE897008180FB00C208DD0001
:104A7000010040000000E800EFE89700E3806000DC
:104A8000CA08DD0001004000010020005FEA970035
:104A90006F426200AFF197008381FB00C719DE000F
:104AA0008341420083C1E8001FF197006341610028
:104AB0000241410002C141000281FB006901510035
:104AC0001D00370000202000800C78004D003700CA
:104AD0002BCE8000648565001E0032006011B80096
:104AE000D0C8B30041FE070018002000E04F50007E
:104AF00071003A0000C0EB00B9FD07000101200081
:104B000078805700E1FD0700E00F50006A00320096
:104B100008C3B30000C0EB00B1FD07000844E90082
:104B2000FCFF3A002FF197000281FB004411DE00E8
:104B300000012000010020000201E9000300330011
:104B40000000400081804800FBFF3700808CBE00E1
:104B50002C0037006011B80090C0B30023FE07009E
:104B600018002000E04F500053003A0001012000DF
:104B700078805700C5FD0700E00F50004E0032005E
:104B8000628465002FF19700BFF097000F0032009C
:104B90000180FB004700DE000000E800F203B200E5
:104BA0000201410002004000DFF197008381FB0019
:104BB000C619DE008301E9000300DD0001002000CA
